:100000000C94890E0C94AA0E0C94AA0E0C94AA0EB1
:100010000C94AA0E0C94AA0E0C94AA0E0C94AA0E80
:100020000C94AA0E0C94AA0E0C9442630C945F6379
:100030000C94AA0E0C94AA0E0C9420640C944D649B
:100040000C947A640C94A7640C94D4640C940165A9
:100050000C942E650C945B650C9488650C94B565C6
:100060000C94AA0E0D943E150D9475150C94AA0EC1
:100070000C94AA0E0C94AA0E0C94AA0E0C94AA0E20
:100080000C94AA0E0C94AA0E0C94AA0E0C94AA0E10
:100090000C94AA0E0C94AA0E0C94AA0E0D94724005
:1000A0000D94A4400D94D6400D9408410C941EF478
:1000B0000C94AA0E0C94AA0E0C94AA0E0C94A4678D
:1000C0000C94D1670C94FE670C942B680C945868C0
:1000D0000C9485680C94B2680C94DF680C940C69DD
:1000E0000C9439690C94AA0E0D9462140D94991411
:1000F0000C94AA0E0C94AA0E0C94AA0E0C94AA0EA0
:100100000C94AA0E0C94AA0E0C9439F70C94AA0E17
:100110000C94AA0E0C94AA0E0C94AA0E0D94AA3F4D
:100120000D94DC3F0D940E400D9440400C94AA0EAB
:100130000C94AA0E0C94E2650C940F660C943C6629
:100140000C9469660C9496660C94C3660C94F066E5
:100150000C941D670C944A670C9477670C94AA0E54
:100160000D94D0140D9407150C94AA0E0C94AA0E9D
:100170000C94AA0E0C94AA0E0C94AA0E0C94AA0E1F
:100180000C94AA0E0C94AA0E0C94AA0E0C94AA0E0F
:100190000C94AA0E0C94AA0E0C94AA0E0C94AA0EFF
:1001A0000C94EBF30C94AA0E0C94AA0E0C94AA0EC9
:1001B0000C9466690C9493690C94C0690C94ED6975
:1001C0000C941A6A0C94476A0C94AA0E0C94AA0E0A
:1001D0000C94AA0E0C94AA0E0C94AA0E0D94AC15B5
:1001E0000D94E3150C94AA0E0C94AA0E0C94AA0E6E
:1001F0000C94AA0E0C94DF750C949A76630FE60F9C
:10020000750FE60F870FE60F990FB30F990FCD0FFC
:10021000CD0F9411A811BC11E211081283127012B3
:1002200083124A124A120F180F1847188418C81858
:100230000518B119CD190A1A68196819BE21C82103
:10024000D221DC21E621F021FA21FF2104220E2215
:100250000E22962696269D269D26B026D3269626E5
:10026000D3269D269D260C270C27142714272927E3
:1002700050270C27502714271427352840284F28AB
:100280006A288028A228E828F1280C29C828C8282C
:10029000805CF75CF75C105CF75CF75CF75CF75C24
:1002A000F75CF75CF75CF75CF75CF75CF75CF75CB6
:1002B000F75CF75C255CF75CF75CF75CF75CF75C78
:1002C000F75CF75C7A5CD85CF75CF75CE55CF75C44
:1002D000F75CF75CF75CF75CF75C935CF75CF75CEA
:1002E000F15CF75CF45CF75CF75CF75CF75CEE5C88
:1002F000F75CF75CF75CF75CF75CF75CF75CF75C66
:10030000F75CF75CF75CF75CF75CF75CF75CF75C55
:10031000F75CF75CF75CF75CF75CF75CF75CF75C45
:10032000F75CF75CF75CF75CF75CF75CF75CF75C35
:10033000F75CF75CF75CF75CF75CF75CF75CF75C25
:10034000F75CF75C7D5CB370B670B970BC70BF7061
:10035000C270C5703278457858786B787E7891781D
:10036000A4789E7D9E7D297D607D607DE17CE17C21
:10037000607D607D607D607D607D607D607D607D95
:10038000607D607D607D607D607D607D607DE17C05
:10039000607D607D607D607D607DAA82EA83E5820C
:1003A0001483EA83EA83EA83EA83EA83EA83EA83BB
:1003B000EA83EA83EA83EA83EA83EA83EA83EA83D5
:1003C000EA83EA83EA83EA83EA83EA83EA83EA83C5
:1003D000EA83EA83EA83EA83EA83EA83EA83EA83B5
:1003E000EA83EA83EA83EA83EA83EA83EA83EA83A5
:1003F000EA83EA83EA83EA83EA83EA838F83EA83F0
:100400004E83EA83EA83AA83EA83EA83EA83EA8360
:10041000EA83EA83EA83EA83EA83EA83EA835D8301
:10042000EA836B83608D908BC98B138C798CC48C21
:10043000D98C0B8D2D8D4E8D138FA08DA88DC58DD4
:10044000048E178E618E838E9A8EAF8E0E8F0E8FD6
:100450000E8F0E8F0E8F0E8F0E8F0E8F0E8F0E8FB4
:10046000C68ECE8ED98EEE8EF48E5BA866A838A886
:1004700044A866A866A866A866A866A866A866A82E
:1004800066A866A866A866A866A866A866A850A812
:1004900066A866A866A866A866A866A866A866A8EC
:1004A00066A866A866A866A866A85BA866A838A815
:1004B00044A866A866A866A866A866A866A866A8EE
:1004C00066A866A866A866A866A866A866A850A8D2
:1004D000BDB2C0B211B311B311B311B311B311B3A3
:1004E00011B311B311B311B311B311B311B311B3EC
:1004F00011B311B311B311B311B3F7B211B311B3F7
:1005000011B311B311B311B3DDB211B311B311B300
:1005100011B311B3C3B211B311B311B311B311B30A
:1005200011B311B311B311B311B311B311B311B3AB
:1005300011B311B311B311B311B3F7B211B311B3B6
:1005400011B311B311B311B3DDB211B311B311B3C0
:1005500011B311B3C3B2BAB5B7B5CCB5CCB5CCB540
:10056000CCB5CCB5CCB5CCB5CCB5CCB5CCB5CCB583
:10057000CCB5CCB5CCB5CCB503B5D6B4F4B4CCB50C
:10058000CCB57AB5BDB4CCB5CCB5CCB5CCB5CCB5C5
:10059000E5B4BDB5CCB5CCB50DB5CCB5CCB5CCB509
:1005A000CCB5CCB5CCB5CCB5CCB5CCB5CCB5CCB543
:1005B000CCB5CCB5CCB5CCB503B5D6B4F4B4CCB5CC
:1005C000CCB57AB5BDB4CCB5CCB5CCB5CCB5CCB585
:1005D000E5B4BDB5CCB5CCB50DB5A2B7E5B7F4B7AC
:1005E000F4B7F4B7F4B7F4B7F4B7F4B7F4B7F4B7B3
:1005F000F4B7F4B7F4B7F4B7D9B6F4B790B78AB78D
:10060000F2B69CB7F4B7F4B702B7D9B6F4B7F4B7FB
:10061000B1B7E6B696B7EAB7F4B7F8B6A7B784B7F6
:10062000FDB6F4B7ACB7D5B6EFB7F4B7F4B7ECB6E0
:10063000F4B7F4B7F4B7F4B7F4B7F4B790B78AB730
:10064000F2B69CB7F4B7F4B702B7D9B6F4B7F4B7BB
:10065000B1B7E6B696B7EAB7F4B7F8B6A7B784B7B6
:10066000FDB6F4B7ACB7D5B6EFB7F4B7F4B7ECB6A0
:10067000B5B6CBBDBBBDBDBDBFBDC1BDC3BDC5BD99
:10068000C7BDE8BDD8BDDABDDCBDDEBDE0BDE2BDA5
:10069000E4BD15BE43BE1DBE43BE1DBE43BE1DBE52
:1006A00043BE1DBE43BE1DBE43BE43BE43BE43BE8E
:1006B00043BE43BE43BE24BE2BBE37BE37BEA2CF11
:1006C000D1CDDDCD28CE59CF3DCE7FCEA3CECCCE61
:1006D00027CF58D658D69AD675D706D8F6D8F8D98F
:1006E000AFDAF8D9C3DBC3DB0FDE0FDE2BDE6CDE47
:1006F0008CDEBBDEF0DE10DFF0DE3FDF74DFCAE150
:10070000FDE130E2B1E225E3ECE3E3E46DE5E3E4AF
:1007100041E652E70D94E4030D94E2010D94FE02CC
:100720000D9466030D947E030D948B024E414E4949
:100730004E495459494E46CDCCCC3D0AD7233C179F
:10074000B7D13877CC2B329595E6241FB14F0A00EC
:100750000020410000C84200401C4620BCBE4CCADC
:100760001B0E5AAEC59D743235304D4F686D003248
:10077000354D4F686D003630487A003530487A0084
:100780004E6F6E2D496E740048692D4C4F004750D6
:10079000530054696D650044697374616E6365004C
:1007A0005075736820427574746F6E00496D706582
:1007B0007269616C004D657472696300494E430053
:1007C000444543004F4E004F4646005B0856084CD8
:1007D00008450839083208260815080708F407E113
:1007E00007327843495053263278444356472641CE
:1007F000435647003278496D702E204349505326A6
:1008000032784443564700506172616C6C656C20CD
:1008100043495053003278496D702E20434950535C
:100820002644435647003278496D702E2043495084
:100830005300347844435647004349505326327896
:100840004443564700327844435647004349505387
:1008500026444356470044435647004349505300FB
:10086000FA103810760FB40EF20D300D6E0CAC0B82
:10087000EA0A280AC7095B119910D70F150F530E02
:10088000910DCF0C0D0C4B0B890AC70953616D708C
:100890006C652F7365633A004552524F52202020F9
:1008A00020202000432D434950532C20522D4349F2
:1008B00050532C2000000000000000000000000049
:1008C0000000000000000000000000000000000028
:1008D0000000000000000000000000000000000018
:1008E0000000000000000000000000000000000008
:1008F00000000000000000000000000000000000F8
:1009000000000000004C6F2D434950532C204869D3
:100910002D434950532C200000000000000000002F
:1009200000000000000000000000000000000000C7
:1009300000000000000000000000000000000000B7
:1009400000000000000000000000000000000000A7
:100950000000000000000000000000000000000097
:10096000000000000000434950532C20000000000C
:100970000000000000000000000000000000000077
:100980000000000000000000000000000000000067
:100990000000000000000000000000000000000057
:1009A0000000000000000000000000000000000047
:1009B0000000000000000000000000000000000037
:1009C00000000000000000414356474C506F6C2C63
:1009D00020414356474C526D732C20414356475299
:1009E000506F6C2C204143564752526D732C20009F
:1009F00000000000000000000000000000000000F7
:100A000000000000000000000000000000000000E6
:100A100000000000000000000000000000000000D6
:100A20000000000000000000522D44435647204FB4
:100A30006E2C204C2D44435647204F6E2C204C6F7B
:100A40002D43495053204F6E2C2048692D43495067
:100A500053204F6E2C20522D44435647204F66663C
:100A60002C204C2D44435647204F66662C204C6F5B
:100A70002D43495053204F66662C2048692D434929
:100A80005053204F66662C2000522D444356472079
:100A90004F66662C204C2D44435647204F66662CEB
:100AA000204C6F2D43495053204F66662C204869D7
:100AB0002D43495053204F66662C20522D444356F7
:100AC00047204F6E2C204C2D44435647204F6E2C10
:100AD000204C6F2D43495053204F6E2C2048692DD8
:100AE00043495053204F6E2C2000432D434950530F
:100AF000204F6E2C20522D43495053204F6E2C20F6
:100B0000432D43495053204F66662C20522D4349B4
:100B10005053204F66662C200000000000000000AB
:100B200000000000000000000000000000000000C5
:100B300000000000000000000000000000000000B5
:100B40000000000000000000000000432D43495059
:100B500053204F66662C20522D43495053204F6638
:100B6000662C20432D43495053204F6E2C20522D8C
:100B700043495053204F6E2C20000000000000001D
:100B80000000000000000000000000000000000065
:100B90000000000000000000000000000000000055
:100BA000000000000000000000000000522D44433F
:100BB0005647204F6E2C204C6F2D43495053204FE9
:100BC0006E2C2048692D43495053204F6E2C2052E3
:100BD0002D44435647204F66662C204C6F2D4349C9
:100BE0005053204F66662C2048692D4349505320AE
:100BF0004F66662C2000000000000000000000008E
:100C000000000000000000000000000000522D4421
:100C1000435647204F66662C204C6F2D4349505356
:100C2000204F66662C2048692D43495053204F665B
:100C3000662C20522D44435647204F6E2C204C6F7B
:100C40002D43495053204F6E2C2048692D43495065
:100C500053204F6E2C200000000000000000000018
:100C600000000000000000000000000000004C6FC9
:100C70002D43495053204F6E2C2048692D43495035
:100C800053204F6E2C204C6F2D43495053204F66FC
:100C9000662C2048692D43495053204F66662C200E
:100CA0000000000000000000000000000000000044
:100CB0000000000000000000000000000000000034
:100CC0000000000000000000000000000000004CD8
:100CD0006F2D43495053204F66662C2048692D43A1
:100CE000495053204F66662C204C6F2D434950537A
:100CF000204F6E2C2048692D43495053204F6E2CB5
:100D000020000000000000000000000000000000C3
:100D100000000000000000000000000000000000D3
:100D200000000000000000000000000000000000C3
:100D3000522D44435647204F6E2C204C2D44435691
:100D400047204F6E2C20462D44435647204F6E2C93
:100D500020422D44435647204F6E2C20522D4443B1
:100D60005647204F66662C204C2D44435647204F53
:100D700066662C20462D44435647204F66662C203D
:100D8000422D44435647204F66662C200000000049
:100D900000522D44435647204F66662C204C2D446C
:100DA000435647204F66662C20462D444356472025
:100DB0004F66662C20422D44435647204F66662CD2
:100DC00020522D44435647204F6E2C204C2D444337
:100DD0005647204F6E2C20462D44435647204F6ED9
:100DE0002C20422D44435647204F6E2C20000000FB
:100DF0000000522D44435647204F6E2C204C2D446A
:100E0000435647204F6E2C2043495053204F6E2CA1
:100E100020522D44435647204F66662C204C2D44CB
:100E2000435647204F66662C2043495053204F6657
:100E3000662C200000000000000000000000000000
:100E400000000000000000000000000000000000A2
:100E5000000000522D44435647204F66662C204C1C
:100E60002D44435647204F66662C2043495053205B
:100E70004F66662C20522D44435647204F6E2C203F
:100E80004C2D44435647204F6E2C2043495053204D
:100E90004F6E2C2000000000000000000000000049
:100EA0000000000000000000000000000000000042
:100EB00000000000522D44435647204F6E2C204C1A
:100EC0002D44435647204F6E2C20522D4443564705
:100ED000204F66662C204C2D44435647204F6666B3
:100EE0002C200000000000000000000000000000B6
:100EF00000000000000000000000000000000000F2
:100F000000000000000000000000000000000000E1
:100F10000000000000522D44435647204F66662CC7
:100F2000204C2D44435647204F66662C20522D44BA
:100F3000435647204F6E2C204C2D44435647204F9C
:100F40006E2C2000000000000000000000000000E7
:100F50000000000000000000000000000000000091
:100F60000000000000000000000000000000000081
:100F7000000000000000522D44435647204F6E2CC5
:100F80002043495053204F6E2C20522D4443564746
:100F9000204F66662C2043495053204F66662C2014
:100FA0000000000000000000000000000000000041
:100FB0000000000000000000000000000000000031
:100FC0000000000000000000000000000000000021
:100FD00000000000000000522D44435647204F6699
:100FE000662C2043495053204F66662C20522D44D6
:100FF000435647204F6E2C2043495053204F6E2CB0
:1010000020000000000000000000000000000000C0
:1010100000000000000000000000000000000000D0
:1010200000000000000000000000000000000000C0
:101030000000000000000000522D44435647204F9E
:101040006E2C20522D44435647204F66662C2000BC
:101050000000000000000000000000000000000090
:101060000000000000000000000000000000000080
:101070000000000000000000000000000000000070
:101080000000000000000000000000000000000060
:10109000000000000000000000522D44435647208D
:1010A0004F66662C20522D44435647204F6E2C200D
:1010B0000000000000000000000000000000000030
:1010C0000000000000000000000000000000000020
:1010D0000000000000000000000000000000000010
:1010E0000000000000000000000000000000000000
:1010F0000000000000000000000043495053204F52
:101100006E2C2043495053204F66662C200000006F
:1011100000000000000000000000000000000000CF
:1011200000000000000000000000000000000000BF
:1011300000000000000000000000000000000000AF
:10114000000000000000000000000000000000009F
:101150000000000000000000000000434950532040
:101160004F66662C2043495053204F6E2C200000C0
:10117000000000000000000000000000000000006F
:10118000000000000000000000000000000000005F
:10119000000000000000000000000000000000004F
:1011A000000000000000000000000000000000003F
:1011B00000000000000000000000000044656C61B9
:1011C000792054696D653B0046696C65204E616D00
:1011D000653A2000436861696E6167652C200000F4
:1011E0004C6F63616C54696D652C204C6F63616C4E
:1011F000444D592C204C61742D4465672C204E536E
:101200002C204C6F6E2D4465672C2045572C2046B2
:101210006978537461742C204E756D5361742C2061
:1012200050444F502C20416C745F4D2C2043686B10
:101230002C20436F6D6D00000000000000000000D6
:10124000000000000000000000000000000000009E
:10125000000000000000000000000000004C6F6370
:10126000616C54696D652C204C6F63616C444D5901
:101270002C204C61742D4465672C204C61742D4DDD
:10128000696E2C204C61742D5365632C204E532CB9
:10129000204C6F6E2D4465672C204C6F6E2D4D6970
:1012A0006E2C204C6F6E2D5365632C2045572C20DF
:1012B000466978537461742C204E756D5361742C9B
:1012C0002050444F502C20416C745F4D2C204368BB
:1012D0006B2C20436F6D6D000000484558434F5202
:1012E0004445522043414C4942482E545854000032
:1012F000007777772E636174682D746563682E6359
:101300006F6D0000000000004C494D4954454420D9
:101310003930352D3835372D313035300000004328
:101320004154484F44494320544543484E4F4C4F45
:1013300047590000007B702C30302C662C007B70ED
:101340002C30302C657D007B702C30302C6F7D0074
:10135000456E746572204143564720282746272052
:10136000666F722046726F6E742C202742272066AB
:101370006F72204261636B290A0D20616E642073D5
:101380007570706C79203332302B363430207369AD
:101390006E65776176652077697468205065616B4A
:1013A000546F5065616B20766F6C74616765206F58
:1013B0006620302E385600456E7465722053434FB8
:1013C000504520766F6C7461676520696E206D569C
:1013D00020284E4E4E4E4E2900456E7465722043B5
:1013E00049505320766F6C7461676520696E206D7B
:1013F000562A313020284E4E4E4E4E2900456E74EE
:101400006572204443564720766F6C74616765208F
:10141000696E206D562A313020284E4E4E4E4E2990
:1014200000571450144C144814441440143114310F
:1014300014432D53474E44205B352D3430565D0008
:10144000432D4200432D4600432D5200432D4C00B6
:10145000522D53474E4400432D53474E44002061C4
:101460006E6420656E74657220766F6C746167655A
:1014700020696E206D562A313020284E4E4E4E4E39
:101480002900506C6561736520636F6E6E656374CF
:1014900020004572726F722C206D697373696E67DC
:1014A00020414443206E756D2028302D3729000AD5
:1014B0000D5363616C696E6743616C6962204F66AE
:1014C000667365743A20004572726F722C20656EE7
:1014D00074657220766F6C7461676520696E206D2B
:1014E000562A313020284E4E4E4E4E29009B157CF8
:1014F0001566155A1536152315FB1443535B302F0B
:10150000312F322F332F345D5B76767676765D2001
:101510002D204443205363616C696E672043616CE6
:101520006962004342202D20426174746572792003
:1015300043616C696200435A5B302F312F322F3385
:101540002F345D202D204443205A65726F4F66660C
:101550007365742043616C69620056202D20566EBD
:10156000756D626572004C5B696E785D5B4F4E2FE6
:101570004F46465D202D204C65647300416E6E2001
:101580002D2052656164204144433120666F7220F2
:101590006E6E207365636F6E64730041202D205260
:1015A0006561642041444331004552524F52004F1F
:1015B0004B00434154482054454348204845584334
:1015C0004F52444552205630302E39390001000226
:1015D0000003000400050006000A000C000F0014C0
:1015E000001E003C007800B400F0002C01680100EF
:1015F0000000000B0002000100B80B0F270100647F
:10160000006801100E010010271027102710271066
:101610002710270100010001000100F8010100016D
:101620000002000100F401000000000100000000C1
:10163000000A00F1D8000001000100C800000064A9
:1016400000640064006400640064000000000000A6
:1016500000000050FE00000000000000000100003B
:101660000000000100000000000A0000000100016D
:1016700000020058020000FA00FA00FA00FA0078AE
:1016800000780000000000000001000000010001DF
:10169000000000000001000100008000190080002F
:1016A00019008000190080001900800019008000D6
:1016B00019008000190080001900000100FF03E6F6
:1016C00000E600F916EB16DD16D616244A42494EFE
:1016D0002C39342C3100244A5341564500244A41C8
:1016E00053432C47504753412C3100244A41534324
:1016F0002C4750524D432C3100244A4153432C4730
:10170000504747412C310024504D544B3636372A30
:1017100033350024504D544B3331342C302C312C84
:10172000302C312C312C302C302C302C302C302CD7
:10173000302C302C302C302C302C302C302C302CC9
:10174000302A323900756E6C6F67206C62616E648E
:10175000747261636B7374617461006C6F67206C89
:1017600062616E64747261636B7374617461206F23
:101770006E74696D6520313000756E6C6F67207016
:101780007372706F7361006C6F6720707372706F2B
:101790007361206F6E74696D65203130006461740F
:1017A000756D20757365720020302E3020302E301C
:1017B00020302E3020302E300075736572646174D5
:1017C000756D2000646174756D207767733834001F
:1017D000756E6C6F67206770616C6D006C6F672051
:1017E0006770616C6D206F6E74696D6520313000BB
:1017F00059184A183B182C1824180B18FE17245097
:1018000047524D432C2C2C39362C00245047524D36
:10181000432C412C2C3130302C2C2C2C2C2C2C2CCF
:101820002C2C2C00245047524D4345002450475245
:101830004D4F2C5047524D542C3000245047524DA0
:101840004F2C5047524D462C3100245047524D4F9B
:101850002C47504753562C3000245047524D4F2CA4
:101860002C3400BA18AB189C188D187E186F1844C9
:101870005A203D20000000000000000000004459F4
:10188000203D20000000000000000000004458201F
:101890003D2000000000000000000000466C617464
:1018A000203D2000000000000000004D616A6F72C2
:1018B00041203D20000000000000535450522044BD
:1018C0004154554D2E54585400061AF919EC19DF9D
:1018D00019D219C519B819AB199E1991198419771C
:1018E000196A195D1950194319361929191C190F4C
:1018F000190219F518414356473220524D53203DE5
:101900002000414356473120524D53203D20004294
:10191000415454202043616C203D2000414320204D
:10192000205343616C203D200041432020205A4336
:10193000616C203D200041444337205653636C20A6
:101940003D200041444337205A43616C203D200034
:1019500041444336205653636C203D2000414443AC
:1019600036205A43616C203D2000414443352056C7
:1019700053636C203D200041444335205A43616C41
:10198000203D200041444334205653636C203D20C9
:101990000041444334205A43616C203D20004144BF
:1019A0004333205653636C203D2000414443332091
:1019B0005A43616C203D200041444332205653631A
:1019C0006C203D200041444332205A43616C203D4D
:1019D000200041444331205653636C203D20004198
:1019E000444331205A43616C203D20004144433040
:1019F000205653636C203D200041444330205A431D
:101A0000616C203D200046696C6520496E646578F4
:101A1000203D2000B41C9E1C881C721C5C1C461CB3
:101A2000301C1A1C041CEE1BD81BC21BAC1B961BC3
:101A3000801B6A1B541B3E1B281B121BFC1AE61A38
:101A4000D01ABA1AA41A8E1A781A621A454E44008D
:101A50000000000000000000000000000000000086
:101A60000000444356472044656665637420566110
:101A70006C203D200000000044435647204465662A
:101A800065637420456E203D2000000000005379FE
:101A90006E632054797065203D2000000000000036
:101AA00000000000434950532052616E6765202BAF
:101AB0002F2D3556203D2000000047505320436F06
:101AC0006F726420696E20444D53203D2000000059
:101AD0004C6F63616C47505354696D654F66667314
:101AE0006574203D20004143204672657175656E26
:101AF0006379203D200000000000000042726F6BFF
:101B0000656E5769726520416C61726D203D2000E1
:101B100000004C6F7720506F7420416C61726D2013
:101B20003D20000000000000496E70757420496D72
:101B3000706564616E6365203D20000000004443D1
:101B400056474D44656C4F4E203D2000000000007C
:101B500000000000444356474D44656C4F46462004
:101B60003D20000000000000000043495053324D6A
:101B700044656C4F4E203D20000000000000000036
:101B800043495053324D44656C4F4646203D20003A
:101B900000000000000043495053314D44656C4F34
:101BA0004E203D200000000000000000434950533B
:101BB000314D44656C4F4646203D2000000000003A
:101BC0000000537461727457697468203D200000EE
:101BD00000000000000000004F666654696D65203B
:101BE0005B6D7365635D203D200000000000546F55
:101BF00074616C4379636C65205B7365635D203D44
:101C00002000000054696D652056616C7565203DAB
:101C100020000000000000000000436861696E6160
:101C2000676520446972656374696F6E203D2000AA
:101C3000537461727420436861696E616765203D09
:101C400020000000000044697374616E63652056D3
:101C5000616C7565203D2000000000004D656173DA
:101C60007572656D656E7420556E697473203D20C4
:101C7000000053746F7261676520416374696F6E11
:101C8000203D2000000000005375727665792054D5
:101C9000797065203D2000000000000000004F70BA
:101CA000657261746F72204E616D65203D20000089
:101CB00000000000537572766579204E616D6520D5
:101CC0003D20000000000000000054532D5453201C
:101CD0004F4E203D200054532D5453204F46462054
:101CE0003D20004E4557205453204F4E203D2000AC
:101CF0004E4557205453204F4646203D2000545314
:101D0000204F4E203D20005453204F4646203D207A
:101D1000000011241FBECFEFCDBFDFE5DEBF00E026
:101D20000CBF1DE2A0E0B0E2E8E4F4E902E00BBF82
:101D300002C007900D92A63FB107D9F722E5A6EFA2
:101D4000BDE201C01D92A633B207E1F70E94CE3B6F
:101D50000D94224A0C940000CF93DF93CDB7DEB7E9
:101D60002B97CDBFDEBFBE016F5F7F4F80E092E05B
:101D70000F948A41AE01485F5F4F68E080E092E0D7
:101D80000F94E6418A819B819F789B8395E09D8398
:101D9000817E8A831C82BE016F5F7F4F80E092E06C
:101DA0000F943A4181E0888788E18987AE01485FD6
:101DB0005F4F68E080E092E00F94AD4180E092E0F8
:101DC0000F949B3F2B96CDBFDEBFDF91CF9108953F
:101DD0009FB7F894E0E0F2E08081806280839FBF4B
:101DE0000895009781F02091060223FF0EC02091F4
:101DF0003C0230913D02FC012083318388E08093D6
:101E0000060281E0089580E0089580E00895CF9271
:101E1000DF92EF92FF92CF93DF930097D1F061159D
:101E20007105C9F0EB01FC01A081B18128EE33E01E
:101E30000F943A456B017C0183E10E94DFB89B015E
:101E4000AC01C701B6010F94E5442883398381E0D2
:101E500003C080E001C080E0DF91CF91FF90EF9060
:101E6000DF90CF900895E6EEF6E31082118214829F
:101E7000158212821382168217828BE00E9403B9A8
:101E8000672B682B692B19F41092EE3603C081E0A2
:101E90008093EE36E6EEF6E3118612860895CF9330
:101EA000DF93EC01892B09F491C0862F90E0FC01AF
:101EB0003197EB30F10508F089C08827E250FF4FD9
:101EC0008F4F0D9423458091EE36811107C0888194
:101ED00099818093EA369093EB3678C08A819B8112
:101EE0008093EA369093EB3671C08091EE36811183
:101EF00007C08A819B818093EA369093EB3666C057
:101F00008E819F818093EA369093EB365FC08091FB
:101F1000EE36811107C08C819D818093EA369093C3
:101F2000EB3654C08A859B858093EA369093EB36D6
:101F30004DC08091EE3681110BC088819981E6EE0B
:101F4000F6E3848395838A819B81868397833EC051
:101F50008C819D81E6EEF6E3848395838E819F815B
:101F60008683978333C08091EE3681110BC08A81BE
:101F70009B81E6EEF6E3848395838C819D81868345
:101F8000978324C0E6EEF6E388859985848395835C
:101F90008A859B858683978319C08091EE3681114F
:101FA0000BC08C819D81E6EEF6E3848395838E8160
:101FB0009F81868397830AC0E6EEF6E38C859D8534
:101FC000848395838E859F8586839783DF91CF91C8
:101FD0000895E6EEF6E3848195818083918386817E
:101FE0009781828393830895E6EEF6E381E081870B
:101FF00012860895E6EEF6E3118612860895809122
:10200000F036089583E10E9403B9672B682B692B92
:1020100019F08091EF36089580E00895CF92DF9215
:10202000EF92FF926B01072E000CEE08FF08C2161C
:10203000D306E406F5067CF486179707E4F0092E2C
:10204000000CAA0BBB0BE1E0281739074A075B0716
:10205000ACF4E0E013C06C01092E000CEE08FF08A0
:10206000C216D306E406F50644F0E1E068177907E6
:102070002CF4E0E003C0E0E001C0E0E08E2FFF9030
:10208000EF90DF90CF900895FF920F931F93CF931F
:10209000DF93C6EED6E30AEE16E3F12CE991F9914F
:1020A000309719F1AF010F2E000C660B770BDB0197
:1020B000CA0177231CF40196A11DB11DB595A79502
:1020C000979587959A01AB01280F391F4A1F5B1F0F
:1020D000BF01FF2314F46F5F7F4F759567958A8169
:1020E0009B819CDF813009F0F394C017D107B1F6D2
:1020F000FF2011F079DF01C07DDF6BDFDF91CF9131
:102100001F910F91FF900895E6EEF6E381E090E0D5
:10211000A0E0B0E08787908BA18BB28B838B948BF0
:10212000A58BB68B178A1386148615861686108E95
:102130000895E6EEF6E381E0878B108E0895E6EED3
:10214000F6E3178A108E08958091FE36089584E193
:102150000E9403B9672B682B692B19F08091FD361B
:10216000089580E00895E6EEF6E387859089A189D9
:10217000B289838B948BA58BB68B83859485A5853B
:10218000B6858787908BA18BB28B08956093F136CB
:102190007093F2368093F3369093F43608958F92CD
:1021A0009F92AF92BF92CF92DF92EF92FF92E6EEB4
:1021B000F6E3C388D488E588F68887859089A18965
:1021C000B289C816D906EA06FB0691F48090F1366A
:1021D0009090F236A090F336B090F436C4DFC81475
:1021E000D904EA04FB0411F4A4DF04C0A8DF02C090
:1021F000BADFFCCFFF90EF90DF90CF90BF90AF9011
:102200009F908F9008958BE10E9403B96093FF36F1
:10221000709300378093013790930237A3E0B7E3C0
:10222000E6EEF6E38EEE96E31D9211A212A232962E
:102230008E179F07C9F7E6EEF6E311A612A60895DA
:1022400081E090910F37911101C080E008958AE1FB
:102250000E9403B9672B682B692B39F081E09091BC
:102260000F37911103C080E0089580E008950F9327
:102270001F938B019C018091FF3690910037A091B4
:102280000137B09102370097A105B10529F1880FF8
:10229000991FAA1FBB1FAC01BD01440F551F661F2C
:1022A000771F440F551F661F771F840F951FA61FAA
:1022B000B71FB901A80133233CF444275527BA01BD
:1022C000401B510B620B730B21E084179507A60787
:1022D000B7071CF020E001C020E0822F1F910F9172
:1022E00008950F931F93CF93DF93009709F40BC1C9
:1022F000A6EEB6E35D961C925D975E961C925E9785
:102300005F961C925F9790961C92462F50E0FA01C0
:102310003297EA30F10508F0F6C0EC018827E75F54
:10232000FE4F8F4F0D9423458091EE36811108C0EA
:102330006C817D818E819F819ADF80930337E3C01A
:10234000688179818A819B8192DF80930337DBC02A
:102350008091EE36811108C0688579858A859B85D4
:1023600086DF80930337CFC0688179818A819B8122
:102370007EDF80930337C7C08091EE36811111C094
:10238000688579858A859B8572DF06EE16E3F801FC
:10239000858F6C857D858E859F8569DFF801868FA9
:1023A000B2C0688179818A819B8161DF06EE16E384
:1023B000F801858F6C817D818E819F8158DFF801C6
:1023C000868FA1C08091EE36811111C06C857D850C
:1023D0008E859F854CDF06EE16E3F801858F6889B0
:1023E00079898A899B8943DFF801868F8CC068814F
:1023F00079818A819B813BDF06EE16E3F801858FA8
:102400006C817D818E819F8132DFF801868F7BC058
:102410008091EE3681111FC0688979898A899B89EC
:1024200026DF06EE16E3F801858F6C897D898E899B
:102430009F891DDFF801868F688D798D8A8D9B8D30
:1024400016DFF801878F6C8D7D8D8E8D9F8D0FDF50
:10245000F80180A358C0688179818A819B8107DF58
:1024600006EE16E3F801858F6C817D818E819F8158
:10247000FEDEF801868F688579858A859B85F7DE83
:10248000F801878F6C857D858E859F85F0DEF8014C
:1024900080A339C08091EE36811111C06889798995
:1024A0008A899B89E4DE06EE16E3F801858F6C8944
:1024B0007D898E899F89DBDEF801868F24C0688143
:1024C00079818A819B81D3DE06EE16E3F801858F40
:1024D0006C817D818E819F81CADEF801868F13C059
:1024E0008091EE36811108C06C857D858E859F8533
:1024F000BEDE8093033707C0688179818A819B8122
:10250000B6DE80930337DF91CF911F910F9108952D
:10251000843040F5E6EEF6E341A552A5242F30E0E5
:10252000082E02C0359527950A94E2F720FF0AC0CD
:10253000252F30E0082E02C0359527950A94E2F742
:1025400020FD10C021E030E0B90102C0660F771F06
:102550008A95E2F7CB01E6EEF6E3462B41A780959C
:10256000852382A70895843090F421E030E0A9010A
:1025700002C0440F551F8A95E2F7CA018095E6EE26
:10258000F6E391A5982391A792A5892382A70895A0
:10259000BF92CF92DF92EF92FF920F931F93CF9350
:1025A000DF9303E017E3C6EED6E36E017801B12CAA
:1025B000F70181917F01F60121A190E0820F911D29
:1025C00022A1820F911D039719F48B2DA1DF02C068
:1025D0008B2DC9DFB394F2E0CF0ED11C84E0B8128A
:1025E000E7CF2EEE36E389A18AA3F80181918F010E
:1025F00089A32296C217D307B1F7DF91CF911F911C
:102600000F91FF90EF90DF90CF90BF9008958430AE
:1026100060F420910F3730E0A90102C0559547952D
:102620008A95E2F7CA018170089580E008958430A8
:1026300060F42091103730E0A90102C0559547950C
:102640008A95E2F7CA018170089581E00895843087
:1026500000F5662379F0E6EEF6E321E030E0A9012B
:1026600002C0440F551F8A95E2F7CA0192A5892B33
:1026700082A70895E6EEF6E321E030E0A90102C06A
:10268000440F551F8A95E2F7CA01809592A58923C8
:1026900082A70895CF93833009F128F4813031F077
:1026A000823061F02CC0883008F129C08091FD365D
:1026B000882329F181E08093FE3621C0C1DD882383
:1026C000F1F061E080E0C3DF61E081E0C0DF61E064
:1026D00082E0BDDF61E083E0BADF11C08091EF36B8
:1026E000882369F081E08093F03609C0CCEFC80FF1
:1026F0008C2F8DDF882319F061E08C2FA8DFCF911C
:102700000895009781F0FC01DC01AE5BBD4F808134
:102710008C936083643021F481E00C94F6F7089583
:1027200080E00C94F6F70895009719F0FC01808181
:10273000089580E008950F931F93CF93DF931F9226
:10274000CDB7DEB7009709F4C0C08C0181E0D80195
:102750008C9311961C92119712961C9212971396B5
:102760001C92139714961C92149715961C92159709
:10277000169682E1E5E0F4E201900D928A95E1F788
:10278000C80148960E9401BFF801808D8783818D22
:102790008087828D8187838D8287CE0101960E94FA
:1027A00022BF89818B3429F481E0D8015C968C9317
:1027B00002C0F801148E80E00E94DFB8673EF3E0AB
:1027C0007F078105910514F59F938F937F936F93F6
:1027D00083EE90E29F938F93C801C5969F938F934A
:1027E0000F945047D801D5968C91D59750968C93DD
:1027F0005097D6968C91D69751968C935197D796A1
:102800008C91D79752968C93CDBFDEBFD8015D9641
:102810001C925D975E961C925E97D1961C92D19702
:10282000D2961C92F801EB5CFD4F1082319610821B
:1028300031961082319681E0808331961082118228
:1028400012821382349681E090E0A0E0B0E08083B1
:102850009183A283B383349610823196D8018C91F0
:102860008083E751F24086E0DF011D928A95E9F707
:10287000E85EFD4F108211823296108211823296EC
:102880001082118232961082118232961082319615
:1028900010823296108231961082319610823196D3
:1028A00010823196108231961082319610821182F8
:1028B00012821382349610823196108231961082E1
:1028C000319688E690E1808391830F90DF91CF91DC
:1028D0001F910F910895009741F0613021F421E09C
:1028E000FC0121AB0895FC0111AA0895009719F08D
:1028F000FC0181A9089580E00895009741F06130BE
:1029000021F421E0FC0122AB0895FC0112AA0895F4
:10291000009719F0FC0182A9089580E008958F9234
:102920009F92AF92BF92DF92EF92FF920F931F930D
:10293000CF93DF934115510509F46BC08A017B01E8
:10294000C82F0E94B0BDD82F8C2F0E94CDBDD82E8D
:10295000DD2309F460C0882309F45FC08D2F0E9435
:10296000DFB84B015C018D2D0E94DFB8672B682B0F
:10297000692B39F4F801108211821282138280E0EF
:102980004DC09701280D391D032E000C440B550B2B
:10299000C63050F4A0E1B7E20F944045F8016083DF
:1029A00071838283938309C0A8EEB3E00F944045FE
:1029B000F80160837183828393838D2D0E94DFB839
:1029C0009B01AC01F80160817181828193810F9438
:1029D000074588279927DC01821B930BA40BB50BB5
:1029E000F80180839183A283B3838C2F0E9483C0DC
:1029F000F80180809180A280B380DC01CB01880D3A
:102A0000991DAA1DBB1D80839183A283B38381E09E
:102A100005C080E003C080E001C080E0DF91CF917D
:102A20001F910F91FF90EF90DF90BF90AF909F901C
:102A30008F900895CF93DF93009709F460C0EC0165
:102A40000F94100A813091F58C830E94DDF4882365
:102A5000F9F08091113D811119C089E0E9EEF0E2B1
:102A6000A5E5B2E401900D928A95E1F7E5E5F2E47F
:102A700001900020E9F73197AF014555524421E01C
:102A800065E572E483E797E30F9466120E9416F5FA
:102A90000E94E0F4882399F183E496E40E9410C632
:102AA0000E94DAF48A830E9427F529C01C820F94C1
:102AB0003C0A8823F9F08091113D811119C089E009
:102AC000E2EFF0E2A5E5B2E401900D928A95E1F71C
:102AD000E5E5F2E401900020E9F73197AF014555B3
:102AE000524421E065E572E483E797E30F946612B0
:102AF0000F943F0A0F94280A81110F942B0ADF913B
:102B0000CF9108950F931F93CF93DF93009709F40C
:102B100063C0EC010F94870C882381F18B818111B4
:102B20005BC08091113D811126C00F94500A182F6F
:102B30000E94DAF41F921F931F928F9384E091E218
:102B40009F938F9305E512E41F930F930F945047C3
:102B5000F80101900020E9F73197AF014555524443
:102B600020E0B80183E797E30F9466128DB79EB714
:102B700008968DBF9EBF81E08B832EC08B818130F4
:102B800059F51B828091113D811126C00F94500A86
:102B9000C82F0E94DAF41F92CF931F928F938BEF6E
:102BA00090E29F938F93C5E5D2E4DF93CF930F9488
:102BB000504709900020E9F72197AE01455552444E
:102BC00020E065E572E483E797E30F9466128DB722
:102BD0009EB708968DBF9EBFDF91CF911F910F9139
:102BE0000895CF92DF92EF92FF920F931F93CF93AE
:102BF000DF93009709F4AAC06115710509F4A6C016
:102C00008B01EC010E94AEC5882309F49FC00F948C
:102C1000CF0A6B017C010F94740C86E10E9403B90A
:102C2000AB01BC018BEE9AE30E9444C6D701C601FA
:102C30000197A109B109883E9340A105B10508F0AB
:102C40003FC00E9435B2823088F18091113D8111E0
:102C50002DC00E94DAF41F928F938091AB511F9286
:102C60008F93FF92EF92DF92CF9287E191E29F9351
:102C70008F930F2EF5E5EF2EF2E4FF2EF02DFF924D
:102C8000EF920F945047F70101900020E9F7319738
:102C9000AF014555524421E0B70183E797E30F9414
:102CA00066128DB79EB70C968DBF9EBF2AE533E4A2
:102CB00044E755E46EEA74E4C8010E94B7D143C00A
:102CC000D701C601895E9340A109B10984369105F7
:102CD000A105B105C0F584E793E40E94A6C5811162
:102CE00032C08091113D811125C0FF92EF92DF9299
:102CF000CF9283E291E29F938F930F2EF5E5EF2E13
:102D0000F2E4FF2EF02DFF92EF920F945047F7015F
:102D100001900020E9F73197AF014555524421E079
:102D2000B70183E797E30F9466128DB79EB70896B5
:102D30008DBF9EBF2AE533E444E755E46EEA74E4B0
:102D4000C8010E94B7D1CE010E94C7C5DF91CF91C3
:102D50001F910F91FF90EF90DF90CF900895FC01AD
:102D6000892B39F0118689E0DF011D928A95E9F7F8
:102D700012860895FC01892B41F0118689E0DF015C
:102D80001D928A95E9F71286138608950F931F9373
:102D9000CF93DF93C4E1D7E30CE617E3CE01DFDF87
:102DA0002B96C017D107D1F788EA9AE3E3DF84EBCB
:102DB0009AE3E0DFDF91CF911F910F910895FC011D
:102DC000892B31F081E09285913019F080E00895EF
:102DD00080E008951F93CF93DF93CDB7DEB7609760
:102DE000CDBFDEBF9C01FE013196AE014F5E5F4F4D
:102DF00021933193255F3F4FE417F507C9F7892BDE
:102E000031F110E010C0E12FF0E0EE0FFF1F81E084
:102E100090E08C0F9D1FE80FF91F80819181CFDF1B
:102E20008823D1F01F5F0F94740D181760F382E0B0
:102E30000E9403B96B3069F48091B33A882359F04A
:102E400081E09091BF3A911107C080E005C080E019
:102E500003C081E001C080E06096CDBFDEBFDF919E
:102E6000CF911F910895CF92DF92EF92FF920F932F
:102E70001F93CF93DF93CDB7DEB72597CDBFDEBFCE
:102E800019821A821B821C824115510559F16A016F
:102E90007B01182FCA0163DFAE014F5F5F4FB7019F
:102EA000812F3DDD8823C9F009811A812B813C8166
:102EB0004BE0BE016B5F7F4FC6010F948619F60190
:102EC00001900020E9F73197EC19FD09D601199618
:102ED000EC93199781E01A968C9369817A818B81A2
:102EE0009C8103C060E070E0CB012596CDBFDEBFC2
:102EF000DF91CF911F910F91FF90EF90DF90CF90D6
:102F000008958F929F92AF92BF92EF92FF920F938C
:102F10001F93CF93DF930097A1F06115710589F09E
:102F2000142F7B01EC010E9429F84B015C01113048
:102F300009F42CD9950184014BE0B701CE010F941F
:102F4000D817DF91CF911F910F91FF90EF90BF9015
:102F5000AF909F908F900895AF92BF92CF92DF92E3
:102F6000EF92FF920F931F93CF93DF93CDB7DEB70E
:102F70006097CDBFDEBF8C01CE0101967C014096EB
:102F8000F70161937193655F7F4FE817F907C9F700
:102F90000115110509F46BC282E00E9403B9D62E17
:102FA00096E0D91206C0C8010F94CF08811165C2FE
:102FB00039C38FEF8D0D823030F4C8010F94CF08E4
:102FC000811107C02FC3C8010F94CF08882309F4CB
:102FD00029C380E2E4E2FEE3DF011D928A95E9F76E
:102FE00080E1E1E8F9E3DF011D928A95E9F78D2D93
:102FF00090E0FC013197EB30F10508F03AC28827E8
:10300000ED5EFE4F8F4F0D94234558010F2EF4E2D5
:10301000CF2EFEE3DF2EF02D01E010E00EC10F9465
:10302000CC08C82E49815A81F801608171811BDF6B
:103030000F2EF4E2EF2EFEE3FF2EF02DD7016D935D
:103040007D938D939C9313974B815C81F8016281F2
:1030500073818C2D08DFD70114966D937D938D932A
:103060009C931797B2E0DB1206C28091243E9091A8
:10307000253EA091263EB091273E809381399093C2
:103080008239A0938339B093843981E0CBC258014F
:103090000F2EF4E2CF2EFEE3DF2EF02D01E010E044
:1030A0000BC01F5F0F5FE2E0EE0EF11CF2E0AF0E0F
:1030B000B11C84E0C80ED11C112309F4FBC11230ED
:1030C00009F4EAC1D7014D915C91F50160817181EC
:1030D00080E0C9DED6016D937D938D939C93139709
:1030E0000430F8F28091243E9091253EA091263E36
:1030F000B091273E8093813990938239A093833990
:10310000B093843981E08EC258010F2EF4E2CF2EA5
:10311000FEE3DF2EF02D01E010E00BC01F5F0F5F1C
:10312000B2E0EB0EF11CE2E0AE0EB11CF4E0CF0E0B
:10313000D11C112309F4DBC1123009F4CAC1D70133
:103140004D915C91F5016081718182E08CDED60148
:103150006D937D938D939C9313970430F8F2E1E87F
:10316000F9E3A4E2BEE34D915D916D917C911397DB
:10317000408351836283738314968D919D910D904A
:10318000BC91A02D84839583A683B78381E04AC236
:1031900058010F2EF4E2CF2EFEE3DF2EF02D01E0DA
:1031A00010E00BC01F5F0F5FB2E0EB0EF11CE2E01E
:1031B000AE0EB11CF4E0CF0ED11C112309F4B8C13E
:1031C000133009F4A3C1113009F4A2C1143009F479
:1031D000A1C1D7014D915C91F5016081718180E0C1
:1031E00042DED6016D937D938D939C9313970630A9
:1031F000C8F2E1E8F9E3A4E2BEE34D915D916D917F
:103200007C911397408351836283738314968D91CD
:103210009D910D90BC91A02D84839583A683B78347
:1032200081E000C21F5F0F5FB2E0EB0EF11CE2E035
:10323000AE0EB11CF4E0CF0ED11C112309F499C1DC
:10324000143009F484C1812F8B7F813009F481C14E
:10325000823009F480C1D7014D915C91F501608104
:10326000718185E000DED6016D937D938D939C93F3
:1032700013970830B8F2E1E8F9E3A4E2BEE34D9118
:103280005D916D917C911397408351836283738329
:1032900014964D915D916D917C9117974483558360
:1032A0006683778318964D915D916D917C911B9704
:1032B00040875187628773871C968D919D910D90F1
:1032C000BC91A02D84879587A687B78781E0AAC186
:1032D00058010F2EF4E2CF2EFEE3DF2EF02D01E099
:1032E00010E00BC01F5F0F5FB2E0EB0EF11CE2E0DD
:1032F000AE0EB11CF4E0CF0ED11C112309F458C15D
:10330000143009F445C1812F8B7F813009F442C10B
:10331000D7014D915C91F5016081718180E0A3DD61
:10332000D6016D937D938D939C9313970830D0F2C3
:10333000E1E8F9E3A4E2BEE34D915D916D917C91EA
:103340001397408351836283738314968D919D916B
:103350000D90BC91A02D84839583A683B78381E0D3
:1033600061C1680104E21EE35E01B9E0AB0EB11C6D
:10337000F701419151917F01D6016D917D916D01D0
:1033800080E071DDF80161937193819391938F01D6
:10339000EA14FB0469F781E045C158010F2EF4E2FD
:1033A000CF2EFEE3DF2EF02D01E010E00BC01F5FFB
:1033B0000F5FF2E0EF0EF11C82E0A80EB11C94E06A
:1033C000C90ED11C112309F402C1133009F40DC137
:1033D000D7014D915C91F5016081718180E043DD01
:1033E000D6016D937D938D939C9313970630F8F2DD
:1033F0008091243E9091253EA091263EB091273E9B
:103400008093813990938239A0938339B093843922
:1034100081E008C158010F2EF4E2CF2EFEE3DF2E2B
:10342000F02D01E010E00BC01F5F0F5FB2E0EB0E6C
:10343000F11CE2E0AE0EB11CF4E0CF0ED11C112362
:1034400009F4E2C0D7014D915C91F5016081718171
:1034500081E0123009F480E006DDD6016D937D93A2
:103460008D939C9313970430F8F281E0DBC080E0E9
:10347000D9C080E0D7C081E0D5C080E2E4E2FEE3BD
:10348000DF011D928A95E9F780E1E1E8F9E3DF01C8
:103490001D928A95E9F7B9CDF70140815181D50197
:1034A0006D917C9183E0DFDCF60160837183828320
:1034B0009383F7CDD7014D915C91F50160817181C6
:1034C00083E0D1DCD6016D937D938D939C9313970C
:1034D000E8CDF70140815181D5016D917C9183E068
:1034E000C2DCF601608371838283938317CED70198
:1034F0004D915C91F5016081718183E0B4DCD6016E
:103500006D937D938D939C93139708CE83E003C0B6
:1035100082E001C082E0F70140815181D5016D91C7
:103520007C91A1DCF60160837183828393833ACE20
:10353000D7014D915C91F5016081718183E093DC4D
:10354000D6016D937D938D939C9313972BCE83E03F
:1035500003C082E001C084E0F70140815181D501C0
:103560006D917C9180DCF60160837183828393830B
:1035700059CED7014D915C91F5016081718183E055
:1035800072DCD6016D937D938D939C9313974ACEF5
:1035900083E001C082E0F70140815181D5016D9146
:1035A0007C9161DCF60160837183828393839ACE80
:1035B000D7014D915C91F5016081718183E053DC0D
:1035C000D6016D937D938D939C9313978BCEF701CA
:1035D00040815181D5016D917C9183E044DCF601FD
:1035E0006083718382839383E2CED7014D915C9196
:1035F000F5016081718183E036DCD6016D937D93A6
:103600008D939C931397D3CEF70140815181D501BF
:103610006D917C9180E027DCF60160837183828369
:10362000938302CF6096CDBFDEBFDF91CF911F9114
:103630000F91FF90EF90DF90CF90BF90AF900895E3
:103640000F949D06882329F00F94AE0684E08093A2
:1036500027060895CF93DF93009799F1EC018881B5
:103660008130A8F0833018F0863019F010C0E8DF00
:1036700025C08091280682FD03C084E08093250642
:103680000F9437068823D1F00F94480617C00F9483
:103690003706882399F00F94480684E08093270624
:1036A0000DC08D8181110DC00F947B06882349F0D8
:1036B0000F948C0684E08093270603C088818630AF
:1036C00081F7DF91CF9108950E94E8C90F94540BC0
:1036D00020E137E240E050E00F94E544672B682B8F
:1036E000692BE1F40E94E8C9813019F40C94FCC8FC
:1036F00008950E94E8C9823021F481E00C94EBC95E
:1037000008950E94E8C9833019F40C94F1CB089510
:103710000E94E8C9843011F40C9445CC08950F93AD
:103720001F93CF93DF931F921F92CDB7DEB71982FD
:103730001A820097B9F08C010E94FF5190E0069622
:103740009E012F5F3F4F43E060E0800F911F0F9479
:103750003716882339F049815A8160E070E080E0B3
:103760000E94EEB80F900F90DF91CF911F910F91B3
:1037700008959F92AF92BF92CF92DF92EF92FF9205
:103780000F931F93CF93DF931F92CDB7DEB70097B0
:1037900009F44BC05C0182E00E9403B9962E8501BA
:1037A000095D1F4FBE016F5F7F4FC8010E94CBD5DF
:1037B000882391F0F501C7A0D0A4E1A4F2A489E088
:1037C0000E9403B9AB01BC010FEE16E42FED36E405
:1037D00089810F946F0B17C0BE016F5F7F4FC801C7
:1037E0000E94A5DDF501C7A0D0A4E1A4F2A489E060
:1037F0000E9411B9AB01BC010FEE16E42FED36E4C7
:1038000089810F946F0BFBE09F120BC0F50147A15C
:1038100050A561A572A587ED96E40F94540E81E042
:1038200005C00F94BE0E81E001C080E00F90DF91D3
:10383000CF911F910F91FF90EF90DF90CF90BF90AD
:10384000AF909F900895CF92DF92EF92FF920F93E7
:103850001F93CF93DF931F92CDB7DEB7009779F117
:103860008C01BE016F5F7F4F87960E9410E0882316
:1038700099F0F801C7A0D0A4E1A4F2A489E00E94C5
:1038800003B9AB01BC010FEE16E42FED36E48981DC
:103890000F946F0B81E014C0F801C7A0D0A4E1A47D
:1038A000F2A489E00E9411B9AB01BC010FEE16E44D
:1038B0002FED36E489810F946F0B81E001C080E029
:1038C0000F90DF91CF911F910F91FF90EF90DF90BC
:1038D000CF90089589E10E9403B9623059F482E0E3
:1038E0000E9403B9673041F0693031F0613021F056
:1038F00081E0089580E0089580E0089589E10E94C4
:1039000019F9623059F482E00E9419F9673041F0E8
:10391000693031F0613021F081E0089580E0089550
:1039200080E008952F923F924F925F926F927F9224
:103930008F929F92AF92BF92CF92DF92EF92FF92BF
:103940000F931F93CF93DF93CDB7DEB76497CDBFAF
:10395000DEBFB82E8B017A0189E10E9403B9A62E41
:103960000115110509F46CC28091113D882339F0CD
:103970000F2EF3E7CF2EF7E3DF2EF02D06C00F2E2C
:10398000FAE7CF2EF8E3DF2EF02D82E08A1508F457
:10399000A12C8BE7F801808383E781838CE282830B
:1039A000F2E3BF1207C082E38A0DF80183838CE241
:1039B00084830BC0F801B3828CE28483F0E3BF16EA
:1039C00009F4E8C182E3B8120FC284E197E3FE0173
:1039D00032969E012E5E3F4F819391930B962E1748
:1039E0003F07D1F788E08983E114F10469F086E0AC
:1039F000F701D801159601900D928A95E1F70F2EE7
:103A0000FBE0FF2EF02D04C00F2EF5E0FF2EF02D71
:103A1000F801EF0DF11D8CE2808382E00E9403B972
:103A2000762E872D072C000C990B9F937F9280E2B6
:103A300091E29F938F93F394C8018F0D911D9F93F3
:103A40008F930F945047F80101900020E9F73197C8
:103A5000E01BF10B7F01FF24F801EE0DFF1D118229
:103A600021E0A701B801C6010F9466120F900F90D4
:103A70000F900F900F900F908091113D811112C007
:103A80001A8A21E040E050E0BE016E5E7F4F83E77E
:103A900097E30F94661220E0A701B80183E797E34C
:103AA0000F94661291E09A1508F4F9C01982912CCE
:103AB0000F2EFCE28F2EF02DF8013196EB8BFC8B54
:103AC0000F2EF1E14F2EFDE35F2EF02D5BC00F9422
:103AD000740D6980861509F45CC0F8018082E62CBB
:103AE000F12CF701EE0FFF1F81E090E08C0F9D1F7E
:103AF000E80FF91FA180B280F501418550E0B501C2
:103B00008B899C890F942247F50181856894332421
:103B100031F8380E8F5FF801E80FF11D8082F70150
:103B20003196EE0FFF1F81E090E08C0F9D1FE80F94
:103B3000F91FA180B280F501418550E0B501C801AF
:103B4000830D911D0F942247F501E1843E0C63948F
:103B500063946982E32CF12CF801EE0DFF1D1182B4
:103B600021E0A701B801C6010F946612F20180811D
:103B7000811107C020E0A701B80183E797E30F9404
:103B8000661293940F94740D8695981608F49FCF3F
:103B900053C1FBE07F12CFC0198280E00F2EFCE200
:103BA0005F2EF02D48019FEF891A990A0F2EF0E33E
:103BB0002F2EFCE23F2EF02D0F2EF1E16F2EFDE3B4
:103BC0007F2EF02DF8015082E82EF12CF701EE0F38
:103BD000FF1FEE0DFF1DEE0FFF1FEE0FFF1FE8553D
:103BE000F54C82858C3419F0823531F00CC0F4012B
:103BF0002082318212820FC081E39CE2F401808333
:103C00009183128208C085E0E5E3F1E2D4010190DE
:103C10000D928A95E1F7F80101900020E9F74E2E08
:103C2000401A5701AA0CBB1CB5016E0D7F1D660F13
:103C3000771F660F771F6855754CFB01418550E073
:103C4000C801840D911D0F942247F501EE0DFF1D53
:103C5000EE0FFF1FEE0FFF1FE855F54CE1844E0CF1
:103C6000E42CF12CF801EE0DFF1D118221E0A701DB
:103C7000B801C6010F946612F3018081811107C05B
:103C800020E0A701B80183E797E30F946612E9806B
:103C900081E08E0D8983823008F494CF4CC0198264
:103CA000612C0F2EFCE25F2EF02D4801FFEF8F1AE2
:103CB0009F0A0F2EF1E1AF2EFDE3BF2EF02D36C08F
:103CC0000F94740D79808715B1F1F8015082E72DBA
:103CD000F0E0EE0FFF1F81E090E08C0F9D1FE80FDA
:103CE000F91FE180F280F701418550E0B701C4017E
:103CF0000F942247F701E184E39473947982F12CC5
:103D0000F801EE0DFF1D118221E0A701B801C601E7
:103D10000F946612F5018081811107C020E0A70190
:103D2000B80183E797E30F94661263940F94740DC0
:103D30008695681628F20F2EFCE2FF2EF02DF80172
:103D4000F08284E00E9403B9605DF8016183F28231
:103D500040E0BE016F5F7F4FC8010396D2D88981D2
:103D600093E0980FF801E90FF11D9DE790838C5FB8
:103D7000E82EF12CF801EE0DFF1D118221E0A701C4
:103D8000B801C6010F9466128091113D882309F491
:103D900045C056C00F2EFDEAEF2EF4E4FF2EF02DA5
:103DA000F701408150E066E774E4C80105960F947E
:103DB0002247F701808195E0980FF801E90FF11D86
:103DC0009DE790838A5FE82EF12CF801EE0DFF1D30
:103DD000118221E0A701B801C6010F9466128091FB
:103DE000113D81112DC011C021E045E050E0B80126
:103DF000C6010F9466128091113D811121C0F0E33C
:103E0000BF120FC045E050E002C04E2D5F2D20E0F4
:103E1000B80183E797E30F94661212C04E2D5F2D11
:103E200002C045E050E021E0B80183E797E30F943A
:103E3000661206C01982B1CE8BE078127CCFFACF21
:103E40006496CDBFDEBFDF91CF911F910F91FF90A0
:103E5000EF90DF90CF90BF90AF909F908F907F902A
:103E60006F905F904F903F902F900895CF93892B44
:103E700081F00E940D51CAE00E94D0510E940A5167
:103E8000882321F00E942051811105C0C150A1F763
:103E900003C0C0E001C0C1E08C2FCF91089589E13B
:103EA0000E9403B9611104C00E94F1F4882371F0EB
:103EB00081E04091B0515091B1516091B2517091F7
:103EC000B351452B462B472B09F080E008958F9284
:103ED0009F92AF92BF92CF92DF92EF92FF920F9399
:103EE0001F93CF93DF930097A9F1EC0186E00E9426
:103EF00003B94B015C0184E00E9403B9162F87E0EF
:103F00000E9403B9062F812F0E940DF80E9429F804
:103F10006B017C0186169706A806B906D9F0AB019D
:103F2000BC0186E00E945BBA8823A1F00E94B6F72C
:103F3000B701A60186E00E94F9B8B701A60186E0A4
:103F40000E942CF9602F812F0E940DF868E0CE01AD
:103F50000E948113DF91CF911F910F91FF90EF90FD
:103F6000DF90CF90BF90AF909F908F90089582E1A7
:103F70000E9403B928E0E2EEF1E5DF01322F1D9245
:103F80003A95E9F7EAEEF1E5DF011D922A95E9F7A6
:103F900021E030E0672B682B692B11F420E030E042
:103FA000F901E153FF4D80818560E8EAF1E582AFD8
:103FB00083AF81E00895009761F0613031F4FC0136
:103FC000EB5CFD4F21E020830895FC01EB5CFD4F8D
:103FD000108208950097B1F0FC0180818430A1F433
:103FE0000F94A70A823039F089E10E9403B9672B48
:103FF000682B692B59F00F94840A91E0811107C056
:1040000090E005C090E003C090E001C090E0892FEF
:1040100008950F931F93CF93DF938C01EB012097AB
:1040200009F442C01882892B19F189E10E9403B971
:10403000F80180818130C0F0833018F08530D0F0F5
:1040400013C0611106C02097B9F087E4888380E02F
:104050002EC06150623090F0209791F087E4888301
:1040600080E025C0209771F082E4888380E01FC043
:1040700080E01DC081E01BC080E019C081E017C056
:1040800080E015C080E013C081E011C080E00FC067
:1040900089E10E9403B9F8018081813018F38330EF
:1040A00080F2853088F3DECF892B91F7EFCFDF9157
:1040B000CF911F910F910895009739F0FC018081F5
:1040C0008150843020F481E0089580E0089580E0FC
:1040D0000895009751F0FC018081813040F08430D8
:1040E00010F0853021F481E0089580E0089580E0AB
:1040F0000895CF92DF92EF92FF92CF93DF930097D4
:1041000009F45FC0EC0183E00E9403B96B017C01FC
:10411000AB01BC0155276627772783E00E945BBA75
:10412000882309F44BC08C2DFE01EA5CFD4FC08250
:10413000813021F1823009F044C088E00E9403B947
:10414000FE01E85CFD4F6083AB01BC01552766278B
:10415000772788E00E945BBA811105C081E0FE01EB
:10416000E85CFD4F8083FE01E95CFD4F1082C75C77
:10417000DD4F188219821A821B8223C087E00E94B9
:1041800003B9F62E84E00E9403B9862F6F2D0E949A
:104190000DF885E00E9403B90E94BEF8FE01E35CC1
:1041A000FD4F60837183828393830E94D6F7C75C3F
:1041B000DD4F188219821A821B8203C0CA5CDD4F50
:1041C0001882DF91CF91FF90EF90DF90CF9008950C
:1041D000009761F1FC01E95CFD4F2081319630814F
:1041E000321710F021111BC0FC01E95CFD4F31506A
:1041F000308332964081518162817381403821E55C
:10420000520721E06207710598F44F5F5F4F6F4FCF
:104210007F4F408351836283738381E00895FC0163
:10422000E95CFD4F2150208380E0089580E00895EF
:1042300080E008950F931F93CF93DF93009741F190
:10424000EC010E94EDF7FE01E35CFD4F008111815E
:10425000228133816017710782079307D8F00E948B
:10426000D6F7FE01E75CFD4F80819181A281B38189
:10427000803821E5920721E0A207B10568F4019694
:10428000A11DB11D80839183A283B38381E005C00A
:1042900080E003C080E001C080E0DF91CF911F91FA
:1042A0000F910895CF93DF93009709F43DC0FC016F
:1042B000EB5CFD4F20812223B9F1EC018BDE8130D4
:1042C00021F4CB5CDD4F18822FC089E10E9403B935
:1042D00061111AC00F94A70A813031F1823089F43C
:1042E000DEDD882309F10F94610ACB5CDD4F188273
:1042F00084E793E40E94A0C583E496E40E94C7C5C6
:1043000013C00F94950A10C0CADD882369F00F947A
:10431000610ACB5CDD4F188284E793E40E94A0C55C
:1043200083E496E40E94C7C5DF91CF910895FF9280
:104330000F931F93CF93DF936115710509F47CC030
:104340004115510509F478C08A01EB01F82E82E18C
:104350000E9419F921E0672B682B692B09F420E0F2
:104360008F2D90E0FC013197EB30F10508F05BC038
:104370008827E25EFE4F8F4F0D9423451882E22F6F
:10438000F0E0E153FF4D80818560F801808354C0E7
:1043900083E08883E22FF0E0E153FF4D8081F80154
:1043A00080834AC01882E22FF0E0E153FF4D808104
:1043B0008160F801808340C083E08883E22FF0E0D1
:1043C000E153FF4D8081F801808336C01882E22FCF
:1043D000F0E0E153FF4D80818160F80180832CC0C3
:1043E00083E08883E22FF0E0E153FF4D8081F80104
:1043F000808322C0188285E0F80180831DC0188266
:1044000081E0F801808318C01882E22FF0E0E153C8
:10441000FF4D80818160F80180830EC0188281E0A9
:10442000F801808309C01882E22FF0E0E153FF4DCC
:1044300080818560F8018083DF91CF911F910F917A
:10444000FF9008958F929F92AF92BF92CF92DF928A
:10445000EF92FF920F931F93CF93DF93892B09F471
:1044600086C089E00E9403B99B01AC01A8EEB3E0CD
:104470000F9440456B017C010F94B80AC616D7060D
:10448000E806F90609F475C0C701B60128EE33E065
:1044900040E050E00F94E544F22ED22F2E3108F088
:1044A0006AC0213009F469C00F94B80A28EE33E0DD
:1044B00040E050E00F94E544822FF21638F46F2D5F
:1044C0000F94B244C92F992309F45CC00F94500A89
:1044D000E82E6D2F0F94B244D92F892F90E08E0DC6
:1044E000911DCA970CF04BC08D2E912CA12CB12C94
:1044F0000F94CF0A162F072FD82EC92EA8EEB3E09F
:10450000A50194010F9440454F2D0F94FD0AC091D1
:10451000113DC11136C00F94CF0A9F938F937F93A3
:104520006F93CF92DF920F931F931F92DF931F928F
:10453000EF928AE391E29F938F9305E512E41F9334
:104540000F930F945047F80101900020E9F731973D
:10455000AF014555524421E0B80183E797E30F943A
:1045600066128DB79EB740968DBF9EBF0BC0C0E050
:1045700009C0C0E007C0C1E005C0C0E003C0C1E0A1
:1045800001C0C0E08C2FDF91CF911F910F91FF9060
:10459000EF90DF90CF90BF90AF909F908F90089555
:1045A000EF92FF920F931F93CF93DF932091113DD2
:1045B000222339F00F2EF3E7EF2EF7E3FF2EF02D35
:1045C00006C00F2EFAE7EF2EF8E3FF2EF02D00972E
:1045D000D1F1EC018BE7888388E689838CE28A83BA
:1045E00092E69B838C837F936F9385E791E29F9301
:1045F0008F93CE0105969F938F930F945047FE01A2
:1046000001900020E9F73197EC1BFD0B8F0111277A
:1046100021E0A801BE01C7010F9466120E9435B2C5
:104620000F900F900F900F900F900F90873059F4CC
:104630008091113D811107C021E0A801BE0183E7EF
:1046400097E30F946612DF91CF911F910F91FF9026
:10465000EF9008958F929F92AF92BF92CF92DF9288
:10466000EF92FF920F931F93CF93DF93009709F47C
:1046700070C02091113D222339F00F2EF3E7EF2E69
:10468000F7E3FF2EF02D06C00F2EFAE7EF2EF8E32A
:10469000FF2EF02DEC018BE7888388E689838CE27E
:1046A0008A8393E79B838C8300EC1AE3F801848C64
:1046B0000E943B9D982EA090103DB0900D3DF801BA
:1046C000C280D0800E94F1F41F928F921F929F921D
:1046D0001F92AF921F92BF921F92CF921F92DF92B2
:1046E0001F928F93F80185811F928F9384811F926F
:1046F0008F9383811F928F938AE591E29F938F938B
:10470000CE0105969F938F930F945047FE01019021
:104710000020E9F73197EC1BFD0B8F01112721E0F9
:10472000A801BE01C7010F9466128DB79EB74896C7
:104730008DBF9EBF8091113D81110BC0A8014250D9
:104740005109BE016F5F7F4F21E083E797E30F942C
:104750006612DF91CF911F910F91FF90EF90DF9044
:10476000CF90BF90AF909F908F900895DF92EF927F
:10477000FF920F931F93CF93DF9300D01F92CDB77B
:10478000DEB78C010F94BF06882349F00F94D00642
:104790000E94E80E8AEF90E45DDF80E066C0CE0103
:1047A00001960E94F10E882309F45FC0F090A806DC
:1047B000E0906806D0902806BE016D5F7F4FCE0165
:1047C00001960E94070F882309F44CC00E9441B251
:1047D0008823C9F18091113D811135C0D0FADD24C3
:1047E000D0F81F92DF92E4FAEE24E0F81F92EF92E5
:1047F000F6FAFF24F0F81F92FF928A818F93898145
:104800008F938C818F938B818F9389E791E29F9314
:104810008F930F2EF5E5EF2EF2E4FF2EF02DFF9291
:10482000EF920F945047F70101900020E9F731977C
:10483000AF014555524421E0B70183E797E30F9458
:104840006612CDBFDEBF6B817C818AEF90E4A8DE6B
:104850000115110549F08B819C81F80180839183BA
:1048600081E003C081E001C081E02496CDBFDEBFBE
:10487000DF91CF911F910F91FF90EF90DF900895FE
:10488000882321F081E08093103D08951092103D1F
:1048900008950F931F93CF93DF936115710571F006
:1048A000009761F0EB018C010F94E106882331F051
:1048B0000F94F206BE01C8010E94468BDF91CF9192
:1048C0001F910F910895CF93DF93009751F0EC0162
:1048D0000F942D07882329F0CE010E94888D0F9414
:1048E0003E07DF91CF910895009791F0FC01ED5BB9
:1048F000FD4F2FEF3FE720833183329620E030E8F1
:104900002083318332961082118232961082118276
:1049100008950F93CF93DF930097A1F0662371F072
:10492000EA01FC01E55BFD4F81E08083C9010F9442
:10493000C60C602FCE010E943E9D04C0FC01E55BC9
:10494000FD4F1082DF91CF910F910895EF92FF926A
:104950000F931F93CF93DF931F921F92CDB7DEB7B4
:10496000009709F458C06115710509F454C0FC01A1
:1049700021A9211104C022A9222309F44CC08B01D2
:104980007C01FC0111AA12AA0E9444100E94CF10BF
:104990000E94C812F70143A954A9B7016B5C7F4F6D
:1049A0009E012F5F3F4FC8010F94473BC8010F94F2
:1049B000F53CF701E85AFD4FD701AE5ABD4F8C9137
:1049C0008083319611968C918083F70123A934A9B5
:1049D00089819A812817390719F00E94EB9D02C03E
:1049E0000E947B9DE6E3F1E4808190E0DC01AA5C1B
:1049F000BE4B25853685880F991FFC01EA5CFE4B6E
:104A0000418152811F960C9161E0C70182DF0E94B3
:104A1000DA8F0F942C0D0F900F90DF91CF911F9193
:104A20000F91FF90EF9008950F931F93CF93DF9313
:104A3000009709F448C06115710509F444C08B0161
:104A4000EC01FC01E55BFD4F80818823C1F1DB01B6
:104A50008C91882341F10F94E20C8823A1F1F80195
:104A6000608161506083611108C00E94B09D0E9406
:104A70009D9DC55BDD4F188226C070E0F801E60FF2
:104A8000F71FD8011D962D913C911E97660F771F39
:104A9000A60FB71F11964D915C911297078561E0A3
:104AA000CE0137DF10C00F94E20C882361F00E9422
:104AB000B09D0E949D9DC55BDD4F188204C00E9481
:104AC000B09D0E949D9DDF91CF911F910F91089500
:104AD0008F929F92BF92CF92DF92FF920F931F937C
:104AE000CF93DF93009709F4DAC06115710509F4DB
:104AF000D6C02091113D222309F4C0C0C3E7D7E3FB
:104B0000BFC08B014C010E94A710B82E0E94271134
:104B1000D82E0E940210C82E8D2D90E08B0D911D75
:104B20008C0D911D892B71F4F401E45BFD4F8081A4
:104B3000813009F4B4C081E0808380E090E00F947C
:104B4000F90CADC0F401E45BFD4F8081823009F4C3
:104B50003EC0BB2051F00E94A410811108C061E04A
:104B6000CE010E94B28F01E003C000E001C000E06E
:104B7000CC2009F48AC00E94FF0F811186C063E037
:104B8000CE010E94B28F01E080C0DD2081F0812F34
:104B90000E940713882359F0812F0E941713811157
:104BA00006C064E0610FCE010E94B28F01E01F5F7A
:104BB000143059F7002309F472C0E401C45BDD4FDF
:104BC00082E0888384EF91E00F94F90C68C00F9421
:104BD000150D882309F463C0BB2009F45DC00E9451
:104BE000A410811159C00E94029ECC2009F44FC02C
:104BF000FF24F39401C0F12C0E94FF0F811149C0E2
:104C00000E94029E16C0D0E0C0E0DD2069F08D2F2A
:104C10000E940713882341F08D2F0E9417138111E2
:104C200003C00E94009EC1E0DF5FD43071F7CC2347
:104C3000E1F084EF91E00F94F90CD8018C9190E0B1
:104C4000F801E80FF91F1D962D913C911E97880FD2
:104C5000991FA80FB91F11964D915C911297078566
:104C600061E080EC9AE355DE1AC0F401E45BFD4F8D
:104C700080818230A1F481E0808311C0CAE7D8E34B
:104C8000FC012081243059F43CCF10E07ECFFF247A
:104C9000F394F110CECFB7CFC110ADCFB4CFDF9129
:104CA000CF911F910F91FF90DF90CF90BF909F9079
:104CB0008F900895009721F0FC01E45BFD4F608325
:104CC0000895CF93DF930097C1F0EC011982188209
:104CD0000E947E1C813031F482E0888389E18983DF
:104CE00091E006C0CE010E9443E191E0811190E085
:104CF00081E0992319F080E001C080E0DF91CF913D
:104D00000895CF93892B09F44CC082E00E9403B927
:104D1000862F90E0FC013297EA30F10508F043C09D
:104D20008827E75DFE4F8F4F0D94234540E050E00C
:104D3000BA0180E00E9455C037C040E050E0BA019F
:104D400080E00E9455C0C82F40E050E0BA0181E0E9
:104D50000E9455C0C80F81E0C23031F180E024C00C
:104D600040E050E0BA0180E00E9455C0C82F40E00A
:104D700050E0BA0181E00E9455C0C80F40E050E009
:104D8000BA0182E00E9455C0C80F40E050E0BA016D
:104D900083E00E9455C0C80F81E0C43029F080E054
:104DA00003C080E001C080E0CF910895CF92DF92F0
:104DB000EF92FF92843098F4E82FF0E0EE0FFF1F9F
:104DC000EE0FFF1FEF57F64CC080D180E280F380DA
:104DD0000E9425C06C197D098E099F0903C060E0FF
:104DE00070E0CB01FF90EF90DF90CF900895CF93CC
:104DF000892B09F453C082E00E9403B9862F90E00A
:104E0000FC013297EA30F10508F04AC08827ED5CD2
:104E1000FE4F8F4F0D94234580E0C8DFAB01BC01EE
:104E200080E00E9455C03DC080E0C0DFAB01BC0106
:104E300080E00E9455C0C82F81E0B8DFAB01BC0103
:104E400081E00E9455C0C80F81E0C23051F180E07E
:104E500028C080E0ABDFAB01BC0180E00E9455C000
:104E6000C82F81E0A3DFAB01BC0181E00E9455C0E7
:104E7000C80F82E09BDFAB01BC0182E00E9455C0FD
:104E8000C80F83E093DFAB01BC0183E00E9455C0F3
:104E9000C80F81E0C43029F080E003C080E001C089
:104EA00080E0CF910895883009F485C028F48330DC
:104EB00041F0853079F1A6C08A50823008F453C0A1
:104EC000A1C0E8EAF1E5868D978DA0A1B1A1428D40
:104ED000538D648D758D841B950BA60BB70B86398E
:104EE0009105A105B10508F48FC046A157A160A5A1
:104EF00071A582A193A1A4A1B5A1481B590B6A0B6E
:104F00007B0B81E0463951056105710508F483C0CA
:104F100080E00895E8EAF1E582A193A1A4A1B5A1FA
:104F2000468D578D60A171A1841B950BA60BB70B05
:104F300086399105A105B10508F468C046A557A5B5
:104F400060A971A982A593A5A4A5B5A5481B590B75
:104F50006A0B7B0B81E0463951056105710508F448
:104F60005AC080E00895E8EAF1E582A193A1A4A1E6
:104F7000B5A1468D578D60A171A1841B950BA60B21
:104F8000B70B86399105A105B10508F441C042A9C6
:104F900053A964A975A986A597A5A0A9B1A9481B7D
:104FA000590B6A0B7B0B81E0463951056105710590
:104FB00090F180E00895E8EAF1E5868D978DA0A153
:104FC000B1A1428D538D648D758D841B950BA60BFD
:104FD000B70B86399105A105B105E0F042A553A5AF
:104FE00064A575A586A197A1A0A5B1A5481B590BDD
:104FF0006A0B7B0B81E0463951056105710558F05C
:1050000080E0089580E0089581E0089581E00895AA
:1050100081E0089581E00895CF9382E10E9403B971
:10502000C1E0672B682B692B09F4C0E082E00E9485
:1050300003B988E0E2EEF1E5DF01982F1D929A9521
:10504000E9F7EAEEF1E5DF011D928A95E9F7862F8F
:1050500090E0FC013197EB30F10508F0EFC08827B4
:10506000E35CFE4F8F4F0D942345EC2FF0E0E153AE
:10507000FF4D80818560E8EAF1E582AF83AFE8C04B
:10508000EC2FF0E0E153FF4D8081E8EAF1E582AFDB
:1050900083AF83E08093EA518093EB51D9C083E0E2
:1050A00002DFEC2FF0E0E153FF4D908121E0811110
:1050B00001C020E0822F892BE8EAF1E582AF84AFBE
:1050C00083E08093EA518093EC51892F816083AF14
:1050D00085AFBEC0EC2FF0E0E153FF4D8081E8EAE0
:1050E000F1E582AF84AF93E09093EA519093EC5155
:1050F00083AF85AF82E08093EB518093ED51A8C0E0
:1051000085E0D1DEEC2FF0E0E153FF4D208191E00E
:10511000811101C090E0892F822BE8EAF1E582AF8E
:1051200085AF93E09093EA519093ED5183AF86AFB2
:1051300082E08093EB518093EE51822F816084AFA7
:1051400087AF86C0EC2FF0E0E153FF4D8081E8EAA5
:10515000F1E582AF86AF93E09093EA519093EE51E0
:1051600083AF87AF92E09093EB519093EF5184AF70
:105170008093E85194E09093EC519093F05185AF77
:105180008093E95185E08093ED518093F15160C0A7
:10519000862F89DE91E0811101C090E0892F8F7008
:1051A000E8EAF1E582AF86AF93E09093EA519093FD
:1051B000EE5183AF87AF82E08093EB518093EF5144
:1051C00081E084AF8093E85195AF9093E95140C05E
:1051D000E8EAF1E585E082AF84AF87E083AF85AF91
:1051E00037C088E060DE91E0811101C090E0EC2FD3
:1051F000F0E0E153FF4D8081892BE8EAF1E582AFD1
:1052000085AF83E08093EA518093ED5191E093AFB5
:1052100096AF84AF87AF1CC0EC2FF0E0E153FF4D99
:1052200080818160E8EAF1E582AF84AF83AF85AF2A
:1052300081E08093EB518093ED510AC0EC2FF0E0B8
:10524000E153FF4D80818560E8EAF1E582AF83AFED
:1052500081E0CF9108951F93CF93DF930097D9F109
:10526000EC0119AA1AAA0E94C61687E00E9403B987
:10527000162F84E00E9403B9862F612F0E940DF83B
:1052800089E10E9403B9613071058105910521F41E
:1052900081E00F94E60A03C080E00F94E60A0E94C2
:1052A0006A1C813031F4CE010E94231C0E94B71F7A
:1052B00004C0CE010E94B91BAFDE0F94770DCE0162
:1052C0000E9479200F94020C0E94330F0E948410D8
:1052D0000E9403111982DF91CF911F910895CF93FE
:1052E000DF93009791F0FC012081243071F4EC01F0
:1052F0000E94671FCE01AFDF0F94730A10920C3D1E
:1053000063E0CE010E9481131982DF91CF9108954D
:10531000882321F081E08093113D08951092113D82
:1053200008958091113D0895AF92BF92CF92DF9280
:10533000EF92FF920F931F93CF93DF93DC010097BF
:1053400009F45AC04115510509F458C02115310519
:1053500009F456C0FA01C081D0E0F901008110E0E3
:105360006115710561F0FC017C01E60EF71E91915B
:10537000C90FD11D0C0F1D1FEE16FF06C1F7F90155
:105380007B016D01DA01CC930083F601E60FF71F74
:105390008CE280838BE181835B01A2E0AA0EB11CC9
:1053A000AC0CBD1C8C2F82958F700F941A16F501D2
:1053B00080835701F3E0AF0EB11CAC0CBD1C8C2FE9
:1053C0008F700F941A16D5018C93E7012496CC0D9B
:1053D000DD1D802F82958F700F941A168883D70158
:1053E0001596E601CA0FDB1F802F8F700F941A16D7
:1053F0008883C701069605C0CB0103C0CB0101C05D
:10540000CB01DF91CF911F910F91FF90EF90DF9033
:10541000CF90BF90AF9008952F923F924F925F929E
:105420006F927F928F929F92AF92BF92CF92DF92B4
:10543000EF92FF920F931F93CF93DF93CDB7DEB719
:105440006197CDBFDEBF7C016B013A01490189E163
:105450000E9403B9562E82E00E9403B9162FE11470
:10546000F10409F41DC1C114D10409F41BC16B304E
:1054700009F020C16114710409F416C1811491046A
:1054800009F414C1FE013296CE014296C192D19226
:105490002BE0C20ED11C8E179F07C1F78DE0D701FC
:1054A000D5968C93D59782E090E0D3968D939C937C
:1054B000D4978AE0D6968C935701B7E3AB0EB11C14
:1054C00041E0BE016F5F7F4FC5010E9481172981B6
:1054D000F70183A994A9820F911D9C012F5F3F4F73
:1054E00023AB34ABE80FF91F2CE225ABF1E0F51547
:1054F00090F5512C0F2EFCE24F2EF02D61C0E52DC2
:10550000F0E0EE0FFF1F81E090E08C0F9D1FE80F91
:10551000F91FC180D280D701D3968D919C91D497E9
:10552000C596F601418550E0B6018E0D9F1D0F9482
:105530002247D60119962C91F70183A994A9820FCD
:10554000911D9C012F5F3F4F23AB34ABE80FF91F38
:1055500045AA539405C0512C0F2EFCE24F2EF02D7E
:105560000F94740D581658F2AAC0E52DF0E0EE0F16
:10557000FF1F81E090E08C0F9D1FE80FF91FC18095
:10558000D280D701D3968D919C91D497C596F60180
:10559000418550E0B6018E0D9F1D0F942247D60124
:1055A00019962C91F70183A994A9820F911D9C0152
:1055B0002F5F3F4F23AB34ABE80FF91F45AA53943D
:1055C0000F94740D8695581680F279C0D6011A96FC
:1055D0008C911F928F933F922F92F70183A994A9E8
:1055E000C5968E0D9F1D9F938F930F945047F30187
:1055F00001900020E9F73197E619F709D701D39612
:10560000ED93FC93D497CF01C596F601418550E008
:10561000B6018E0D9F1D0F942247D60119962C912D
:10562000F70183A994A9820F911D9C012F5F3F4F21
:1056300023AB34ABE80FF91F15ABFCE0CF0ED11C48
:105640000F900F900F900F900F900F904C145D04DF
:1056500009F0BCCF0130D9F4D701D3968D919C913C
:10566000D497C596840101501F4FF801408150E046
:10567000B4018E0D9F1D0F942247D8012C91F70184
:1056800083A994A9820F911D83AB94AB2BC0D70142
:10569000D396ED91FC91D497EE0DFF1D15AA22C073
:1056A00080E03FC080E03DC080E03BC080E039C08A
:1056B00080E037C08114910409F0E4CEF9CF1B30AB
:1056C00049F663012301B8E14B0E511C0F2EF8E996
:1056D0002F2EF1E23F2EF02D3701E5E36E0E711C07
:1056E0001CE274CFA7014E5A5D4FF701E85AFD4FF7
:1056F0008081DA018C9397012D5A3D4F319680813C
:10570000F9018083D701D3966D917C91D497625033
:105710007109C50109DE0296F70183AB94AB81E004
:1057200081AB6196CDBFDEBFDF91CF911F910F910D
:10573000FF90EF90DF90CF90BF90AF909F908F90B1
:105740007F906F905F904F903F902F9008952F9291
:105750003F924F925F926F927F928F929F92AF9201
:10576000BF92CF92DF92EF92FF920F93CF93DF938E
:10577000CDB7DEB76097CDBFDEBF009709F46EC02E
:105780006115710509F46AC09B01FE013196DE01C5
:10579000519621933193255F3F4FEA17FB07C9F7D5
:1057A0006A017B011C01B12C12C0EB2DF0E0EE0F61
:1057B000FF1F81E090E08C0F9D1FE80FF91F808193
:1057C00091810E94DF16882309F448C0B3940F9496
:1057D000740DB81650F30F94CF0A4B015C010F946F
:1057E000B80A2B013C0184E793E40E94A6C5082F68
:1057F00081110BC09EE1890E911CA11CB11C841467
:105800009504A604B70450F115C040E050E06AEFDB
:1058100070E480E30E94921C24E733E4A601B70100
:10582000C101FADD46E754E46AEF70E482E30E94C6
:10583000921C0EC000E024E733E4A601B701C101C9
:10584000EBDD40E050E06AEF70E482E30E94921CDE
:1058500084E793E40E94A0C50E94C6166096CDBF5F
:10586000DEBFDF91CF910F91FF90EF90DF90CF904F
:10587000BF90AF909F908F907F906F905F904F9070
:105880003F902F900895009789F06115710571F090
:105890004115510559F02115310541F0FC011082E7
:1058A000FB011082FA011082F901108208952F92F3
:1058B0003F924F925F926F927F928F929F92AF92A0
:1058C000BF92CF92DF92EF92FF920F931F93CF93ED
:1058D000DF93CDB7DEB72597CDBFDEBF009709F4C4
:1058E00061C04115510509F45FC02115310509F466
:1058F0005DC0613BE4E07E0708F45AC02B01E0EB99
:105900004E1AE4E05E0A612C712CE2E04E1651045E
:10591000610471040CF454C02C833D831A018C0182
:10592000C12CD12C7601C3944B01A12CB12CB50113
:10593000A4014C195D096E097F09C8010F94473D08
:105940009E012F5F3F4F41E050E0BE016D5F7F4FF2
:10595000C8010F94FB3981112DC08B818B3191F1DE
:105960008FEFC81AD80AE80AF80AC414D504E60466
:10597000F704ECF225C089819A810497E8F0B1011F
:1059800085E592E40F940C1A982F882341F16C81DD
:105990007D8187E592E40F940C1A91E081111FC07C
:1059A00090E01DC090E01BC090E019C090E017C0CF
:1059B00090E015C090E013C090E011C090E00FC0DF
:1059C00090E00DC09E012F5F3F4F44E050E065E541
:1059D00072E4C8010F94FB39882369F2EFCF892F55
:1059E0002596CDBFDEBFDF91CF911F910F91FF9024
:1059F000EF90DF90CF90BF90AF909F908F907F906F
:105A00006F905F904F903F902F9008950097A9F06E
:105A100061157105B1F0FC019C01260F371F60E094
:105A200070E0CB0141914D3021F46F5F7F4F8F4F7C
:105A30009F4F2E173F07B1F7089560E070E0CB014C
:105A4000089560E070E0CB0108952F923F924F924D
:105A50005F926F927F928F929F92AF92BF92CF92FE
:105A6000DF92EF92FF920F931F93CF93DF9300D0BB
:105A70001F92CDB7DEB7009709F455C00115110587
:105A800009F453C0613B7440C0F4F80110821182E4
:105A90001282138280E04CC009811A81B801C101D1
:105AA000B5DF460E571E681E791E0815190500F150
:105AB000C00ED11EE11CF11C0BC00B831C834901DD
:105AC0001A015C01C12CD12C7601412C512C3201E0
:105AD000B701A601C5010F94473D9E012F5F3F4FBF
:105AE000A401B101C5010F94FB398823A9F21FC09D
:105AF000F6E24F1651046104710440F4EB81FC811D
:105B0000108211821282138281E012C0F5E24F1AD4
:105B1000510861087108EB81FC81408251826282E8
:105B2000738281E005C080E003C080E001C080E0B6
:105B30002496CDBFDEBFDF91CF911F910F91FF90D3
:105B4000EF90DF90CF90BF90AF909F908F907F901D
:105B50006F905F904F903F902F900895009741F085
:105B6000FC01EC5AFD4F608171818281938108951F
:105B700060E070E0CB010895009739F0FC01EC5A29
:105B8000FD4F10821182128213820895CF93DF930A
:105B9000009781F12091113D21112CC0EC010F944F
:105BA000BB07882339F1CE010E9416940F94A007F9
:105BB0000E94DAF41F928F938CE991E29F938F9366
:105BC000C5E5D2E4DF93CF930F94504709900020AE
:105BD000E9F72197AE014555524420E065E572E4AE
:105BE00083E797E30F9466120F900F900F900F903A
:105BF0000F900F90DF91CF9108952115310551F04D
:105C0000505861097109F90140835183628373839C
:105C100081E0089580E00895009719F0FC01848DDB
:105C2000089580E008952F923F924F925F926F9275
:105C30007F928F929F92AF92BF92CF92DF92EF921C
:105C4000FF920F931F93CF93DF93CDB7DEB72597C6
:105C5000CDBFDEBFE114F10409F49EC01701480175
:105C600059016A017B01182FC1010E94BA16240153
:105C700035014C185D086E087F08143031F484E15A
:105C80000E94DFB89B01AC0105C085E10E94DFB82E
:105C90009B01AC01440C551C661C771CD301C2014E
:105CA000880F991FAA1FBB1F880F991FAA1FBB1F10
:105CB000480E591E6A1E7B1E2115310541055105EE
:105CC00049F0C301B2010F9407452A833B834C83FB
:105CD0005D8308C08FEF8A8390EE9B83A5EFAC8332
:105CE000B5E0BD836A817B818C819D812AE030E0B3
:105CF00040E050E00F9407455F934F933F932F93FD
:105D0000FF92EF92DF92CF92BF92AF929F928F92CB
:105D1000C301B2012AE030E040E050E00F940745B3
:105D20005F934F933F932F9387EB91E29F938F93D2
:105D300005E512E41F930F930F945047F80101906B
:105D40000020E9F73197AF014555524420E0B801F2
:105D500083E797E30F9466120A811B812C813D81B2
:105D60004BE0BE016F5F7F4FC1010F948619F101B7
:105D700001900020E9F73197E219F309D101199652
:105D8000EC93199781E01B968C93CDBFDEBF6A819F
:105D90007B818C819D8104C060E070E080E090E0B8
:105DA0002596CDBFDEBFDF91CF911F910F91FF9060
:105DB000EF90DF90CF90BF90AF909F908F907F90AB
:105DC0006F905F904F903F902F9008952F923F9249
:105DD0004F925F926F927F928F929F92AF92BF92FB
:105DE000CF92DF92EF92FF920F931F93CF93DF93A7
:105DF000CDB7DEB72897CDBFDEBFCA01E982FA82F0
:105E0000CD82DE82AB82BC826115710509F4B7C018
:105E1000009709F4B6C0EF2809F4B5C0802E912E82
:105E2000A22EB32E25EB82169104A104B10438F002
:105E30000F2EF4EB8F2E912CA12CB12CF02DDB0129
:105E4000CD90DD90ED90FC90B0E8DB1AE108F10810
:105E5000FB01C082D182E282F38221E02093CD3027
:105E6000F2E08F169104A104B10408F46AC0FB01AA
:105E70002DEC30E32F83388794012150304C220FD2
:105E8000331F220F331F1B01220E331E4601570101
:105E900000E010E098014481558166817781505877
:105EA00061097109448355836683778341905190DA
:105EB0006190719044195509660977091416150601
:105EC0001606170634F441E0AF81B88511964C935D
:105ED00004C0AF81B88511961C92AF81B885119628
:105EE0005C911197BD016F5F7F4F6F8378874C91F5
:105EF000541781F0D801AA0FBB1FAA0FBB1FA80F10
:105F0000B91F4D925D926D927C9213970F5F1F4F58
:105F10002F4F3F4F4081518162817381C416D50656
:105F2000E606F70614F46A017B01481559056A056F
:105F30007B0514F44A015B01E215F30509F0ABCFD0
:105F400005C04601570100E010E09801A981BA811F
:105F50000D931D932D933C931397ED81FE81309704
:105F600021F080829182A282B382EB81FC81309702
:105F700061F0C082D182E282F38281E007C080E0DA
:105F800005C080E003C080E001C081E02896CDBF5D
:105F9000DEBFDF91CF911F910F91FF90EF90DF90C7
:105FA000CF90BF90AF909F908F907F906F905F90B9
:105FB0004F903F902F9008958F929F92AF92BF92F3
:105FC000CF92DF92EF92FF920F931F93FC01892BE8
:105FD000A1F16115710599F100811181228133814F
:105FE00084819581A681B781081719072A073B0785
:105FF00044F5C084D184E284F384C816D906EA0645
:10600000FB060CF584849584A684B784C814D9044F
:10601000EA04FB04D4F488159905AA05BB05BCF471
:106020000C151D052E053F0524F481E0FB0180833E
:106030000FC0FB01108281E00BC080E009C080E04E
:1060400007C080E005C080E003C080E001C080E0C0
:106050001F910F91FF90EF90DF90CF90BF90AF9086
:106060009F908F9008953F924F925F926F927F9290
:106070008F929F92AF92BF92CF92DF92EF92FF9258
:106080000F931F93CF93DF93009709F448C0211516
:10609000310509F446C0443051056105710508F425
:1060A00042C06A017B01E4E0CE1AD108E108F108A0
:1060B000E1F159018C01912C312C812C412C512C76
:1060C0003201E501C90DD11DBE01C201880F991F22
:1060D000880F991F800F911F6FDF882379F08881C7
:1060E000882311F0839401C0339483E0480E511C3F
:1060F000611C711C9394E2E0E91550F08FEF481A8F
:10610000580A680A780A4C145D046E047F04C8F2C9
:10611000882069F081E0332059F080E009C080E0F8
:1061200007C080E005C080E003C081E001C081E0DD
:10613000DF91CF911F910F91FF90EF90DF90CF9063
:10614000BF90AF909F908F907F906F905F904F9097
:106150003F9008952F923F924F925F926F927F925D
:106160008F929F92AF92BF92CF92DF92EF92FF9267
:106170000F931F93CF93DF93CDB7DEB76A97CDBF51
:10618000DEBF582ED92E862E972E19821A821B8298
:106190001C821D821E821F82188619861A861B8603
:1061A0001C861D861E861F86188A82E00E9403B9FF
:1061B0006B3009F0CAC00F94AD0E882309F4C6C035
:1061C0000F949C0E252C3D2CCE0101968B8B9C8B25
:1061D000DE011996AD8BBE8BA98BBA8B652C7D2CFD
:1061E0006894552452F8298E3A8E482C392C4C014B
:1061F0006F8A788EA988BA8864010F2EF6EFEF2E89
:10620000FDE2FF2EF02D04EB10E020E030E04DEF3A
:106210005DE2B301852DDADD882331F14091F62D61
:106220005091F72D6091F82D7091F92D2AEF3DE2F4
:106230008DEF9DE218DF882361F08091FA2D90E0C8
:10624000A0E0B0E0EF89F88D80839183A283B383CF
:1062500014C08EEF90E0A0E0B0E0EF89F88D80836D
:106260009183A283B38309C08FEF90E0A0E0B0E0F8
:10627000F30180839183A283B3835394F0E36F1A75
:10628000FDEF7F0A84E0880E911CA989BA891496D3
:10629000A98BBA8BB6E05B12ABCF932C298C3A8CCE
:1062A000642C792C6894552452F80F2EF5E44F2E67
:1062B000F02D0F2EF2E5DF2EF02D0F2EFCE4CF2E69
:1062C000F02DAB88BC888D889E88698A7A8AF40113
:1062D00001911191219131914F01D5014D915D9124
:1062E0006D917D915D017301852D9DDC6531710599
:1062F000810591051CF4F30142861AC0F1018081E9
:106300009181A281B3810097A105B10529F4A989E2
:10631000BA891A96CC920CC00197A105B10521F457
:10632000E989FA89D28604C0A989BA891A964C9259
:106330005394BCE06B0E711CE0E32E1AEDEF3E0AA5
:10634000F6E05F12C2CF81E001C080E06A96CDBF67
:10635000DEBFDF91CF911F910F91FF90EF90DF9003
:10636000CF90BF90AF909F908F907F906F905F90F5
:106370004F903F902F9008951F93CF93DF930097F6
:1063800009F4DAC0EC018881843069F128F48130A5
:1063900049F08230C9F0D0C0883011F1893009F459
:1063A000A7C0CAC08B81813009F0C6C08C81813002
:1063B00009F0C2C00F94950ACE010E942B2962E019
:1063C000CE010E948113B8C08091CF46813029F45C
:1063D00063E0CE010E948113AFC00E94641BACC079
:1063E0000E94624CA9C0CE010E94522182E00E940C
:1063F00003B96B3041F064E177E388E99AE30E94E6
:10640000AC17182F10C00F94AD0E8823E1F064E193
:1064100077E388E99AE30E94AC17182F68EA7AE3D9
:1064200088E09CE497DE113071F482E00E9403B9A9
:10643000162F88E99AE30E944F0F612F84E29EE3B2
:106440000E94711107C084E197E30E94EA16882335
:1064500009F465C048EA5AE364E177E3CE0177D9ED
:106460005EC00E94FEF8882309F463C00F94130CE9
:1064700064E67EE3CE010E94A6240E94EDF859C096
:106480008981811159C0CE010E941A21882341F0CF
:106490000F94130C64E67EE3CE010E94A6244CC048
:1064A00019AA81E08AAB48C089A9882309F444C0AD
:1064B0008981811141C0CE010E94E820882341F0EA
:1064C0000F94130C64E67EE3CE010E94A62434C030
:1064D00019AA32C00E94FEF8882371F10F94130CA0
:1064E00064E67EE3CE010E94A6240E94EDF824C05B
:1064F000CE010E94522164E177E388E99AE30E9489
:1065000024FD813031F084E197E30E9479FD8823F6
:1065100099F064E177E3CE010F94A2000DC0FE0173
:10652000EA5CFD4F8081813009F49BCF823091F687
:10653000BBCF89A98111A4CFDF91CF911F9108957D
:10654000CF930E94C4C0C82F88E10E9403B9C61728
:1065500041F061E080E00E94DAF661E081E00E94B3
:10656000DAF6CF910895CF930E94C4C0C82F88E176
:106570000E9403B9C61749F061E080E00E94DAF694
:1065800061E081E00E94DAF608C060E080E00E94ED
:10659000DAF660E081E00E94DAF6CF910895CF93B9
:1065A000DF93EC018091113D882319F0E3E7F7E3D5
:1065B00002C0EAE7F8E3209729F18BE7888388E6B1
:1065C00089839CE29A8382E68B839C838CE68D830D
:1065D0008DE78E831F8221E047E050E0BE01CF01AE
:1065E0000F9466120E9435B2873061F48091113D9C
:1065F000811108C021E047E050E0BE0183E797E346
:106600000F946612DF91CF910895EF92FF920F934E
:106610001F93CF93DF93CDB7DEB72797CDBFDEBFF4
:106620007C01FB0184818D8385818E8386818F83AC
:1066300080819181A281B38189839A83AB83BC835A
:10664000870180EAE81688E0F80629F460E183E033
:106650000F946D2414C080EBE81688E0F80629F446
:1066600060E283E00F946D2413C080EAE81689E0AD
:10667000F80629F460E184E00F946D2412C0003B19
:1066800089E0180729F460E284E00F946D2412C0B9
:10669000003A8AE0180729F460E185E00F946D2440
:1066A00010C0003B8AE0180729F460E285E00F94EF
:1066B0006D2407C0003A1B4021F460E186E00F948E
:1066C0006D24BE016F5F7F4FC7010E94956C2796B6
:1066D000CDBFDEBFDF91CF911F910F91FF90EF9063
:1066E0000895DC01892BE1F0E62FE695E695E69525
:1066F00080E2E89FF0011124FA5F8085677021E055
:1067000030E002C0220F331F6A95E2F7282381E0B0
:1067100009F480E08C9311968C93119712961C9239
:106720000895CF93DF93009709F4A5C06D3209F067
:10673000A4C03091A80621E0432F407235FF20E02D
:10674000FC0120833181231709F499C0EC01442313
:1067500009F46BC0311169C00F944F070097F9F429
:106760000E949129811119C086E0EFEDF1E2A5E5C3
:10677000B2E401900D928A95E1F7E5E5F2E401902B
:106780000020E9F73197AF014555524421E065E516
:1067900072E483E797E30F9466121A8268C0803D23
:1067A000974008F50E949129811119C086E0E5EE15
:1067B000F1E2A5E5B2E401900D928A95E1F7E5E5F5
:1067C000F2E401900020E9F73197AF0145555244BA
:1067D00021E065E572E483E797E30F9466120F9476
:1067E00063071A8244C081E08A830F9463070E9482
:1067F000912981113CC086E0EBEEF1E2A5E5B2E41F
:1068000001900D928A95E1F7E5E5F2E40190002010
:10681000E9F73197AF014555524421E065E572E44F
:1068200083E797E30F94661222C01A8281E090E01A
:106830000F9476070E949129811119C086E0E1EF3B
:10684000F1E2A5E5B2E401900D928A95E1F7E5E564
:10685000F2E401900020E9F73197AF014555524429
:1068600021E065E572E483E797E30F94661288817F
:1068700089838A8105C080E003C080E001C080E098
:10688000DF91CF91089583E496E40C9473CD08953D
:106890000E949129811117C067ED72E483E797E3A5
:1068A0000F94121280915943813029F547ED52E43B
:1068B00069ED72E483E797E30E9489B687ED92E47D
:1068C0000D940312089567ED72E483E797E30E9445
:1068D000AE9A80915943813071F420EC3AE347ED50
:1068E00052E469ED72E483E797E30E949F9A87ED93
:1068F00092E40D94031208950E941B8F882329F0BF
:1069000085ED9FE30C94632408950E9491298111E1
:106910002EC063EF7FE38AE798E30E94AE9A8091EE
:106920007540813021F50E949129811112C062E4E5
:1069300080917337909174370E947A6B4091F33F46
:106940005091F43F21E065EF7FE383E797E30F94F5
:10695000661220EC3AE343EF5FE365EF7FE38AE7FB
:1069600098E30E949F9A83EF9FE30D94031208958A
:10697000CF92DF92EF92FF920F931F93CF93DF930B
:106980000E949129882319F003E717E302C00AE760
:1069900018E384EE9FE30E94B99C882331F064EEF3
:1069A0007FE3C8010E94492488C28091F23F815050
:1069B000823008F054C10E943B9D882309F47DC2B7
:1069C0006FE97EE38DE19DE30E94409C8091D03F82
:1069D000813009F072C2E0909F3EF090A03E82E0CC
:1069E000E816F10408F469C28091F23F813039F46D
:1069F0008091A43E8F7D8C3409F0CBC00AC0809179
:106A0000A43E843209F0C5C08091A53E833509F0CB
:106A1000C0C00E949129811156C087E0E7EFF1E2E2
:106A2000A5E5B2E401900D928A95E1F7E5E5F2E47F
:106A300001900020E9F73197AF014555524420E01D
:106A400065E572E483E797E30F9466121092A13E26
:106A50001092A23EE114F104A1F080E090E0CFE9B1
:106A6000DEE3FC01E156F14C658183E797E30F9487
:106A7000F2128A819B8101968A839B838E159F05E2
:106A800080F30F94250C1F928F938EEF91E29F93CA
:106A90008F93C5E5D2E4DF93CF930F9450470990CD
:106AA0000020E9F72197AE014555524421E065E504
:106AB00072E483E797E30F9466120F900F900F90A4
:106AC0000F900F900F900F94250C882371F181E0A7
:106AD0000E94898A813069F48FE99EE30E94869C36
:106AE0008FE99EE30E94989C0F94020C0E948A9D5D
:106AF00002C00E94EB9DE6E3F1E4808190E0DC01BE
:106B0000AA5CBE4B25853685880F991FFC01EA5C7F
:106B1000FE4B418152811F960C9161E080EC9AE31B
:106B20000E9489240F942C0D93C0E092D33FF092E1
:106B3000D43F0F94250C682FC8010E94678D0E94D6
:106B40009129811185C00F94250C1F928F938091FC
:106B5000F23F1F928F9384E092E29F938F93C5E55B
:106B6000D2E4DF93CF930F94504709900020E9F7C8
:106B70002197AE014555524421E065E572E483E773
:106B800097E30F946612EDB7FEB73896EDBFFEBFE0
:106B90005FC00E949129811157C08091F23F8230DD
:106BA00049F48091A43E843229F48091A53E873433
:106BB00009F44AC08AE0E2E2F2E2A5E5B2E401901B
:106BC0000D928A95E1F7E5E5F2E401900020E9F7FE
:106BD0003197AF014555524420E065E572E483E703
:106BE00097E30F946612EFE9FEE31282138280812D
:106BF0009181892BA9F080E090E0EF01FC01E15642
:106C0000F14C658183E797E30F94F2128A819B81AF
:106C100001968A839B83288139818217930770F3B9
:106C2000E5E5F2E480E290E080839183019000202A
:106C3000E9F73197AF014555524421E065E572E42B
:106C400083E797E30F9466128FE99EE30E94989C76
:106C50008FE99EE30E94869C0F94020C2EC10F9434
:106C6000C5076B017C016FE97EE38DE19DE30E9426
:106C7000D59B8091D03F813039F0F5E6CF16D10415
:106C8000E104F10408F419C10F94DC078091D03FAE
:106C9000813079F48FE99EE30E94099D882321F0D9
:106CA000E090D23FF12C40C0E0909F3EF090A03E9B
:106CB0003BC00F2EFFE9EF2EFEE3FF2EF02DF70174
:106CC00081818F9380818F938CE292E29F938F9347
:106CD000C5E5D2E4DF93CF930F945047099000208D
:106CE000E9F72197AE014555524421E065E572E48C
:106CF00083E797E30F9466121092D23F0F900F90A4
:106D00000F900F900F900F90F7018081918187393C
:106D1000910530F086E990E080939F3E9093A03EED
:106D2000E0909F3EF090A03E0E94912981115DC0AD
:106D3000FF92EF928BE492E29F938F93C5E5D2E4AA
:106D4000DF93CF930F94504709900020E9F72197E4
:106D5000AE014555524420E065E572E483E797E3D0
:106D60000F9466121092A13E1092A23E0F900F90C7
:106D70000F900F900F900F90E114F104A1F080E0BC
:106D800090E0CFE9DEE3FC01E156F14C658183E759
:106D900097E30F94F2128A819B8101968A839B83E9
:106DA0008E159F0580F30F94250C1F928F938EEF05
:106DB00091E29F938F93C5E5D2E4DF93CF930F9435
:106DC000504709900020E9F72197AE0145555244FC
:106DD00021E065E572E483E797E30F9466120F9074
:106DE0000F900F900F900F900F900F94250C882309
:106DF00071F181E00E94898A813069F48FE99EE314
:106E00000E94869C8FE99EE30E94989C0F94020C3E
:106E10000E948A9D02C00E94EB9DE6E3F1E480811E
:106E200090E0DC01AA5CBE4B25853685880F991F52
:106E3000FC01EA5CFE4B418152811F960C9161E09E
:106E400080EC9AE30E9489240F942C0D30C0E092CC
:106E5000D33FF092D43F0F94250C682FC8010E94B5
:106E6000678D0E949129811122C00F94250C1F92D9
:106E70008F9388E592E29F938F93C5E5D2E4DF93E9
:106E8000CF930F94504709900020E9F72197AE0166
:106E90004555524421E065E572E483E797E30F949A
:106EA00066120F900F900F900F900F900F908FE938
:106EB0009EE30E94869C0F94020CDF91CF911F915C
:106EC0000F91FF90EF90DF90CF9008958F929F9257
:106ED000AF92BF92CF92DF92EF920F931F93CF9317
:106EE000DF93EC0180E00E94DFB84B015C0120974A
:106EF00009F45CC11E8EFE01E15BFD4F1082CE01E4
:106F00000E94361F882309F451C16E0185E3C80E23
:106F1000D11CBE01625E7F4FC6010E941DEE8D8FA7
:106F200081111FC00E949129811119C08BE1ECE6EB
:106F3000F2E2A5E5B2E401900D928A95E1F7E5E56C
:106F4000F2E401900020E9F73197AF014555524432
:106F500021E065E572E483E797E30F94661281E030
:106F60008E8F61E075E4C6010E94E6F2FE01E25BED
:106F7000FD4F808381E095E40E9491BF8823A1F1B9
:106F800081E0FE01E15BFD4F808381E095E40E949A
:106F90002EBF0E949129811127C0FE01E15BFD4FA8
:106FA00080811F928F93319780811F928F9387E802
:106FB00092E29F938F9305E512E41F930F930F9432
:106FC0005047F80101900020E9F73197AF0145558E
:106FD000524421E0B80183E797E30F946612ADB7FE
:106FE000BEB71896ADBFBEBF8E8D813039F0FE01A1
:106FF000E15BFD4F8081813009F05CC00E949129E6
:10700000811119C08CE1EAE9F2E2A5E5B2E4019050
:107010000D928A95E1F7E5E5F2E401900020E9F7A9
:107020003197AF014555524421E065E572E483E7AD
:1070300097E30F9466126894EE24E2F806EB12E2EE
:10704000A5019401BE01685E7F4FCE0106960E94A5
:10705000E9548D8340E050E0BA01CE010E94BC2D7E
:107060008D81882309F4A2C082E00E9403B9062F13
:107070008BE00E9403B921E0611120E0BE016D5C4C
:107080007F4F44E65EE3C6010E94ED4DCE010E94B3
:107090008F1B9E01275A3D4FAE01485A5D4FBE01DE
:1070A0006D5A7D4FCE018E5A9D4F0E94432C0E94F7
:1070B000F2F97CC08E010A5F1F4FB80184E69EE39F
:1070C0000E94C1538D83811139C0A5019401BE0175
:1070D000685E7F4FC8010E9423518D8340E050E0DD
:1070E000BA01CE010E94BC2D8D81882309F45EC0B7
:1070F00082E00E9403B9062F8BE00E9403B921E0D1
:10710000611120E0BE016D5C7F4F44E65EE3C60185
:107110000E94ED4DCE010E948F1B9E01275A3D4FCC
:10712000AE01485A5D4FBE016D5A7D4FCE018E5A59
:107130009D4F0E94432C0E94F2F938C08E010C5AD8
:107140001D4F0F2EF4E6AF2EFEE3BF2EF02DF501FE
:107150006285738520E032E0A601C5010E94252DDD
:10716000015011096E01FEEACF1AFDEFDF0AD501C9
:107170001A966D917C911B979801A601C5010E94FA
:10718000572CFE01E85AFD4FD6018C918083C75AD7
:10719000DD4FF80180818883D5011A964D915D916C
:1071A0006D917C911D97C5010F94473DDF91CF9163
:1071B0001F910F91EF90DF90CF90BF90AF909F9075
:1071C0008F9008956DE281E197E3ABDA882309F4AB
:1071D00067C080918131882309F446C00E940C5F0A
:1071E00084E0809326060F948C0681E095E40E944B
:1071F00024CC80EC9AE36ADE80910F3D8823F1F085
:107200000E94E8C9813019F0823069F017C080917E
:107210000E3D882329F081E095E40E9486C90EC0C6
:107220000E9459C90BC080910E3D882329F081E04E
:1072300095E40E9408CB02C00E94D3CA109281310B
:107240000F942C0D80EC9AE30E94222281110F945E
:10725000950A80EC9AE30E942B296091023D80EC14
:107260009AE30E9481131CC00F942C0D0F94730A93
:1072700066E080EC9AE30E94811361E086EC9AE379
:107280000E948F530E940E510F942F1B0E94E25EAA
:1072900081E08093813184E0809325060F948C06F1
:1072A00080918131882331F00E94605D8111FCCF93
:1072B0008091813108954F925F926F927F928F9269
:1072C0009F92AF92BF92CF92DF92EF92FF921F9365
:1072D000CF93DF93CDB7DEB72797CDBFDEBF7C015D
:1072E0001092D04610E00F2E812CFBE49F2EA12C93
:1072F000B12CF02D0F2EF5E5CF2EF2E4DF2EF02D80
:107300000F2EF0E84F2EF5E25F2E612C712CF02D40
:10731000111120C080E096E9A0E0B0E0F701808381
:107320009183A283B3838AE0EBEBF2E2D601019072
:107330000D928A95E1F7F60101900020E9F7319767
:10734000AF014555524421E0B60183E797E30F941E
:1073500066125CC0113001F580EC92E1A0E0B0E073
:10736000F70180839183A283B38389E0E5ECF2E2A5
:10737000D60101900D928A95E1F7F6010190002067
:10738000E9F73197AF014555524421E0B60183E753
:1073900097E30F9466123AC01230E9F4D7014D9288
:1073A0005D926D927C92139789E0EEECF2E2D60149
:1073B00001900D928A95E1F7F60101900020E9F71E
:1073C0003197AF014555524421E0B60183E797E379
:1073D0000F9466121BC0F70180829182A282B38251
:1073E00089E0E7EDF2E2D60101900D928A95E1F78E
:1073F000F60101900020E9F73197AF01455552445D
:1074000021E0B60183E797E30F946612D701149643
:107410008C9114978D8315968C9115978E83169663
:107420008C9116978F838D919D910D90BC91A02D7D
:1074300089839A83AB83BC8360E185E00F946D24DC
:10744000BE016F5F7F4F80EA9AE00E94956C0F94B7
:107450009F0C08C083E496E40E9473CD813041F014
:107460000E94201B0F94B20C803A9F4098F37AC080
:1074700011111DC08CE0E0EEF2E2A5E5B2E401904E
:107480000D928A95E1F7E5E5F2E401900020E9F735
:107490003197AF014555524421E065E572E483E739
:1074A00097E30F94661282E08093D04678C0113043
:1074B000E9F48BE0ECEEF2E2A5E5B2E401900D9286
:1074C0008A95E1F7E5E5F2E401900020E9F73197CC
:1074D000AF014555524421E065E572E483E797E347
:1074E0000F94661281E08093D04659C01230E9F4BF
:1074F0008BE0E7EFF2E2A5E5B2E401900D928A9508
:10750000E1F7E5E5F2E401900020E9F73197AF01FA
:107510004555524421E065E572E483E797E30F9413
:10752000661283E08093D0463AC08BE0E2E0F3E25B
:10753000A5E5B2E401900D928A95E1F7E5E5F2E464
:1075400001900020E9F73197AF014555524421E001
:1075500065E572E483E797E30F94661284E0809315
:10756000D0461DC01F5F143009F0D2CE89E0EDE097
:10757000F3E2A5E5B2E401900D928A95E1F7E5E525
:10758000F2E401900020E9F73197AF0145555244EC
:1075900021E065E572E483E797E30F94661227968E
:1075A000CDBFDEBFDF91CF911F91FF90EF90DF90B5
:1075B000CF90BF90AF909F908F907F906F905F9093
:1075C0004F900895CF92DF92EF92FF920F931F9307
:1075D000CF9380EC9AE30E949413883009F4D6C0CC
:1075E00080EC9AE30E949413863009F4CFC0809116
:1075F0001B3D90911C3D8E349C4008F4BEC00E94FF
:10760000A6C08111B4C0C2C00F946D0D81111FC0FE
:107610000F94700D0E949129811119C088E1E6E153
:10762000F3E2A5E5B2E401900D928A95E1F7E5E574
:10763000F2E401900020E9F73197AF01455552443B
:1076400021E065E572E483E797E30F9466120F94F7
:10765000590D811129C09AC08CE1EEE2F3E2A5E553
:10766000B2E401900D928A95E1F7E5E5F2E401902C
:107670000020E9F73197AF014555524421E065E517
:1076800072E483E797E30F9466120F946A06C0E0F2
:107690000F945906882331F00F946A06CF5FCA30E1
:1076A000B9F702C0CA30A0F30F94730A0E940E51BA
:1076B0000E949129811119C08EE0ECE3F3E2A5E567
:1076C000B2E401900D928A95E1F7E5E5F2E40190CC
:1076D0000020E9F73197AF014555524421E065E5B7
:1076E00072E483E797E30F9466120F946A0601E051
:1076F00010E0C0E00F2EF2E1CF2EF1E2DF2EF02DF0
:107700000F2EF5E5EF2EF2E4FF2EF02D0F94590623
:10771000882341F10F946A06CF5F0E94912981115D
:107720001CC01F930F93DF92CF92FF92EF920F94A2
:107730005047F70101900020E9F73197AF01455517
:10774000524421E0B70183E797E30F9466120F904C
:107750000F900F900F900F900F900F5F1F4FC3303F
:1077600019F0D4CFC33090F20E941AF40FC00F94D6
:10777000630D882309F46BCF47CF8AEF90E40E9412
:10778000CF320E949129811180CF66CFCF911F9176
:107790000F91FF90EF90DF90CF900895F8940E94A2
:1077A00014620F9418240F942F1B0E94689B0E9450
:1077B000B6F60E942DD441E060EA78E08AE798E3CB
:1077C0000F94C81265E170E280EA98E00E940533E8
:1077D000E0EAF8E083818F7C8061838383EF9FE31D
:1077E0000F94031261E085ED9FE30E94A99C41E0A4
:1077F00060EA7BE08DE19DE30F94C8126EE070E2D9
:1078000080EA9BE00E940533E0EAFBE083818F7C05
:10781000806183838FE99EE30E94869C8FE99EE3CB
:107820000E94989C61E084EE9FE30E94A99C1092C4
:10783000F23F1092F94086E790E40F94031241E082
:1078400060EA7AE081E999E30F94C81267E070E298
:1078500080EA9AE00E940533E0EAFAE083818F7CB7
:107860008061838341E060EA79E083E797E30F94E6
:10787000C81260E070E280EA99E00E940533E0EA15
:10788000F9E083818F7C8061838387ED92E40F949C
:1078900003120F94F8050F940E080F949F090F948C
:1078A0003B0C0F9432080F940B0E0E94C9F40E94F7
:1078B0007DF80E94AC0EC0E060E08C2F0E94DAF6EA
:1078C000CF5FC830C9F787E08093A2007894E0E2E8
:1078D000F6E082E0868384E086830E949BB8811173
:1078E00010C00E94A1B90E94CBB90E94F2BE0E94B2
:1078F00082BF0E9477C00E94BEC081E080930D3D90
:1079000027C00E9465BE882309F181E080930D3D68
:107910000E94912981111CC08DE1EAE4F3E2A5E502
:10792000B2E401900D928A95E1F7E5E5F2E4019069
:107930000020E9F73197AF014555524421E065E554
:1079400072E483E797E30F94661202C010920D3D34
:107950000E94EABD0E94F2F90E9445BE81E00F94A8
:1079600051096DE281E197E30E9471330E949D9D70
:1079700064E773E483E496E40E94E7C583E496E455
:107980000E94C9C080EC9AE30E949B1380E00E9491
:10799000F6F781E095E40E9424CC80EC9AE396DA35
:1079A00081E00E9438B280E00E9432B280E00E9402
:1079B0003BB280E00E943EB20E94C6160E94A032F6
:1079C0000E946C9B83E496E40E94C9C087E090E229
:1079D00072DC0E94E8C9813029F480910E3D0E943A
:1079E000B6CF25C00E94E8C9823091F481E00E94A0
:1079F000EBC980910E3D882329F081E095E40E9437
:107A000008CB02C00E94D3CA81E00E949DCA0FC069
:107A10000E94E8C9833029F485E592E40E94CDCB29
:107A200006C00E94E8C9843011F40E94F4CF84E0BB
:107A3000809326060E9439D480EC9AE30E942B2979
:107A400083E797E30E949EA50E94E80E07E613E2F3
:107A5000C5E5D2E40E94433464E773E483E496E42A
:107A60000E94F11580EC9AE30E94821580EC9AE363
:107A70000E941A1580EC9AE30E94C62D80EC9AE3CE
:107A80000E94BC310E9448349DDB0E947C340E94DD
:107A9000B83480EC9AE30E942A1B0E9466D40E94AC
:107AA00035B2833031F50E944F1F882311F10E94B7
:107AB000912981111EC00F94500A1F928F931F931A
:107AC0000F93DF93CF930F945047FE010190002056
:107AD000E9F73197AF014555524421E0BE0183E7F4
:107AE00097E30F9466120F900F900F900F900F90E6
:107AF0000F908BE19DE30E94B62366E371E480EC76
:107B00009AE30E94142566E371E480EC9AE30E94F4
:107B100068250E9401F956DD0FB607FC9BCF80E077
:107B20000E9491770E94A577FFCFEF92FF920F936B
:107B30001F93CF93DF93009749F16115710541F1D0
:107B40004115510539F18A017B01EC010F94D746AB
:107B5000F80180839183892B89F0D70120E030E000
:107B6000FE01E20FF31FE491ED932F5F3F4FF80109
:107B7000808191812817390798F302C020E030E016
:107B8000F701E20FF31F108281E005C080E003C01F
:107B900080E001C080E0DF91CF911F910F91FF90B5
:107BA000EF9008950F931F93CF93DF930097C9F041
:107BB00061157105C1F041155105B9F0EA018B015C
:107BC000FC0165917491C8010F94D046F8010190B1
:107BD0000020E9F73197E01BF10BE883F98381E09E
:107BE00005C080E003C080E001C080E0DF91CF915C
:107BF0001F910F9108957F928F929F92AF92BF92A3
:107C0000CF92DF92EF92FF920F931F93CF93DF9368
:107C10001F921F92CDB7DEB7009709F49BC0611584
:107C2000710509F497C0D42E7B018C01AE014F5F22
:107C30005F4FBC018FE193E178DF882309F48AC0AC
:107C400089819A815C012FEFA21AB20AF801E80F2C
:107C5000F91F20E22083B8016A0D7B1DAE014F5F42
:107C60005F4F88E093E161DF882309F473C0898165
:107C70009A81A80EB91EF801EA0DFB1D8DE08083E4
:107C800082E0A80EB11C8AE08183B8016A0D7B1DD9
:107C9000AE014F5F5F4F81EF92E147DF882309F428
:107CA00059C0A981BA81AA0EBB1E48018A0C9B1C2F
:107CB0000F2EFDE07F2EF02DF40170820F2EFAE0E2
:107CC000CF2EF02DC182C5010296800F911F0E9418
:107CD000C1B8F401748ED5015E96C58EDD2059F1D0
:107CE000A00FB11F8AE0EFE6F3E201900D928A95B2
:107CF000E1F7F7E2AF0EB11C0E94C5BEBC01C8019E
:107D00008A0D9B1D0F9432470E94C5BEFC01019055
:107D10000020E9F73197E81BF90BE131F10518F480
:107D2000E983FA8304C080E190E089839A83A98182
:107D3000BA81AA0DBB1DF801EA0FFB1F8DE08083FD
:107D400012968AE08183F801EA0FFB1F1082F70187
:107D5000A083B1830F900F90DF91CF911F910F916E
:107D6000FF90EF90DF90CF90BF90AF909F908F905B
:107D70007F900895CF92DF92EF92FF920F931F931F
:107D8000CF93DF931F921F92CDB7DEB761157105B8
:107D900091F14115510579F1009769F17A016B0173
:107DA0008C0119821A82AE014F5F5F4F88EC91E11E
:107DB000BCDE882301F1C80106969F938F9389E763
:107DC00093E29F938F9389819A818C0D9D1D9F9340
:107DD0008F930F945047F60101900020E9F73197F7
:107DE000EC19FD09D701ED93FC930F900F900F90C4
:107DF0000F900F900F900F900F90DF91CF911F91E8
:107E00000F91FF90EF90DF90CF900895BF92CF92A7
:107E1000DF92EF92FF920F931F93CF93DF931F9206
:107E20001F92CDB7DEB7009709F482C061157105C6
:107E300009F47EC06B018C0119821A82DB011D924C
:107E40001C92AE014F5F5F4FBC018CEB91E16DDE88
:107E5000882309F46DC0E8EAF1E587858F9386856C
:107E60008F9385858F9384858F9383E09AE29F9388
:107E70008F9389819A81800F911F9F938F930F9485
:107E80005047F80101900020E9F73197E01BF10B12
:107E9000E983FA83CDBFDEBFB12C0F2EFEE7EF2EB4
:107EA000F3E2FF2EF02D2DC0EB2DF0E0EE0FFF1FC3
:107EB000EE0FFF1FE855FE4ADF015A9613968C918C
:107EC00013978F9312968C9112978F9311968C9192
:107ED0008F93828D8F93FF92EF9289819A81800F89
:107EE000911F9F938F930F945047F80101900020AA
:107EF000E9F73197E01BF10BE983FA83B394CDBF27
:107F0000DEBF0F94740DB81678F2E981FA81E00FA4
:107F1000F11F8DE09AE0808391831282F801019035
:107F20000020E9F73197E01BF10BD601ED93FC93AC
:107F30000F900F90DF91CF911F910F91FF90EF90D5
:107F4000DF90CF90BF900895AF92BF92CF92DF9213
:107F5000EF921F93CF93DF9300D01F92CDB7DEB780
:107F600019821A821B821C82009709F47FC0611556
:107F7000710509F47BC0E42E5B016C011FEF120F49
:107F80001B3008F068C0AE014F5F5F4FBC0184ED4D
:107F900091E1CBDD882309F469C01A3079F5EE2030
:107FA00069F069817A816C0D7D1DAE014D5F5F4F77
:107FB00088E898E0F7DD81110EC058C069817A81A8
:107FC0006C0D7D1DAE014D5F5F4F82E798E0EADDED
:107FD000882309F44BC069817A818B819C81680F69
:107FE000791F69837A836C0D7D1DAE014D5F5F4FF4
:107FF00084E798E0D7DD811124C038C0EE2089F0F5
:1080000069817A816C0D7D1D812F90E0880F991F09
:10801000AE014D5F5F4F8A58974FC4DD811111C08B
:1080200025C069817A816C0D7D1D812F90E0880FBC
:10803000991FAE014D5F5F4F805A974FB3DD882384
:10804000A9F029813A818B819C81820F931FF501D0
:10805000808391830BC0AE014F5F5F4FBC0184ED05
:1080600091E163DD882311F010E0C8CF2496CDBFE5
:10807000DEBFDF91CF911F91EF90DF90CF90BF9047
:10808000AF90089589E10E9403B981E0623009F060
:1080900080E00895CF92DF92EF92FF921F93CF93EB
:1080A000DF9300D01F92CDB7DEB719821A821B82F0
:1080B0001C82009709F453C06115710509F44FC083
:1080C000142F6B017C01AE014F5F5F4FBC0184ED4B
:1080D00091E12BDD882309F442C0173089F0193073
:1080E000E1F0113039F569817A816E0D7F1DAE01A5
:1080F0004D5F5F4F86E699E018DD811127C02FC0E4
:1081000069817A816E0D7F1DAE014D5F5F4F85E005
:1081100099E00BDD81111AC022C069817A816E0D50
:108120007F1DAE014D5F5F4F84EA98E0FEDC811158
:108130000DC015C069817A816E0D7F1DAE014D5F46
:108140005F4F86E699E0F1DC882349F029813A8186
:108150008B819C81820F931FF601808391832496EB
:10816000CDBFDEBFDF91CF911F91FF90EF90DF90E9
:10817000CF900895EF92FF920F931F93CF93DF93C9
:108180001F921F92CDB7DEB719821A82009751F164
:108190006115710539F17B018C0187E10E9403B9FA
:1081A000662351F0AE014F5F5F4FB8018DE592E15C
:1081B000BCDC81110AC016C0AE014F5F5F4FB80131
:1081C00080EE91E1B2DC882369F089819A81F8011F
:1081D000E80FF91F2DE020832AE021830296F701A2
:1081E000808391830F900F90DF91CF911F910F911A
:1081F000FF90EF900895EF92FF920F931F93CF930C
:10820000DF931F921F92CDB7DEB7009709F47EC0AF
:108210004115510509F47CC0F22E8A01E62EAE010B
:108220004F5F5F4FB801BEDC811102C019821A8214
:1082300083E0E81629F18E1538F091E0E91659F03F
:1082400082E0E81699F03AC094E0E91619F185E069
:10825000E81651F133C0E1E0F5E401900020E9F7C0
:108260003197E150F54461E075E42BC0E8E1F5E4B5
:1082700001900020E9F7E951F54468E175E421C077
:10828000EFE2F5E401900020E9F7E053F5446FE2F6
:1082900075E417C0E6E4F5E401900020E9F7E7543F
:1082A000F54466E475E40DC0EDE5F5E401900020C9
:1082B000E9F7EE55F5446DE575E403C061E075E45A
:1082C000E0E0EF3008F0EEE0CB018E0F911DFC01F5
:1082D000108289819A81800F911F0F943247F80193
:1082E00001900020E9F73197E01BF10BFF2091F09E
:1082F000C8018E0F911DFC018CE29DE0808391836B
:108300008AE090E08283938381E005C080E003C02F
:1083100080E001C081E00F900F90DF91CF911F911D
:108320000F91FF90EF9008958F929F92AF92BF921E
:10833000CF92DF92EF92FF920F931F93CF93DF9331
:108340001F921F92CDB7DEB730910E3D311104C0A0
:10835000FB011082118236C00097A1F1672B91F1C9
:108360004115510579F1022F4A016C010F2EF5E6F6
:10837000EF2EF8E1FF2EF02D11E0202FA601612F46
:10838000C70139DF8823A9F0F60101900020E9F741
:1083900031975F01AC18BD089E012F5F3F4FA501CB
:1083A000B601C4010F94473B89819A81A816B9068A
:1083B00031F41F5FF2E0EF0EF11C1630F1F6C4014C
:1083C0000F94F53C0F900F90DF91CF911F910F917B
:1083D000FF90EF90DF90CF90BF90AF909F908F90E5
:1083E00008958F929F92AF92BF92DF92EF92FF9289
:1083F0000F931F93CF93DF93CDB7DEB72597CDBFF4
:10840000DEBF009709F494C44115510509F492C4E4
:10841000D22E7A01162FAE014F5F5F4FB701C2DB3C
:10842000811102C019821A82163109F06DC00E94B2
:10843000D5E94B015C01672B682B692BE1F486E1E0
:108440000E9403B920E13EE040E050E00F94074570
:108450005F934F933F932F9389E893E29F938F937A
:1084600089819A818E0D9F1D9F938F930F94504702
:10847000CDBFDEBF46C486E10E9403B9992324F52F
:1084800086E10E9403B920E13EE040E050E00F9415
:108490000745CA01B9010F947F17BF92AF929F920F
:1084A0008F929F938F937F936F9384E893E29F9330
:1084B0008F9389819A818E0D9F1D9F938F930F9427
:1084C0005047CDBFDEBF1DC486E10E9403B9BF92F5
:1084D000AF929F928F9220E13EE040E050E00F94F7
:1084E00007455F934F933F932F9385E893E29F93C4
:1084F0008F9389819A818E0D9F1D9F938F930F94E7
:108500005047CDBFDEBFFDC3123060F4812F0E9403
:1085100068B929813A81BC01C701820F931F0F946A
:108520003247EFC3163081F486E00E9403B98B0115
:108530009C0189819A814BE0BE016B5F7F4F8E0D5C
:108540009F1D0F94D817DDC3153081F485E00E947C
:1085500003B98B019C0189819A814BE0BE016B5F5D
:108560007F4F8E0D9F1D0F942419CBC3123009F03D
:108570006EC082E00E9403B96C30710581059105DF
:1085800024F061E070E080E090E0013009F049C043
:1085900029813A812E0D3F1DDC01CB010197A109F4
:1085A000B109880F991FAE014D5F5F4FB901855327
:1085B000984FF8DA8130F9F4F70101900020E9F7DB
:1085C0003197EE19FF09E983FA8382E00E9403B92B
:1085D0009F938F937F936F938EE893E29F938F93F4
:1085E00089819A818E0D9F1D9F938F930F94504781
:1085F000CDBFDEBF86C382E00E9403B99F938F93F5
:108600007F936F938FE893E29F938F9389819A81F1
:108610008E0D9F1D9F938F930F945047CDBFDEBF4C
:1086200070C382E00E9403B99F938F937F936F93EF
:1086300084E09AE29F938F9389819A818E0D9F1D8A
:108640009F938F930F945047CDBFDEBF5AC31B300B
:1086500059F08DEE810F823038F089EE810F823033
:1086600018F01A3109F05CC0812F0E9403B94B0148
:108670005C01011113C0BF92AF929F926F9384E08F
:108680009AE29F938F9389819A818E0D9F1D9F936C
:108690008F930F945047CDBFDEBF33C3672B682B3A
:1086A000692BF9F469817A816E0D7F1DAE014D5FF2
:1086B0005F4F87EC97E039DA811123C31F921F9235
:1086C0001F921F9284E09AE29F938F9389819A81EF
:1086D0008E0D9F1D9F938F930F945047CDBFDEBF8C
:1086E00010C369817A816E0D7F1DAE014D5F5F4FB2
:1086F00084EC97E01ADA811104C3BF92AF929F9283
:108700008F9284E09AE29F938F9389819A818E0D54
:108710009F1D9F938F930F945047CDBFDEBFF1C233
:10872000173009F05CC087E00E9403B94B015C017F
:10873000011113C0BF92AF929F926F9384E09AE2AF
:108740009F938F9389819A818E0D9F1D9F938F9305
:108750000F945047CDBFDEBFD4C2672B682B692B67
:10876000F9F469817A816E0D7F1DAE014D5F5F4F17
:1087700080EC97E0DAD98111C4C21F921F921F9238
:108780001F9284E09AE29F938F9389819A818E0D44
:108790009F1D9F938F930F945047CDBFDEBFB1C2F3
:1087A00069817A816E0D7F1DAE014D5F5F4F8CEB4D
:1087B00097E0BBD98111A5C2BF92AF929F928F92D1
:1087C00084E09AE29F938F9389819A818E0D9F1DF9
:1087D0009F938F930F945047CDBFDEBF92C214304A
:1087E00009F05CC084E00E9403B94B015C010111F7
:1087F00013C0BF92AF929F926F9384E09AE29F93CF
:108800008F9389819A818E0D9F1D9F938F930F94D3
:108810005047CDBFDEBF75C2672B682B692BF9F4BB
:1088200069817A816E0D7F1DAE014D5F5F4F85EBD3
:1088300097E07BD9811165C21F921F921F921F92F0
:1088400084E09AE29F938F9389819A818E0D9F1D78
:108850009F938F930F945047CDBFDEBF52C2698163
:108860007A816E0D7F1DAE014D5F5F4F8CEA97E000
:108870005CD9811146C2BF92AF929F928F9284E0E1
:108880009AE29F938F9389819A818E0D9F1D9F936A
:108890008F930F945047CDBFDEBF33C2133009F022
:1088A000ABC083E00E9403B94B015C01011113C00E
:1088B000BF92AF929F926F9384E09AE29F938F93BF
:1088C00089819A818E0D9F1D9F938F930F9450479E
:1088D000CDBFDEBF16C291E089169104A104B10498
:1088E00061F182E088169104A104B10409F445C045
:1088F00081149104A104B10409F05FC069817A81F7
:108900006E0D7F1DAE014D5F5F4F80EA97E00DD980
:108910008111F7C11F921F921F921F9284E09AE269
:108920009F938F9389819A818E0D9F1D9F938F9323
:108930000F945047CDBFDEBFE4C169817A816E0DCF
:108940007F1DAE014D5F5F4F87E997E0EED8811143
:10895000D8C11F921F921F9281E08F9384E09AE208
:108960009F938F9389819A818E0D9F1D9F938F93E3
:108970000F945047CDBFDEBFC4C169817A816E0DAF
:108980007F1DAE014D5F5F4F82E997E0CED8811128
:10899000B8C11F921F921F9282E08F9384E09AE2E7
:1089A0009F938F9389819A818E0D9F1D9F938F93A3
:1089B0000F945047CDBFDEBFA4C169817A816E0D8F
:1089C0007F1DAE014D5F5F4F80EA97E0AED8811109
:1089D00098C1BF92AF929F928F9284E09AE29F9348
:1089E0008F9389819A818E0D9F1D9F938F930F94F2
:1089F0005047CDBFDEBF85C1193109F0ABC089E159
:108A00000E9403B94B015C01011113C0BF92AF92E8
:108A10009F926F9384E09AE29F938F9389819A81CA
:108A20008E0D9F1D9F938F930F945047CDBFDEBF38
:108A300068C191E089169104A104B10461F182E05A
:108A400088169104A104B10409F445C0811491046D
:108A5000A104B10409F05FC069817A816E0D7F1DA8
:108A6000AE014D5F5F4F8EE897E05FD8811149C13D
:108A70001F921F921F921F9284E09AE29F938F93FE
:108A800089819A818E0D9F1D9F938F930F945047DC
:108A9000CDBFDEBF36C169817A816E0D7F1DAE010B
:108AA0004D5F5F4F88E897E040D881112AC11F923F
:108AB0001F921F9281E08F9384E09AE29F938F939D
:108AC00089819A818E0D9F1D9F938F930F9450479C
:108AD000CDBFDEBF16C169817A816E0D7F1DAE01EB
:108AE0004D5F5F4F80E897E020D881110AC11F9247
:108AF0001F921F9282E08F9384E09AE29F938F935C
:108B000089819A818E0D9F1D9F938F930F9450475B
:108B1000CDBFDEBFF6C069817A816E0D7F1DAE01CB
:108B20004D5F5F4F8EE897E000D88111EAC0BF9299
:108B3000AF929F928F9284E09AE29F938F93898164
:108B40009A818E0D9F1D9F938F930F945047CDBF99
:108B5000DEBFD7C0123109F05EC082E10E9403B9C6
:108B60004B015C01011113C0BF92AF929F926F93B2
:108B700084E09AE29F938F9389819A818E0D9F1D45
:108B80009F938F930F945047CDBFDEBFBAC0672B22
:108B9000682B692B01F569817A816E0D7F1DAE010D
:108BA0004D5F5F4F8FE697E00E94953D8111A9C010
:108BB0001F921F921F921F9284E09AE29F938F93BD
:108BC00089819A818E0D9F1D9F938F930F9450479B
:108BD000CDBFDEBF96C069817A816E0D7F1DAE016B
:108BE0004D5F5F4F87E697E00E94953D811189C0F8
:108BF000BF92AF929F928F9284E09AE29F938F935D
:108C000089819A818E0D9F1D9F938F930F9450475A
:108C1000CDBFDEBF76C0153109F05EC085E10E9490
:108C200003B94B015C01011113C0BF92AF929F9237
:108C30006F9384E09AE29F938F9389819A818E0D3E
:108C40009F1D9F938F930F945047CDBFDEBF59C098
:108C5000672B682B692B01F569817A816E0D7F1D69
:108C6000AE014D5F5F4F8BE797E00E94953D81110C
:108C700048C01F921F921F921F9284E09AE29F9316
:108C80008F9389819A818E0D9F1D9F938F930F944F
:108C90005047CDBFDEBF35C069817A816E0D7F1D23
:108CA000AE014D5F5F4F86E797E00E94953D8111D1
:108CB00028C0BF92AF929F928F9284E09AE29F93D6
:108CC0008F9389819A818E0D9F1D9F938F930F940F
:108CD0005047CDBFDEBF15C0812F0E9403B99F93BF
:108CE0008F937F936F9384E09AE29F938F93898110
:108CF0009A818E0D9F1D9F938F930F945047CDBFE8
:108D0000DEBFF70101900020E9F73197EE19FF0966
:108D1000DD2091F0C7018E0F911DFC018CE29DE0DA
:108D2000808391838AE090E08283938381E005C011
:108D300080E003C080E001C081E02596CDBFDEBFAA
:108D4000DF91CF911F910F91FF90EF90DF90BF9037
:108D5000AF909F908F9008956F927F928F929F9285
:108D6000AF92BF92CF92DF92EF92FF920F931F9339
:108D7000CF93DF931F921F92CDB7DEB70097B1F16B
:108D8000672BA1F14115510589F1802E922E3A01F0
:108D90006C010F2EF4E1EF2EFAE1FF2EF02D10E022
:108DA000082D292DA601612FC7011BDB8823A9F0FF
:108DB000F60101900020E9F731975F01AC18BD087A
:108DC0009E012F5F3F4FA501B601C3010F94473BA2
:108DD00089819A81A816B90631F41F5F82E0E80EF6
:108DE000F11C1C31E9F6C3010F94F53C0F900F9074
:108DF000DF91CF911F910F91FF90EF90DF90CF9077
:108E0000BF90AF909F908F907F906F9008958F92BA
:108E10009F92AF92BF92DF92EF92FF920F931F93B8
:108E2000CF93DF931F921F92CDB7DEB7009709F45F
:108E30005EC06115710509F45AC04B017C010E94A6
:108E4000C5BE9F938F9385E993E29F938F93FF9283
:108E5000EF920F945047F70101900020E9F7319706
:108E6000AF014E195F094231510510F041E150E068
:108E70009E012F5F3F4FB701C4010F94473B0F90F6
:108E80000F900F900F900F900F90D12C0F2EF3ECAE
:108E9000AF2EF9E2BF2EF02D8D2D0E94DFB89F93EB
:108EA0008F937F936F93BF92AF92FF92EF920F9445
:108EB0005047F70101900020E9F731978F010E1913
:108EC0001F099E012F5F3F4FA801B701C4010F94F6
:108ED000473BCDBFDEBF89819A810817190721F46E
:108EE000D39496E1D912D8CFC4010F94F53C0F90DA
:108EF0000F90DF91CF911F910F91FF90EF90DF9036
:108F0000BF90AF909F908F9008952F923F924F9275
:108F10005F926F927F928F929F92AF92BF92CF9209
:108F2000DF92EF92FF920F931F93CF93DF93CDB712
:108F3000DEB7E197CDBFDEBF91E09BA7611571055C
:108F400009F4B7C34115510509F4B5C38A017B0182
:108F500089AB0F942C0D29A9213089F4A80162E86E
:108F600071E3CE010B960E943452182F86E08BA736
:108F70000E94A0FA6DA77EA78FA798AB1AC0A80180
:108F800062E871E3CE010B960E94A952182F0E944D
:108F9000A0FA6DA77EA78FA798AB82E00E9419F96F
:108FA000862FAE01445D5F4FBE01655D7F4F0E941D
:108FB0009721112309F481C341E0BE01675F7F4F10
:108FC000C7010E94FB3D49855A85CA01A0E0B0E077
:108FD00089839A83AB83BC839E01275F3F4FB70190
:108FE000CE010B960F94473BCE010B960F94F53CA8
:108FF000BE01655F7F4FC7010ADF0DE0D7010C930B
:109000001AE011961C939E01275F3F4F42E050E00B
:10901000B701CE010B960F94473BCE010B960F94F0
:10902000F53CE2E8F1E3018B128B9E01275F3F4F95
:1090300043E150E0BF01CE010B960F94473BCE01B8
:109040000B960F94F53CB9A9B1113DC30E94F5FAF6
:109050000E94DEFA38C301E021E0A701612FC601BA
:10906000C0D9882381F0F70101900020E9F73197FA
:10907000AF014E195F099E01275F3F4FB701CE0137
:109080000B960F94473BE2E0CE0ED11C1F5F1330CE
:1090900011F70F2EF6E2CF2EFAE1DF2EF02D19E0B8
:1090A00001E021E0A701612FC6019BD9882381F04F
:1090B000F70101900020E9F73197AF014E195F09E0
:1090C0009E01275F3F4FB701CE010B960F94473BA0
:1090D000F2E0CF0ED11C1F5F1B3011F70F2EF2E113
:1090E0008F2E912CA12CB12CF02D28E18216910409
:1090F000A104B10451F401E021E0A70169E186E493
:109100009AE16FD981110EC030C001E021E0A701C2
:10911000682DC401880F991F8C5E954E62D98823F3
:10912000C1F007C00F2EF9E18F2E912CA12CB12C8C
:10913000F02DF70101900020E9F73197AF014E19AA
:109140005F099E01275F3F4FB701CE010B960F9439
:10915000473B33E0830E911CA11CB11C4AE18416ED
:109160009104A104B10408F4C0CFCE010B960F9472
:10917000F53C89E00E9403B96F31710581059105C5
:10918000C0F4DC01CB01072E7CE0880F991FAA1FD9
:10919000BB1F7A95D1F7702D89839A83AB83BC83EB
:1091A00080E090E1A0E0B0E08D839E83AF83B8873C
:1091B00017C0DC01CB01072E79E0880F991FAA1F89
:1091C000BB1F7A95D1F7702D89839A83AB83BC83BB
:1091D00080E092E0A0E0B0E08D839E83AF83B8870B
:1091E00089819A81AB81BC812DA53EA54FA558A947
:1091F000281739074A075B07A1F1AE01475F5F4FA8
:10920000B70188E998E00E94953D813081F4F7012B
:1092100001900020E9F73197AF014E195F099E01D7
:10922000275F3F4FB701CE010B960F94473BCE010E
:109230000B960F94F53CCE010B960F943C3D39A94B
:1092400031113DC20E946CFB80EC9AE30E94222205
:1092500081110F94950A80EC9AE30E942B2980E0FB
:109260003AC2AE01475F5F4FB7018CE898E00E94B9
:10927000953D813081F4F70101900020E9F73197A5
:10928000AF014E195F099E01275F3F4FB701CE0125
:109290000B960F94473B48A94F935FA55F938EA50C
:1092A0008F939DA59F9388858F938F818F938E81B8
:1092B0008F938D818F9389E993E29F938F93FF9290
:1092C000EF920F945047F70101900020E9F7319792
:1092D000AF014E195F099E01275F3F4FB701CE01D5
:1092E0000B960F94473B88E290E089879A8768E263
:1092F000C7010E94D8A4482F50E060E070E0498385
:109300005A836B837C83682F70E0C7010F946819C0
:10931000CDBFDEBF8823C9F049815A819E01275FF6
:109320003F4FB701CE010B960F94473B8DE0F701FD
:1093300080838AE081839E01275F3F4F42E050E0B7
:10934000B701CE010B960F94473BBE016F5F7F4F75
:10935000C7010E94BA4049815A819E01275F3F4F51
:10936000B701CE010B960F94473B6BE370E0C7014A
:109370000E942BA4A0E0B0E089839A83AB83BC83D6
:109380000E94912981110EC0F70101900020E9F798
:109390003197AF014E195F0920E0B70183E797E3EA
:1093A0000F94661249815A816B817C814115510568
:1093B00061057105C1F09E01275F3F4FB701CE01E6
:1093C0000B960F94473B8DE0D7018C938AE0119662
:1093D0008C939E01275F3F4F42E050E0B701CE01E2
:1093E0000B960F94473BCE010B960F94F53C0E94D1
:1093F000C85619821A821B821C822DA53EA54FA534
:1094000058A9232B242B252B09F433C180E090E0AD
:10941000DC010F2EF2ED2F2EF3E23F2EF02D0F2E5A
:10942000F4EA8F2EF3E29F2EF02D880F991FAA1FCA
:10943000BB1FBC01CD017E5F8F4F9F4F0E94D05656
:109440000E945B598111FCCF80E091E0EBE4F1E4F4
:10945000DF019C011D9221503040E1F76F010F2E7A
:10946000FBE4AF2EF2E4BF2EF02D8F010E94ECA39F
:10947000D8018D939D938D01AA16BB06B9F70E9462
:109480009B570F942F1BCE010B960F94F53C412C4C
:10949000512C3201F601619171916F01AE014B5F68
:1094A0005F4F8BA50E948F14882309F496C088858E
:1094B0008F938F818F938E818F938D818F938981ED
:1094C0009A81AB81BC81840D951DA61DB71DBF93EC
:1094D000AF939F938F939F928F92FF92EF920F94EF
:1094E0005047F70101900020E9F73197AF014E197D
:1094F0005F099E01275F3F4FB701CE010B960F9486
:10950000473B182FCDBFDEBF882309F48CC00E94D3
:109510009129811126C089819A81AB81BC81840DFA
:10952000951DA61DB71DBF93AF939F938F931F9259
:109530001F934EEA53E25F934F93FF92EF920F9483
:109540005047F70101900020E9F73197AF014E191C
:109550005F0920E0B70183E797E30F946612CDBF60
:10956000DEBFF70101900020E9F73197AF014E19F6
:109570005F099E01275F3F4FB701CE010B960F9405
:10958000473B182F0E94912981114DC089819A81F2
:10959000AB81BC81840D951DA61DB71DBF93AF93F4
:1095A0009F938F931F921F93EFEBF3E2FF93EF9341
:1095B000FF92EF920F945047F70101900020E9F7D6
:1095C0003197AF014E195F0920E0B70183E797E3B8
:1095D0000F946612CDBFDEBF26C00E949129811173
:1095E00022C089819A81AB81BC81840D951DA61D05
:1095F000B71DBF93AF939F938F933F922F92FF928C
:10960000EF920F945047F70101900020E9F731974E
:10961000AF014E195F0920E0B70183E797E30F948C
:109620006612CDBFDEBF9FEF491A590A690A790A4F
:10963000A0E84A1651046104710409F02BCFCE0151
:109640000B960F94F53C89819A81AB81BC8180583F
:109650009F4FAF4FBF4F89839A83AB83BC832DA5A8
:109660003EA54FA558A982179307A407B50708F48C
:10967000DCCECE010B960F94F53CCE010B960F94E9
:109680003C3D1092933182E891E30E94885339A9BE
:10969000311117C00E946CFB80EC9AE30E942222D9
:1096A00081110F94950A80EC9AE30E942B2981E0A6
:1096B00012C080E010C080E00EC080E00CC080E0EE
:1096C0000AC081E008C00F2EF4E1CF2EFAE1DF2EB0
:1096D000F02D10E0C0CCE196CDBFDEBFDF91CF9181
:1096E0001F910F91FF90EF90DF90CF90BF90AF90C0
:1096F0009F908F907F906F905F904F903F902F90B2
:109700000895CF92DF92EF92FF920F931F93CF9322
:10971000DF931F921F92CDB7DEB7009709F457C0B1
:109720006115710509F453C07B018C01AE014F5FD7
:109730005F4FBC018FE193E10E94953D882309F4BE
:1097400046C089819A816C012FEFC21AD20AF801B2
:10975000E80FF91F20E22083B8016C0D7D1DAE01DA
:109760004F5F5F4F88E093E10E94953D882379F138
:1097700089819A81C80ED91EF801EC0DFD1D8DE07E
:10978000808382E0C80ED11C8AE08183B8016C0D11
:109790007D1DAE014F5F5F4F8AED92E10E94953DC6
:1097A0008823A9F089819A81C80ED91EF801EC0D91
:1097B000FD1D8DE0808322E0C20ED11C8AE08183F2
:1097C000F801EC0DFD1D1082F701C082D1820F90CF
:1097D0000F90DF91CF911F910F91FF90EF90DF904D
:1097E000CF900895EF92FF920F931F93CF93DF9343
:1097F000CDB7DEB7A297CDBFDEBF009709F451C049
:109800006115710509F44FC07B018C0160E0CE0148
:10981000039614D7882309F44BC0B701C80171DF40
:10982000F701408151819E012F5F3F4FB801CE016A
:1098300003960F94473BCE0103960F94F53CF70136
:109840002081318189819A812817390771F5BE01FC
:109850006D5F7F4FC801DBDAA701B8018CE49AE1A4
:109860000E94953D813099F4F701408151819E011C
:109870002F5F3F4FB801CE0103960F94473BF7018E
:109880002081318189819A812817390781F4CE019D
:1098900003960F943C3D81E011D70F942C0D81E08D
:1098A00007C080E005C080E003C080E001C080E028
:1098B000A296CDBFDEBFDF91CF911F910F91FF9098
:1098C000EF9008950F931F93CF93DF931F921F92F2
:1098D000CDB7DEB70F942C0D8091013D823009F495
:1098E00062C028F4882359F0813081F1D6C08430D9
:1098F00009F485C008F464C08A30E1F0CEC060E0AD
:1099000084E49EE37ED5811107C06091023D80EC26
:109910009AE30E948113C9C00E94F1F4811104C02E
:1099200081E08093013DC1C08AE08093013D0F94A6
:109930003D0BBBC00F94540B6C3D754081059105E8
:1099400008F4B3C081E08093013DAFC040E063EF15
:109950007AE385EF9AE30E94FB3D00EC1AE3F801FD
:1099600043A954A99E012F5F3F4F65EF7AE384E43A
:109970009EE30F94473B84E49EE30F94F53CF8018B
:1099800023A934A989819A812817390741F01092B7
:10999000013D6091023DC8010E94811386C082E0B2
:1099A0008093013D82C000E021E044E45EE363EF88
:1099B0007AE385EF9AE3D0D983E08093013D75C0C7
:1099C00043EF5AE365EF7AE38CE49AE10E94953D18
:1099D000813069F44091F33A5091F43A9E012F5F3F
:1099E0003F4F65EF7AE384E49EE30F94473B84E4C2
:1099F0009EE30F943C3D84E08093013D56C00E945D
:109A0000E8C9882381F10F94870C8823C9F00E944C
:109A10004F1F882309F449C080EC9AE30E94222258
:109A200081110F94950A80EC9AE30E942B291092E1
:109A3000013D6091023D80EC9AE30E94811335C0A4
:109A400080EC9AE30E94222281110F94950A80EC07
:109A50009AE30E942B291092013D61E080EC9AE389
:109A60000E94811322C00F94CF0A672B682B692BA9
:109A7000E1F480EC9AE30E94222281110F94950A6E
:109A800080EC9AE30E942B291092013D6091023DE7
:109A900080EC9AE30E94811308C01092013D60910E
:109AA000023D80EC9AE30E9481130F900F90DF91AA
:109AB000CF911F910F9108959F92AF92BF92CF9235
:109AC000DF92EF92FF920F931F93CF93DF9300D01B
:109AD000CDB7DEB7009709F471C06115710509F4BF
:109AE0006DC0A42E6B017C018EE0EDEDF3E2D70199
:109AF00001900D928A95E1F7F70101900020E9F7B6
:109B00003197EE19FF09E983AF0155279E012E5FBA
:109B10003F4FB701C6010F94473BB12C0F2EFCE21B
:109B20009F2EF02D8B2D0E9425C08B019C0148E0BB
:109B3000BE016F5F7F4FC7010F94861982E08B15BE
:109B400050F08981F701E80FF11D90828F5FF701D6
:109B5000E80FF11D1082F70101900020E9F731971D
:109B6000EE19FF09E983AF0155279E012E5F3F4F94
:109B7000B701C6010F94473B898190E02A813B8160
:109B80008217930721F4B394E4E0BE12CBCFAA204E
:109B900081F08DE0F70180838AE0818382E0898310
:109BA0009E012E5F3F4F42E050E0B701C6010F9487
:109BB000473BC6010F94F53C0F942C0D2396CDBF67
:109BC000DEBFDF91CF911F910F91FF90EF90DF905B
:109BD000CF90BF90AF909F9008959F92AF92BF9209
:109BE000CF92DF92EF92FF920F931F93CF93DF9369
:109BF0001F921F92CDB7DEB7009709F4E0C0611540
:109C0000710509F4DEC04115510509F4DCC0902E40
:109C1000122F5A016B017C010F942C0D41E0B6010B
:109C2000C7010E94FB3DF601408151819E012F5FDB
:109C30003F4FB701C5010F94473BC5010F94F53C59
:109C4000F6012081318189819A812817390709F02D
:109C5000BCC08DE0EBEEF3E2D70101900D928A9546
:109C6000E1F7F70101900020E9F73197AF014E19B4
:109C70005F0955279E012F5F3F4FB701C5010F9424
:109C8000473BC5010F94F53CB501C701C0D88DE035
:109C9000F70180838AE081839E012F5F3F4F42E07E
:109CA00050E0B701C5010F94473BC5010F94F53C47
:109CB00041E0B501C70100DFA601B70180EC9AE3DE
:109CC0000E94BA3EF601408151819E012F5F3F4FB5
:109CD000B701C5010F94473BC5010F94F53CF60150
:109CE0002081318189819A812817390709F06FC055
:109CF000B601C7010E94063FF601408151819E01D5
:109D00002F5F3F4FB701C5010F94473BC5010F942B
:109D1000F53CF6012081318189819A812817390724
:109D200009F057C001E021E0A501B601C70114D830
:109D300021E0A501B601C7010E9494410E94424062
:109D4000882331F0492DB601C7010E944A4006C060
:109D5000292D412FB601C7010E94A43FF601408181
:109D600051819E012F5F3F4FB701C5010F94473BC3
:109D7000C5010F94F53CF6012081318189819A81DA
:109D80002817390741F5B601C7010E94BA40F6010C
:109D9000408151819E012F5F3F4FB701C5010F9454
:109DA000473BC5010F94F53C81E0F60140815181AC
:109DB00029813A814217530779F080E00DC080E095
:109DC0000BC080E009C080E007C080E005C080E0F3
:109DD00003C080E001C080E00F900F90DF91CF9131
:109DE0001F910F91FF90EF90DF90CF90BF90AF90B9
:109DF0009F9008952F923F924F925F926F927F9221
:109E00008F929F92AF92BF92CF92DF92EF92FF928A
:109E10000F931F93CF93DF93CDB7DEB7A897CDBF36
:109E2000DEBF4115510509F4D7C12115310509F4EB
:109E3000D5C16115710509F4D3C1280169011A0161
:109E40007B0188A70F942C0DA60162E871E3CE0177
:109E50000796A7D6882309F4C5C141E0BE016B5F10
:109E60007F4FC1010E94FB3D4D815E819E012B5FB2
:109E70003F4FB101CE0107960F94473BCE010796A5
:109E80000F94F53CBE01695F7F4FC1010E940747F7
:109E90001DE0F10110830AE001839E012B5F3F4F1B
:109EA00042E050E0B101CE0107960F94473BCE014E
:109EB00007960F94F53CE2E8F1E3118B028B9E01CB
:109EC0002B5F3F4F43E150E0BF01CE0107960F9457
:109ED000473BCE0107960F94F53C0F2EF4E1CF2EB1
:109EE000FAE1DF2EF02D10E001E021E0A101612F69
:109EF000C6010E94F141882381F0F1010190002008
:109F0000E9F73197AF01421953099E012B5F3F4F8B
:109F1000B101CE0107960F94473BF2E0CF0ED11C62
:109F20001F5F133009F70F2EF6E2CF2EFAE1DF2E76
:109F3000F02D19E001E021E0A101612FC6010E948E
:109F4000F141882381F0F10101900020E9F7319778
:109F5000AF01421953099E012B5F3F4FB101CE0162
:109F600007960F94473B22E0C20ED11C1F5F1B30A7
:109F700009F70F2EF2E18F2E912CA12CB12CF02D90
:109F800088E188169104A104B10491F401E021E074
:109F9000A10169E186E49AE10E94F141811116C0B4
:109FA0000F2EFCE18F2E912CA12CB12CF02D31C065
:109FB00001E021E0A101682DC401880F991F8C5E8A
:109FC000954E0E94F1418823C1F007C00F2EF9E1A0
:109FD0008F2E912CA12CB12CF02DF101019000209D
:109FE000E9F73197AF01421953099E012B5F3F4FAB
:109FF000B101CE0107960F94473B93E0890E911C67
:10A00000A11CB11CEAE18E169104A104B10408F46C
:10A01000B7CF1F92F8A5FF9388EF93E29F938F939A
:10A020003F922F920F945047F10101900020E9F7E1
:10A030003197AF01421953099E012B5F3F4FB10188
:10A04000CE0107960F94473BCE0107960F94F53C3F
:10A05000612C712C0F900F900F900F900F900F901C
:10A06000411451046104710409F4A7C0870175010A
:10A070006401812C912C5401F8014191519161911D
:10A0800071918F019E012F5F3F4F88A50E94FD2D8A
:10A09000882309F482C08C818F938B818F938A816E
:10A0A0008F9389818F93BF92AF929F928F9284EA10
:10A0B00093E29F938F933F922F920F945047F10119
:10A0C00001900020E9F73197AF01421953099E0131
:10A0D0002B5F3F4FB101CE0107960F94473B8FA3F3
:10A0E000CDBFDEBF9FA1992309F457C00E949129DB
:10A0F00081111FC0FF92EF92DF92CF921F92EFA1CA
:10A10000EF938EEA93E29F938F933F922F920F9457
:10A110005047F10101900020E9F73197AF01421952
:10A12000530920E0B10183E797E30F946612CDBF96
:10A13000DEBFF10101900020E9F73197AF0142192C
:10A1400053099E012B5F3F4FB101CE0107960F943B
:10A15000473B8FA30E94912981111FC0FF92EF926C
:10A16000DF92CF921F929FA19F93EFEBF3E2FF93B9
:10A17000EF933F922F920F945047F10101900020EE
:10A18000E9F73197AF014219530920E0B10183E7A4
:10A1900097E30F946612CDBFDEBF9FEF891A990A2D
:10A1A000A90AB90AEFEFCE1ADE0AEE0AFE0A8414F3
:10A1B0009504A604B70408F45FCFCE0107960F9468
:10A1C000F53CCE0107960F943C3D1092933182E806
:10A1D00091E39ED281E007C080E005C080E003C02B
:10A1E00080E001C080E0A896CDBFDEBFDF91CF91B7
:10A1F0001F910F91FF90EF90DF90CF90BF90AF90A5
:10A200009F908F907F906F905F904F903F902F9096
:10A210000895089580919731089508951092973187
:10A2200080919631882331F01092963184E69EE336
:10A230000D943C3D089584E69EE30D943C3D0895C5
:10A24000809196310895CF92DF92EF92FF921F9303
:10A25000CF93DF93CDB7DEB76897CDBFDEBF6C017C
:10A260007B0184E1E3E0F4E2DE01159601900D92BA
:10A270008A95E1F7DA01C9010196A11DB11D883E59
:10A2800023E09207A105B1050CF460C01F921F9254
:10A290001F9281E08F9383EE90E29F938F93CE0184
:10A2A00001969F938F930F9450478981898B8A8160
:10A2B0008A8B8B818B8B80E38D838AE38E83CDBFEA
:10A2C000DEBFE114F10459F0D701FE0138969E017A
:10A2D000245F3F4F8D918193E217F307D9F710E385
:10A2E00046E0BE016B5F7F4F84E69EE30F94A93882
:10A2F00099EF980F9230C8F48B89893399F48A8941
:10A30000893361F48989893321F41092963180E090
:10A310003CC08F5F898B1A8B1B8BE2CF1B8B8F5FAF
:10A320008A8BDECF8F5F8B8BDBCF882321F010925F
:10A33000963180E02AC081E080939631BE01695F4A
:10A340007F4FC6010F94324781E01FC0BF93AF9388
:10A350009F938F9383EE90E29F938F93CE0101960C
:10A360009F938F930F9450478981898B8A818A8B21
:10A370008B818B8B80E38D838AE38E83CDBFDEBFA1
:10A38000E114F10409F0A0CFAACF6896CDBFDEBFDB
:10A39000DF91CF911F91FF90EF90DF90CF900895C4
:10A3A00080E00E9438F5882361F08250823030F5D9
:10A3B00080919731882311F1109297311092963144
:10A3C000089580919731811119C081E08093973170
:10A3D0008EE292E0E8E9F1E3DF019C011D92215059
:10A3E0003040E1F7BF0180E00F948B388B3019F4D7
:10A3F00010929631089581E08093963108958AE015
:10A400000895CF93DF93CDB7DEB76097CDBFDEBFA2
:10A41000009719F120E329832AE32A832BE0E7E15F
:10A42000F4E2DE01139601900D922A95E1F7613076
:10A4300041F441E0BE016F5F7F4F0F94A938982F20
:10A4400007C04AE0BE016F5F7F4F0F94A938982F75
:10A4500081E0992319F080E001C080E06096CDBFD3
:10A46000DEBFDF91CF910895DF92EF92FF920F93BD
:10A470001F93CF93DF93CDB7DEB76497CDBFDEBF19
:10A480008C0184E1E2E2F4E2DE01119601900D928A
:10A490008A95E1F70115110509F449C061157105A7
:10A4A00009F447C080E389838AE38A834115510513
:10A4B00059F0DA01FE0134969E01285F3F4F9D91CD
:10A4C0009193E217F307D9F77B010F2EF0E3DF2E0C
:10A4D000F02D46E0BE016F5F7F4FC8010F94A93891
:10A4E00099EF980F9230A8F49F85993379F48E856F
:10A4F000893341F48D858933F1F08F5F8D87DE8656
:10A50000DF86E7CFDF868F5F8E87E3CF9F5F9F87F2
:10A51000E0CF811112C081E1FE013396D701019095
:10A520000D928A95E1F7F701118A81E007C080E07A
:10A5300005C080E003C080E001C080E06496CDBF2C
:10A54000DEBFDF91CF911F910F91FF90EF90DF90D1
:10A550000895DF92EF92FF920F931F93CF93DF93B3
:10A56000CDB7DEB76497CDBFDEBF8C0184E1E6E3F3
:10A57000F4E2DE01119601900D928A95E1F7011542
:10A58000110509F449C06115710509F447C080E35C
:10A5900089838AE38A834115510559F0DA01FE0166
:10A5A00034969E01285F3F4F9D919193E217F307E8
:10A5B000D9F77B010F2EF0E3DF2EF02D46E0BE0130
:10A5C0006F5F7F4FC8010F94A93899EF980F9230B1
:10A5D000A8F49F85993379F48E85893341F48D856C
:10A5E0008933F1F08F5F8D87DE86DF86E7CFDF86E8
:10A5F0008F5F8E87E3CF9F5F9F87E0CF811112C06F
:10A6000081E1FE013396D70101900D928A95E1F721
:10A61000F701118A81E007C080E005C080E003C037
:10A6200080E001C080E06496CDBFDEBFDF91CF91B6
:10A630001F910F91FF90EF90DF9008950F931F935C
:10A64000CF93DF93CDB7DEB76097CDBFDEBF009766
:10A6500061F18C0180E389838AE38A838BE0EAE4F9
:10A66000F4E2DE01139601900D928A95E1F76130D4
:10A6700049F441E0BE016F5F7F4FC8010F94A938D4
:10A68000982F0EC041E060E0CE0103960F94193F71
:10A690004AE0BE016F5F7F4FC8010F94A938982F21
:10A6A00081E0992319F080E001C080E06096CDBF81
:10A6B000DEBFDF91CF911F910F910895CF93DF936C
:10A6C000CDB7DEB76097CDBFDEBF9BE0EAE4F4E232
:10A6D000DE01119601900D929A95E1F7813041F4D7
:10A6E00041E061E0CE0101960F94193F982F07C019
:10A6F00041E060E0CE0101960F94193F982F81E070
:10A70000911180E06096CDBFDEBFDF91CF910895BB
:10A71000009721F041E061E00D94193F08951F93E7
:10A72000CF93DF93CDB7DEB76497CDBFDEBF009781
:10A7300001F1162FBC0180E389838AE38A83CE016D
:10A7400003960F943247113041F441E061E0CE01AD
:10A7500001960F94193F982F07C041E060E0CE01A9
:10A7600001960F94193F982F81E0992319F080E00A
:10A7700001C080E06496CDBFDEBFDF91CF911F9115
:10A780000895EF92FF920F931F93CF93DF93CDB76E
:10A79000DEB76497CDBFDEBF6115710589F1009703
:10A7A00089F18B017C0180E389838AE38A83CE016E
:10A7B00003960F94324743E0BE016F5F7F4FC7019E
:10A7C0000F94A938873069F460E0C801A8DF982F9A
:10A7D0008823D9F043E0BE016F5F7F4FC7010F941C
:10A7E000A938811111C0F7014285538564857585AB
:10A7F000C7010F94473D91E0882339F090E005C0F0
:10A8000090E003C090E001C090E0892F6496CDBF36
:10A81000DEBFDF91CF911F910F91FF90EF900895D0
:10A82000CF93DF93CDB7DEB76097CDBFDEBF009784
:10A83000C1F020E329832AE32A832AE0E5E5F4E254
:10A84000DE01139601900D922A95E1F741E0BE01D9
:10A850006F5F7F4F0F94A93891E0882319F090E043
:10A8600001C090E0892F6096CDBFDEBFDF91CF9110
:10A8700008953F924F925F926F927F928F929F9234
:10A88000AF92BF92CF92DF92EF92FF920F931F93FE
:10A89000CF93DF93CDB7DEB76197CDBFDEBF611534
:10A8A000710509F470C0009709F46FC04115510596
:10A8B00009F46DC03FEF320F383008F06AC0322E15
:10A8C0007A018C01FB01138A41E00F94A9388111B0
:10A8D00062C0F8014285538564857585483EF3E082
:10A8E0005F076105710508F458C0413B84E05807D3
:10A8F0006105710508F053C0C32CD12C5601E6E068
:10A90000AE0EB11C25010B2C000C6608770844190B
:10A91000550966097709C8010F94473D811141C067
:10A92000A50160E070E0CE0103960F942B479E01D5
:10A930002F5F3F4FA501BE016D5F7F4FC8010F9490
:10A94000FB39C8010F943C3DFE01EC0DFD1D128644
:10A950008E010D5F1F4F812C912C5401A601B8016F
:10A96000C7010F941547892BF1F0FFEF8F1A9F0A4B
:10A97000AF0ABF0A0F5F1F4F481459046A047B04D3
:10A9800068F780E011C080E00FC080E00DC080E07B
:10A990000BC080E009C080E007C081E005C080E016
:10A9A00003C080E001C081E06196CDBFDEBFDF91D2
:10A9B000CF911F910F91FF90EF90DF90CF90BF90BC
:10A9C000AF909F908F907F906F905F904F903F904F
:10A9D00008954F925F926F927F92AF92BF92CF9203
:10A9E000DF92EF92FF920F931F93CF93DF93CDB738
:10A9F000DEB76897CDBFDEBF680114E1E3E0F4E2A3
:10AA0000DE01159601900D921A95E1F7009709F471
:10AA100091C0C114D10409F48FC0EFEFEE0DE830FE
:10AA200008F08CC0860129013A015B016C01283EC7
:10AA300083E03807410551050CF482C01F921F9234
:10AA40001F9281E08F9383EE90E29F938F93CE01CC
:10AA500001969F938F930F9450478981898B8A81A8
:10AA60008A8B8B818B8B80E38D838AE38E83CDBF32
:10AA7000DEBFA114B10459F0D501FE0138969E0144
:10AA8000245F3F4F8D918193E217F307D9F70F2E83
:10AA9000F0E3FF2EF02D46E0BE016B5F7F4F84E6B2
:10AAA0009EE30F94A93899EF980F923090F52E2DD0
:10AAB000A801BE016B5F7F4F84E69EE3DADE882348
:10AAC00079F060E0C6012BDE882351F04AE0BE0138
:10AAD0006B5F7F4F84E69EE30F94A9388823F9F0DB
:10AAE0009B89993399F48A89893361F489898933F7
:10AAF00021F41092963180E042C08F5F898BFA8AF0
:10AB0000FB8AC9CFFB8A8F5F8A8BC5CF9F5F9B8BE8
:10AB1000C2CF882321F01092963180E030C081E0CE
:10AB200080939631BE01695F7F4FC6010F94324713
:10AB300081E025C080E023C080E021C080E01FC00C
:10AB40007F926F925F922F9383EE90E29F938F9309
:10AB5000CE0101969F938F930F9450478981898BE3
:10AB60008A818A8B8B818B8B80E38D838AE38E83B2
:10AB7000CDBFDEBFA114B10409F07ECF88CF6896A7
:10AB8000CDBFDEBFDF91CF911F910F91FF90EF906E
:10AB9000DF90CF90BF90AF907F906F905F904F907D
:10ABA0000895DF92EF92FF920F931F93CF93DF935D
:10ABB000CDB7DEB76497CDBFDEBF8C0184E1EFE592
:10ABC000F4E2DE01119601900D928A95E1F70115EC
:10ABD000110509F449C06115710509F447C080E306
:10ABE00089838AE38A834115510559F0DA01FE0110
:10ABF00034969E01285F3F4F9D919193E217F30792
:10AC0000D9F77B010F2EF0E3DF2EF02D46E0BE01D9
:10AC10006F5F7F4FC8010F94A93899EF980F92305A
:10AC2000A8F49F85993379F48E85893341F48D8515
:10AC30008933F1F08F5F8D87DE86DF86E7CFDF8691
:10AC40008F5F8E87E3CF9F5F9F87E0CF811112C018
:10AC500081E1FE013396D70101900D928A95E1F7CB
:10AC6000F701118A81E007C080E005C080E003C0E1
:10AC700080E001C080E06496CDBFDEBFDF91CF9160
:10AC80001F910F91FF90EF90DF9008958091C63350
:10AC900008950895089581E08093C6330895109231
:10ACA000C6330895CF92DF92EF92FF920F931F93D6
:10ACB0006623B9F081111DC0C12CD12C760100E0B2
:10ACC00010E62AEE30E040E06CE170E280EB98E0C4
:10ACD0000F9423256CE170E280EB98E00F946D25D2
:10ACE00008C0811106C06CE170E280EB98E00F941F
:10ACF00083251F910F91FF90EF90DF90CF900895E3
:10AD0000CF93DF931F921F92CDB7DEB78091C733E9
:10AD10009091C833A091C933B091CA33072E75E121
:10AD2000B695A795979587957A95D1F7702D61E09F
:10AD3000B9DF87ED8A8341E050E0BE016E5F7F4F4F
:10AD400080EB98E00F943E2541E050E0BE016F5F3C
:10AD50007F4F80EB98E00F94552589818823A4F7D5
:10AD60008091C7339091C833A091C933B091CA3351
:10AD7000072E75E1B695A795979587957A95D1F7A2
:10AD8000702D60E08FDF0F900F90DF91CF910895CD
:10AD900080EB98E00F94EC241092CB3381E008957F
:10ADA0001F93CF93DF93CDB7DEB72C97CDBFDEBF18
:10ADB0006115710520E28207910508F0A1C0DC0150
:10ADC000CB018093C7339093C833A093C933B0931A
:10ADD000CA338091CB33811193DF1092CB338091B2
:10ADE000C7339091C833A091C933B091CA33072EAD
:10ADF00075E1B695A795979587957A95D1F7702DBA
:10AE000061E050DF82ED8C8741E050E0BE01645F7D
:10AE10007F4F80EB98E00F943E258091C73390914F
:10AE2000C833A091C933B091CA33AC01BD01032E20
:10AE300039E076956795579547953A95D1F7302D36
:10AE4000032E3AE0440F551F661F771F3A95D1F73E
:10AE5000302D9170AA27BB27842B952BA62BB72BBF
:10AE600089839A83AB83BC838B818D8341E050E0DF
:10AE7000BE016B5F7F4F80EB98E00F943E258A8187
:10AE80008E8341E050E0BE016A5F7F4F80EB98E027
:10AE90000F943E2589818F8341E050E0BE01695FB8
:10AEA0007F4F80EB98E00F943E2515E5188741E031
:10AEB00050E0BE01685F7F4F80EB98E00F943E2525
:10AEC000198741E050E0BE01675F7F4F80EB98E05B
:10AED0000F943E251A8741E050E0BE01665F7F4F28
:10AEE00080EB98E00F943E251B8741E050E0BE01C7
:10AEF000655F7F4F80EB98E00F943E2581E001C0B5
:10AF000080E02C96CDBFDEBFDF91CF911F910895D9
:10AF1000052E59E0660F771F881F991F5A95D1F7A4
:10AF2000502D6115710520E28207910510F438CF8C
:10AF3000089580E008958091C7339091C833A0911F
:10AF4000C933B091CA330097A105B10569F00197E3
:10AF5000A109B109072E75E1B695A7959795879533
:10AF60007A95D1F7702D01C080E060E09BDE1092F1
:10AF7000CB330895CF93DF93CDB7DEB72897CDBFFE
:10AF8000DEBF6115710520E28207910508F078C0E7
:10AF9000DC01CB018093C7339093C833A093C933AE
:10AFA000B093CA338091CB338111AADE1092CB3398
:10AFB0008091C7339091C833A091C933B091CA33FF
:10AFC000072E75E1B695A795979587957A95D1F750
:10AFD000702D61E067DE82E8888741E050E0BE01C5
:10AFE000685F7F4F80EB98E00F943E258091C733D8
:10AFF0009091C833A091C933B091CA33AC01BD015F
:10B00000032E39E076956795579547953A95D1F790
:10B01000302D032E3AE0440F551F661F771F3A95D7
:10B02000D1F7302D9170AA27BB27842B952BA62B07
:10B03000B72B89839A83AB83BC838B818D8341E05B
:10B0400050E0BE016B5F7F4F80EB98E00F943E2590
:10B050008A818E8341E050E0BE016A5F7F4F80EBC2
:10B0600098E00F943E2589818F8341E050E0BE0136
:10B07000695F7F4F80EB98E00F943E2581E001C02F
:10B0800080E02896CDBFDEBFDF91CF910895CF93AA
:10B09000DF931F92CDB7DEB78091C7339091C8334D
:10B0A000A091C933B091CA33AC01BD01517066277C
:10B0B0007727452B462B472B31F1198241E050E091
:10B0C000BE016F5F7F4F80EB98E00F943E2580912B
:10B0D000C7339091C833A091C933B091CA33019658
:10B0E000A11DB11D8093C7339093C833A093C9337A
:10B0F000B093CA33AC01BD01517066277727452B49
:10B10000462B472BD1F60097A105B10569F00197B1
:10B11000A109B109072E75E1B695A7959795879571
:10B120007A95D1F7702D01C080E060E0BBDD81E051
:10B130008093CB330F90DF91CF9108950F931F939E
:10B14000CF93DF931F92CDB7DEB78091CB338823A7
:10B15000B1F01092CB338091C7339091C833A09156
:10B16000C933B091CA33BC01CD01052E59E0969583
:10B170008795779567955A95D1F7502DC9DE41E0AF
:10B1800050E0BE016F5F7F4F80EB98E00F94552534
:10B190008091C7339091C833A091C933B091CA331D
:10B1A000AC01BD014F5F5F4F6F4F7F4F4093C7337F
:10B1B0005093C8336093C9337093CA338A019B019B
:10B1C000117022273327012B022B032BA1F4452BCF
:10B1D000462B472B51F0072E75E1B695A79597950D
:10B1E00087957A95D1F7702D01C080E060E05ADD37
:10B1F00081E08093CB3389810F90DF91CF911F91B4
:10B200000F9108950F931F93CF93DF931F92CDB7A4
:10B21000DEB7182F8091CB33882349F06091C73374
:10B220007091C8338091C9339091CA33A3DE1983DA
:10B2300041E050E0BE016F5F7F4F80EB98E00F94DC
:10B240003E258091C7339091C833A091C933B09106
:10B25000CA33AC01BD014F5F5F4F6F4F7F4F4093CB
:10B26000C7335093C8336093C9337093CA338A018C
:10B270009B01117022273327012B022B032BA1F4F2
:10B28000452B462B472B51F0072E75E1B695A79518
:10B29000979587957A95D1F7702D01C080E060E091
:10B2A00001DD81E08093CB3381E00F90DF91CF917E
:10B2B0001F910F910895CF93DF931F921F92CDB7E7
:10B2C000DEB78091CB33882309F440C08091C73327
:10B2D0009091C833A091C933B091CA33072E75E15C
:10B2E000B695A795979587957A95D1F7702D61E0DA
:10B2F000D9DC87ED8A8341E050E0BE016E5F7F4F6D
:10B3000080EB98E00F943E2541E050E0BE016F5F76
:10B310007F4F80EB98E00F9455258091C733909133
:10B32000C833A091C933B091CA33072E75E1B695E1
:10B33000A795979587957A95D1F7702D60E0B2DC47
:10B3400089818095881F8827881F01C080E00F9021
:10B350000F90DF91CF910895CF93DF93EC01803C64
:10B3600028E0920729F468E083E00F946D2410C070
:10B37000803C29E0920729F468E084E00F946D2472
:10B3800007C0803C9A4021F468E085E00F946D246A
:10B39000888180618883DF91CF910895EF92FF9239
:10B3A0000F931F93CF937C01C42FB901A80100E034
:10B3B00010E62AEE30E00E94D863882344F0F701BB
:10B3C0008081CC0FCC0FCC70837FC82BC083CF91F2
:10B3D0001F910F91FF90EF90089580E0089591E004
:10B3E000811101C090E09093843E81E080934420DD
:10B3F00008950F931F930DEC1BE52FE130E04CE017
:10B4000054E361E082E00E945B74811105C069EF42
:10B4100079E582E00E94AB751F910F910895CF935B
:10B42000DF931092EF331092F0330F94992581112E
:10B4300004C010920834D0E012C0815080930834C8
:10B440002ADCD82F882359F0C0E060E08C2F0F94BD
:10B45000AF25CF5F809108348C17B8F7CADF8D2FE6
:10B46000DF91CF910895C5CF08950F931F9303E304
:10B470001AE52DE030E048E450E260E081E80E9407
:10B480005B74811105C065E37AE581E80E94AB75C4
:10B490001F910F9108958091F033882341F082E04D
:10B4A0000E9484756BE47AE582E00C94AB75089594
:10B4B0008091F033882341F081E80E94847568E52B
:10B4C0007AE581E80C94AB750895809150209091B5
:10B4D0005120A0915220B0915320892B8A2B8B2B85
:10B4E00059F080911834882324F481E80E948475EF
:10B4F00003C082E00E9484758091103490911134D1
:10B50000A0911234B091133480934C2090934D202D
:10B51000A0934E20B0934F20A8CF0895E4EFF3E31B
:10B5200082E1DF011D928A95E9F780EF80838AE04E
:10B5300087830895DF92EF92FF920F931F93CF932B
:10B54000DF93D82EC62FD72F122F032FF42EE52EE0
:10B55000E5DF81E080935420E4EFF3E3D282E382DD
:10B56000F48205831683D487C587DF91CF911F911D
:10B570000F91FF90EF90DF90089520E030E0A90157
:10B5800060E074E285E0D6CF08950F931F93209179
:10B59000183442276CF000915020109151202091D6
:10B5A000522030915320061717072807390720F437
:10B5B000E4DF8BDF80E001C081E01F910F910895EF
:10B5C00020E030E0A90160E070E084E0B3CF0895AE
:10B5D0000F931F93262F30E00EE01BE5AC0161E0D6
:10B5E00081E80E945B74811102C0EADF6EDF1F9167
:10B5F0000F91089520E030E0A90160E078E286E054
:10B6000099CF089520E030E0A90160E07AE382E07C
:10B6100091CF089583DF109254200895CF93DF9344
:10B62000811111C0EB01F6DFE8E4F0E2808591853D
:10B63000A285B3858C1B9D0BA109B10980879187D9
:10B64000A287B38742DFDF91CF9108951F93CF93F5
:10B65000DF93D82F84E1E4EDF3E3DF011D928A95B7
:10B66000E9F7DD2331F090912334ECEDF3E318E0BA
:10B6700005C090911F34E8EDF3E314E080911D3490
:10B680008F738C3111F08F3339F48CE180838AE031
:10B69000818385E08383145FC12F911708F4C92F3C
:10B6A0008C2F90E0A0E0B0E040E8BC01CD016DDF60
:10B6B000882309F1809119340F94B625811102C0B5
:10B6C00020E001C020E8DD2361F0E4EDF3E3812F09
:10B6D00090E0029798278927982780839183238376
:10B6E00006C0E4EDF3E38FEF810F808322836C2F9C
:10B6F00084ED93E36DDFDF91CF911F910895CF9398
:10B70000C82F81110FC0809119340F94B62588235A
:10B7100049F020E030E0A90160E077E287E00ADF4D
:10B72000D4DE39C0AAEEB3E3ECE0F4E381891396EA
:10B730008C931397828912968C9312978389119612
:10B740008C93119784898C93A8EEB3E38689119624
:10B750008C93119787898C936091E8337091E933CA
:10B76000CB01A0E0B0E0BC01CD01052E59E0660F91
:10B77000771F881F991F5A95D1F7502DC11102C00C
:10B7800040E001C040E801DF882329F0C093EE3398
:10B7900081E08093EF33CF9108950F931F93CF9360
:10B7A000DF93811132C16F31710569F480910C34DE
:10B7B00090910D34A0910E34B0910F34853593459E
:10B7C000A244B34431F081E08093F03364DE70DE54
:10B7D0001CC1ECE0F4E395859F7095878091083457
:10B7E000891718F4CADE71DE10C1ECE0F4E340857D
:10B7F000518562857385409350205093512060930A
:10B80000522070935320478550E04B35510508F086
:10B81000EEC0FA018827E85BFE4F8F4F0D94234559
:10B82000C0911F34C33108F0C2E18C2F90E0A0E03A
:10B83000B0E040E8BC01CD01A8DE882309F4E5C0F2
:10B840006C2F84EF93E3C4DEE0C0C0911F34C53297
:10B8500008F0C4E28C2F90E0A0E0B0E040E8BC012A
:10B86000CD0193DE882309F4D0C080911C3483700D
:10B8700021F4D0911D34DD2319F07FDE26DEC5C012
:10B88000809119340F94BD258111D0E800E210E2B7
:10B89000F801D183809119340F94C42520E1FC0173
:10B8A0003196A0E3B0E201900D922A95E1F7F801FC
:10B8B0008089882309F4A4C0823209F4A3C0E1E39B
:10B8C000F0E281E09191992309F49DC0923209F44C
:10B8D0009AC08F5F8031B1F708C0E82FF0E0E05EDA
:10B8E000FF4D908B8F5F8031C1F76C2F80E290E22B
:10B8F0006FDE8BC080E0AADE88C081E0A7DE85C055
:10B90000892F0F949B25823039F0833019F08111F3
:10B9100005C006C06FDE05C075DE03C051DE01C084
:10B9200079DED3DD72C040E868E070E080E090E04E
:10B930002CDE882309F469C06CEC73E38091193420
:10B940000F94A225823041F0833019F0811107C095
:10B9500009C050DEBADD59C055DEB7DD56C030DE55
:10B96000B4DD53C0ECECF3E380E090E0A2E0B0E0A3
:10B9700084839583A683B78380819181A281B381DB
:10B980005A2F4B2F60E070E0982789279827A0E076
:10B99000B0E0DC0199278827842B952BA62BB72BA9
:10B9A00080839183A283B38368E0CF0111DE2DC031
:10B9B00080911F3481FF06C08095682F6170892FA8
:10B9C0000F94AF2527DE81DD20C080911F348111C7
:10B9D00002C020DE01C0D1DD78DD17C01BDE75DDC1
:10B9E00014C081E08CDE11C080E089DE0EC020E052
:10B9F00030E0A90160E070E285E09CDD66DD05C015
:10BA000080E001C080E090E268CFDF91CF911F918C
:10BA10000F9108951092EF3342C9089580918D3EA1
:10BA20008823F4F480768032D9F580918E3E8E3F63
:10BA3000C9F58091933E9091943E0197A9F580912C
:10BA40008F3E9091903E892B89F5EDE8FEE388E0EA
:10BA500094E38087918781E090E0828793870895BF
:10BA60008076803229F580918E3E8F3F19F5809146
:10BA7000933E9091943E892BF9F480918F3E909162
:10BA8000903E892BD9F41092F0331092EF3382E07C
:10BA90000E94197581E80E941975ABDC81E0089558
:10BAA00080E0089580E0089580E0089580E00895A2
:10BAB00080E0089580E0089580E0089580E0089592
:10BAC000CF93C091EF33CC23A9F11092EF33809143
:10BAD000EE33882389F02091E8333091E9334091A7
:10BAE000EA335091EB336091EC337091ED338091F8
:10BAF00019340F94CC2510C02091E8333091E933EC
:10BB00004091EA335091EB336091EC337091ED3317
:10BB1000809119340F94F025823041F0833021F068
:10BB2000811106C077DD05C065DD03C06BDD01C096
:10BB300047DDCBDC8C2FCF910895EF92FF920F93CE
:10BB40001F93CF93DF93982F80914420882309F48B
:10BB500048C0109244202115310511F0890102C01E
:10BB60000FEE19E5911102C082E001C081E8E90100
:10BB70007A01AB01970160E00E945B74811104C0FF
:10BB800091E0909344202DC0CD2BD9F48091442096
:10BB90008823E1F38091843E811122C0E8E4F0E241
:10BBA00080859185A285B3858E199F09A109B10968
:10BBB00080879187A287B3879091843E81E089270F
:10BBC00010C0E8E4F0E240855185628573854E1926
:10BBD0005F0961097109408751876287738701C0D6
:10BBE00080E0DF91CF911F910F91FF90EF9008952A
:10BBF000E0913134F09132340190F081E02D2281D6
:10BC000033812E0F3F1FFC014081E40FF11DE2172D
:10BC1000F307A0F481818430A1F0861306C014C01C
:10BC200081818430A1F08617A9F08081E80FF11D91
:10BC3000E217F307A8F380E090E0089580E090E039
:10BC4000089580E090E008958E2F9F2F089580E062
:10BC500090E008958E2F9F2F089580918F3E8F77CB
:10BC60000C947673089590913334992381F1E09187
:10BC70003134F09132340190F081E02D94818917B4
:10BC800040F5E0932F34F0933034228133812E0F2E
:10BC90003F1FE217F307F8F49181943061F4928129
:10BCA000891309C09381961306C0E0932F34F09353
:10BCB000303481E008959081E90FF11DE217F30718
:10BCC00058F3E0932F34F093303480E0089580E00F
:10BCD000089580E0089580E00895EF92FF921F9309
:10BCE000CF93DF93C82F60E0BEDF182F882381F148
:10BCF000A0913134B0913234EC2FF0E0EE0FFF1F01
:10BD000012968D919C911397E80FF91FE080F180B6
:10BD1000D7011696ED91FC9117971995682F8C2FE6
:10BD2000A2DF182F8823A1F0C0912F34D091303496
:10BD300065E0CE015DDFEC01892B21F08A810E9454
:10BD40006875F6CFD7011296ED91FC91139719956E
:10BD5000812FDF91CF911F91FF90EF9008951F9356
:10BD6000CF93DF93182F7FDF882341F1C0912F34C9
:10BD7000D091303465E0CE013BDFEC01892B49F0F6
:10BD80004C815D816B818A810E9483738111F2CF26
:10BD900015C0A0913134B0913234E12FF0E0EE0FB4
:10BDA000FF1F12968D919C911397E80FF91F019038
:10BDB000F081E02D0190F081E02D1995DF91CF9178
:10BDC0001F9108950C940E730895CF93809133348E
:10BDD0008823C1F0E0913134F09132340190F08148
:10BDE000E02D8481882371F0C0E08C2F76DFCF5F57
:10BDF000E0913134F09132340190F081E02D848172
:10BE0000C81798F31092333481E090E08093343473
:10BE100090933534CF9108950E94DA72D6CF089569
:10BE2000CF9380913334882349F1A0913134B0917C
:10BE30003234ED91FC91119784818823F9F0C0E0B0
:10BE4000EC2FF0E0EE0FFF1F12968D919C9113974F
:10BE5000E80FF91F0190F081E02D0084F185E02DBD
:10BE6000309709F01995CF5FA0913134B0913234F9
:10BE7000ED91FC9111978481C81710F3CF9108952B
:10BE80000F931F93CF93DF93EDE8FEE312861386A3
:10BE90001486158616861786808188230CF060C26A
:10BEA0002091933E3091943E2115310509F05DC2F9
:10BEB0004FC28F7109F097C090918E3E963081F0FD
:10BEC000983009F485C091118EC02230310509F0F7
:10BED000FBC162E070E084E394E30E947C734EC295
:10BEE00080918F3E9091903E292F3327223031054B
:10BEF00089F02330310579F12130310509F0A6C1EF
:10BF00008091622090916320DC016C9170E00E942E
:10BF10007C734FC0E0916220F091632021898217E9
:10BF200008F0D2C19927880F991F880F991FE091B7
:10BF30006420F0916520E80FF91F80819181FC0158
:10BF4000628173810E947C73E091953EF091963EF0
:10BF500082E081832EC099278130910599F058F0B5
:10BF60008230910509F406C2039709F078C13CE0DC
:10BF7000E3E7F4E20AC064E070E088EC90E20E943B
:10BF80007C7317C0EEEBF0E239E0A2EAB0E220E009
:10BF9000819190E08D939D932F5F2317C8F3632FBA
:10BFA000660F6E5F6093A02070E080EA90E20E94CE
:10BFB0007C73EDE8FEE386819781228533858217C5
:10BFC000930708F0DBC18093973E9093983ED6C1CB
:10BFD0002130310509F078C161E070E083E394E33A
:10BFE0000E947C73CBC18130E9F590918E3E9A30EE
:10BFF000C9F52130310509F037C1809133348823E8
:10C0000009F432C1C091913ED091923E00913134F9
:10C0100010913234D801ED91FC918481C81708F059
:10C0200023C160E08C2F1FDE882309F418C1CE01E4
:10C030009927880F991FD8011296ED91FC911397BB
:10C04000E80FF91F0190F081E02D86819781FC01B6
:10C05000199580932E3461E070E08EE294E30E94A3
:10C060007C738CC1823009F0FAC080918E3E8111C0
:10C07000EFC02230310509F027C18091913E0E9426
:10C080000B7490E080932C3490932D3462E070E038
:10C090008CE294E30E947C7371C18F7109F084C0BB
:10C0A00090918E3E933009F4D5C018F49130A1F0F0
:10C0B0007BC0953019F0993039F176C08091933E6C
:10C0C0009091943E892B09F0FFC08DE29EE580930C
:10C0D000993E90939A3E52C18091933E9091943EA6
:10C0E000892B09F0F1C080918F3E9091903E01978D
:10C0F00009F0EAC080913434909135348D7F80937B
:10C100003434909335343AC18091933E9091943E6B
:10C11000892B09F0D9C00E947973882309F49FC044
:10C1200020918F3E3091903E3327E0916220F09134
:10C130006320818990E08217930708F490C045DE60
:10C1400080918F3E9091903E80933334882309F400
:10C1500015C199278150904C880F991F880F991FFE
:10C16000E0916420F0916520E80FF91FE0933134ED
:10C17000F09332340190F081E02D8481882309F41A
:10C18000FDC0C0E060E08C2FEADD882309F467C0C1
:10C19000CF5FE0913134F09132340190F081E02DA5
:10C1A0008481C81778F3EAC08130E9F490918E3E1B
:10C1B0009B30C9F48091933E9091943E892B09F075
:10C1C00053C080913334882309F44EC0EDE8FEE378
:10C1D000C481D2818C2F81DD882309F440C06D2F6A
:10C1E0008C2FBDDD3AC08230D1F580918E3E8130FA
:10C1F00019F08330A1F030C08091933E9091943E2D
:10C20000892B09F061C080918F3E9091903E892BDF
:10C2100009F05AC08091913E0E9426741EC0809100
:10C22000933E9091943E892B09F04EC080918F3EB1
:10C230009091903E892B09F047C0CDE8DEE38C81D8
:10C240000E9419758C810E94847507C080E005C02A
:10C2500080E003C080E001C080E0811190C0809147
:10C260008D3E8F71813081F580913334882309F4BC
:10C2700071C00091913E1091923EC0913134D091A5
:10C280003234E881F9818481081708F065C060E0E4
:10C29000802FE9DC8823C1F0F801FF27CF01880F48
:10C2A000991FEA81FB81E80FF91FC081D181EE81DE
:10C2B000FF811995682F802FD6DC882329F0EC8127
:10C2C000FD81199581115BC080918D3E8F71823007
:10C2D00009F044C0809133348823B1F1A091313406
:10C2E000B0913234ED91FC9111978481882371F1E2
:10C2F000C0E0EC2FF0E0EE0FFF1F12968D919C91A5
:10C300001397E80FF91F00811181D8011696ED915E
:10C31000FC9117971995682F8C2FA5DC882379F14C
:10C32000D8011496ED91FC9115971995811127C0AC
:10C33000CF5FA0913134B0913234ED91FC911197DF
:10C340009481C917B0F21BC080E019C080E017C00B
:10C3500080E015C080E013C080E011C080E00FC015
:10C36000982F907609F07BCF98CE982F907609F091
:10C3700076CF9FCD33E0EAEBF0E207CE81E0DF91AC
:10C38000CF911F910F9108958038910558F1672B37
:10C3900021F4873C910571F41CC08F3F910509F091
:10C3A000F8F49C01220F331FF901E05CF84D808105
:10C3B00091810895E2E4F8E221E030E04191519169
:10C3C0008417950741F02F5F3F4F20383105B1F7B3
:10C3D00002C020E030E020583F4FC901992708955E
:10C3E00080E090E008958136910589F0E2E6F6E27A
:10C3F00040E050E04F5F5F4F2191319121153105B1
:10C4000091F028173907B1F7892B19F40AC040E0D9
:10C4100050E0440F551FFA01E058FB4D8081918197
:10C42000089580E090E0089543E050E060E880E007
:10C4300096E00F94C52443E050E064E080E296E08B
:10C440000F94C52443E050E062E080E296E00F9450
:10C45000C52440E058E160E280EA96E00F94C524EC
:10C4600041E050E062E080EA96E00F94C52443E0AA
:10C4700050E060E180E896E00F94C52443E050E08E
:10C4800060E180E496E00F94C52441E050E061E073
:10C4900080E496E00F94C52441E050E062E080E43F
:10C4A00096E00F94C52441E050E060E280E696E01B
:10C4B0000F94C52441E050E062E080E096E00F94E4
:10C4C000C52441E050E062E080E896E00F94C52486
:10C4D00043E050E062E080E696E00F94C52440E03F
:10C4E00050E061E080EA96E00F94C52440E050E01F
:10C4F00061E080E096E00F94C52440E050E068E001
:10C5000080E096E00F94C52441E050E060E480E0D4
:10C5100096E00F94C52440E058E161E080E896E0A1
:10C520000F94C52440E050E061E080E096E00F9475
:10C53000C52440E050E060E280E096E00F94C5241E
:10C5400040E050E064E080E096E00F94C52440E0D5
:10C5500050E061E080EA96E00F94C52443E050E0AB
:10C5600060E880E496E00F94C52443E050E060E288
:10C5700080E496E00F94C52440E050E060E480E45D
:10C5800096E00F94C52441E050E060E880E896E032
:10C590000F94C52441E050E060E280E896E00F94FB
:10C5A000C52440E050E060E480E896E00F94C524A4
:10C5B00043E050E068E080E496E00F94C52440E05A
:10C5C00050E064E080E496E00F94C52443E050E03E
:10C5D00068E080E696E00F94C52440E050E064E017
:10C5E00080E696E00F94C52443E050E068E080E8E0
:10C5F00096E00F94C52440E050E064E080E896E0C7
:10C600000F94C52443E050E068E080EA96E00F9480
:10C61000C52440E050E064E080EA96E00F94C52431
:10C6200040E058E160E480EA96E00F94C52440E0E1
:10C6300058E160E180E696E00F94C52440E058E1BF
:10C6400061E080E296E00F94C52443E050E060E8AA
:10C6500080E496E00F94C52443E050E060E280E47B
:10C6600096E00F94C52440E050E060E480E496E05A
:10C670000F94C52443E050E060E880EA96E00D9412
:10C68000C52408951F920F920FB60F9211240BB676
:10C690000F928F939F93EF93FF93E5E8FEE38081E2
:10C6A0009181019680839183FF91EF919F918F916A
:10C6B0000F900BBE0F900FBE0F901F9018951F92FA
:10C6C0000F920FB60F9211240BB60F92CF92DF92FA
:10C6D000EF92FF920F931F932F933F934F935F938C
:10C6E0006F937F938F939F93AF93BF93EF93FF933A
:10C6F000E5E8FEE3808191812281338182179307EF
:10C70000F0F121E020930204E0918B3EF0918C3E09
:10C710003097A9F16091080470910904A0E0B0E09D
:10C72000DC0199278827AB0160E070E08C019D0156
:10C73000042B152B262B372BC901B801A5E8BEE326
:10C7400012960D911C91139720E030E0980111276B
:10C7500000271496CD90DC901597E12CF12C0C2934
:10C760001D292E293F29061717072807390730F0FA
:10C77000C901B8016F5F7F4F8F4F9F4F1995FF9190
:10C78000EF91BF91AF919F918F917F916F915F9149
:10C790004F913F912F911F910F91FF90EF90DF905C
:10C7A000CF900F900BBE0F900FBE0F901F9018955B
:10C7B000CF92DF92EF92FF920F931F93CF93DF936D
:10C7C000EC016A017B01DB01CA010197A109B109F2
:10C7D000BC01CD01600F711F821F931FA70196013D
:10C7E0000F94E5442138310541055105F8F4213411
:10C7F00060F4213260F4213160F4293060F4253096
:10C8000060F4233060F490E80BC093E009C092E03C
:10C8100007C092E805C091E003C091E801C090E034
:10C8200088818C77892B888381E001C08FEFDF912D
:10C83000CF911F910F91FF90EF90DF90CF900895CF
:10C840001F920F920FB60F9211240BB60F922F93D7
:10C850003F934F935F936F937F938F939F93AF9388
:10C86000BF93EF93FF93E0917C34F0917D34309748
:10C8700009F01995FF91EF91BF91AF919F918F9121
:10C880007F916F915F914F913F912F910F900BBED0
:10C890000F900FBE0F901F9018951F920F920FB61A
:10C8A0000F9211240BB60F922F933F934F935F93E8
:10C8B0006F937F938F939F93AF93BF93EF93FF9368
:10C8C000E0917A34F0917B34309709F01995FF911B
:10C8D000EF91BF91AF919F918F917F916F915F91F8
:10C8E0004F913F912F910F900BBE0F900FBE0F9065
:10C8F0001F9018951F920F920FB60F9211240BB62E
:10C900000F922F933F934F935F936F937F938F93E8
:10C910009F93AF93BF93EF93FF93E0917834F0919F
:10C920007934309709F01995FF91EF91BF91AF914C
:10C930009F918F917F916F915F914F913F912F9137
:10C940000F900BBE0F900FBE0F901F9018951F9267
:10C950000F920FB60F9211240BB60F922F933F93A5
:10C960004F935F936F937F938F939F93AF93BF93F7
:10C97000EF93FF93E0917634F0917734309709F09C
:10C980001995FF91EF91BF91AF919F918F917F91F9
:10C990006F915F914F913F912F910F900BBE0F9030
:10C9A0000FBE0F901F9018951F920F920FB60F9207
:10C9B00011240BB60F922F933F934F935F936F9376
:10C9C0007F938F939F93AF93BF93EF93FF93E091E8
:10C9D0007434F0917534309709F01995FF91EF9107
:10C9E000BF91AF919F918F917F916F915F914F9187
:10C9F0003F912F910F900BBE0F900FBE0F901F9085
:10CA000018951F920F920FB60F9211240BB60F922A
:10CA10002F933F934F935F936F937F938F939F9346
:10CA2000AF93BF93EF93FF93E0917234F09173341F
:10CA3000309709F01995FF91EF91BF91AF919F91B8
:10CA40008F917F916F915F914F913F912F910F90B7
:10CA50000BBE0F900FBE0F901F9018951F920F9254
:10CA60000FB60F9211240BB60F922F933F934F9353
:10CA70005F936F937F938F939F93AF93BF93EF9346
:10CA8000FF93E0917034F0917134309709F019956B
:10CA9000FF91EF91BF91AF919F918F917F916F9196
:10CAA0005F914F913F912F910F900BBE0F900FBE52
:10CAB0000F901F9018951F920F920FB60F9211248E
:10CAC0000BB60F922F933F934F935F936F937F9388
:10CAD0008F939F93AF93BF93EF93FF93E0916E3447
:10CAE000F0916F34309709F01995FF91EF91BF9154
:10CAF000AF919F918F917F916F915F914F913F91F6
:10CB00002F910F900BBE0F900FBE0F901F90189596
:10CB10001F920F920FB60F9211240BB60F922F9304
:10CB20003F934F935F936F937F938F939F93AF93B5
:10CB3000BF93EF93FF93E0916C34F0916D34309795
:10CB400009F01995FF91EF91BF91AF919F918F914E
:10CB50007F916F915F914F913F912F910F900BBEFD
:10CB60000F900FBE0F901F9018951F920F920FB647
:10CB70000F9211240BB60F922F933F934F935F9315
:10CB80006F937F938F939F93AF93BF93EF93FF9395
:10CB9000E0916A34F0916B34309709F01995FF9168
:10CBA000EF91BF91AF919F918F917F916F915F9125
:10CBB0004F913F912F910F900BBE0F900FBE0F9092
:10CBC0001F9018951F920F920FB60F9211240BB65B
:10CBD0000F922F933F934F935F936F937F938F9316
:10CBE0009F93AF93BF93EF93FF93E0916834F091DD
:10CBF0006934309709F01995FF91EF91BF91AF918A
:10CC00009F918F917F916F915F914F913F912F9164
:10CC10000F900BBE0F900FBE0F901F9018951F9294
:10CC20000F920FB60F9211240BB60F922F933F93D2
:10CC30004F935F936F937F938F939F93AF93BF9324
:10CC4000EF93FF93E0916634F0916734309709F0E9
:10CC50001995FF91EF91BF91AF919F918F917F9126
:10CC60006F915F914F913F912F910F900BBE0F905D
:10CC70000FBE0F901F9018951F920F920FB60F9234
:10CC800011240BB60F922F933F934F935F936F93A3
:10CC90007F938F939F93AF93BF93EF93FF93E09115
:10CCA0006434F0916534309709F01995FF91EF9154
:10CCB000BF91AF919F918F917F916F915F914F91B4
:10CCC0003F912F910F900BBE0F900FBE0F901F90B2
:10CCD00018951F920F920FB60F9211240BB60F9258
:10CCE0002F933F934F935F936F937F938F939F9374
:10CCF000AF93BF93EF93FF93E0916234F09163346D
:10CD0000309709F01995FF91EF91BF91AF919F91E5
:10CD10008F917F916F915F914F913F912F910F90E4
:10CD20000BBE0F900FBE0F901F9018951F920F9281
:10CD30000FB60F9211240BB60F922F933F934F9380
:10CD40005F936F937F938F939F93AF93BF93EF9373
:10CD5000FF93E0916034F0916134309709F01995B8
:10CD6000FF91EF91BF91AF919F918F917F916F91C3
:10CD70005F914F913F912F910F900BBE0F900FBE7F
:10CD80000F901F9018951F920F920FB60F921124BB
:10CD90000BB60F922F933F934F935F936F937F93B5
:10CDA0008F939F93AF93BF93EF93FF93E0915E3484
:10CDB000F0915F34309709F01995FF91EF91BF9191
:10CDC000AF919F918F917F916F915F914F913F9123
:10CDD0002F910F900BBE0F900FBE0F901F901895C4
:10CDE0001F920F920FB60F9211240BB60F922F9332
:10CDF0003F934F935F936F937F938F939F93AF93E3
:10CE0000BF93EF93FF93E0915C34F0915D343097E2
:10CE100009F01995FF91EF91BF91AF919F918F917B
:10CE20007F916F915F914F913F912F910F900BBE2A
:10CE30000F900FBE0F901F9018951F920F920FB674
:10CE40000F9211240BB60F922F933F934F935F9342
:10CE50006F937F938F939F93AF93BF93EF93FF93C2
:10CE6000E0915A34F0915B34309709F01995FF91B5
:10CE7000EF91BF91AF919F918F917F916F915F9152
:10CE80004F913F912F910F900BBE0F900FBE0F90BF
:10CE90001F9018951F920F920FB60F9211240BB688
:10CEA0000F922F933F934F935F936F937F938F9343
:10CEB0009F93AF93BF93EF93FF93E0915834F0911A
:10CEC0005934309709F01995FF91EF91BF91AF91C7
:10CED0009F918F917F916F915F914F913F912F9192
:10CEE0000F900BBE0F900FBE0F901F9018951F92C2
:10CEF0000F920FB60F9211240BB60F922F933F9300
:10CF00004F935F936F937F938F939F93AF93BF9351
:10CF1000EF93FF93E0915634F0915734309709F036
:10CF20001995FF91EF91BF91AF919F918F917F9153
:10CF30006F915F914F913F912F910F900BBE0F908A
:10CF40000FBE0F901F9018951F920F920FB60F9261
:10CF500011240BB60F922F933F934F935F936F93D0
:10CF60007F938F939F93AF93BF93EF93FF93E09142
:10CF70005434F0915534309709F01995FF91EF91A1
:10CF8000BF91AF919F918F917F916F915F914F91E1
:10CF90003F912F910F900BBE0F900FBE0F901F90DF
:10CFA00018951F920F920FB60F9211240BB60F9285
:10CFB0002F933F934F935F936F937F938F939F93A1
:10CFC000AF93BF93EF93FF93E0915234F0915334BA
:10CFD000309709F01995FF91EF91BF91AF919F9113
:10CFE0008F917F916F915F914F913F912F910F9012
:10CFF0000BBE0F900FBE0F901F9018951F920F92AF
:10D000000FB60F9211240BB60F922F933F934F93AD
:10D010005F936F937F938F939F93AF93BF93EF93A0
:10D02000FF93E0915034F0915134309709F0199505
:10D03000FF91EF91BF91AF919F918F917F916F91F0
:10D040005F914F913F912F910F900BBE0F900FBEAC
:10D050000F901F9018951F920F920FB60F921124E8
:10D060000BB60F922F933F934F935F936F937F93E2
:10D070008F939F93AF93BF93EF93FF93E0914E34C1
:10D08000F0914F34309709F01995FF91EF91BF91CE
:10D09000AF919F918F917F916F915F914F913F9150
:10D0A0002F910F900BBE0F900FBE0F901F901895F1
:10D0B0001F920F920FB60F9211240BB60F922F935F
:10D0C0003F934F935F936F937F938F939F93AF9310
:10D0D000BF93EF93FF93E0914C34F0914D34309730
:10D0E00009F01995FF91EF91BF91AF919F918F91A9
:10D0F0007F916F915F914F913F912F910F900BBE58
:10D100000F900FBE0F901F9018951F920F920FB6A1
:10D110000F9211240BB60F922F933F934F935F936F
:10D120006F937F938F939F93AF93BF93EF93FF93EF
:10D13000E0914A34F0914B34309709F01995FF9102
:10D14000EF91BF91AF919F918F917F916F915F917F
:10D150004F913F912F910F900BBE0F900FBE0F90EC
:10D160001F9018951F920F920FB60F9211240BB6B5
:10D170000F922F933F934F935F936F937F938F9370
:10D180009F93AF93BF93EF93FF93E0914834F09157
:10D190004934309709F01995FF91EF91BF91AF9104
:10D1A0009F918F917F916F915F914F913F912F91BF
:10D1B0000F900BBE0F900FBE0F901F9018951F92EF
:10D1C0000F920FB60F9211240BB60F922F933F932D
:10D1D0004F935F936F937F938F939F93AF93BF937F
:10D1E000EF93FF93E0914634F0914734309709F084
:10D1F0001995FF91EF91BF91AF919F918F917F9181
:10D200006F915F914F913F912F910F900BBE0F90B7
:10D210000FBE0F901F9018951F920F920FB60F928E
:10D2200011240BB60F922F933F934F935F936F93FD
:10D230007F938F939F93AF93BF93EF93FF93E0916F
:10D240004434F0914534309709F01995FF91EF91EE
:10D25000BF91AF919F918F917F916F915F914F910E
:10D260003F912F910F900BBE0F900FBE0F901F900C
:10D2700018951F920F920FB60F9211240BB60F92B2
:10D280002F933F934F935F936F937F938F939F93CE
:10D29000AF93BF93EF93FF93E0914234F091433407
:10D2A000309709F01995FF91EF91BF91AF919F9140
:10D2B0008F917F916F915F914F913F912F910F903F
:10D2C0000BBE0F900FBE0F901F9018951F920F92DC
:10D2D0000FB60F9211240BB60F922F933F934F93DB
:10D2E0005F936F937F938F939F93AF93BF93EF93CE
:10D2F000FF93E0914034F0914134309709F0199553
:10D30000FF91EF91BF91AF919F918F917F916F911D
:10D310005F914F913F912F910F900BBE0F900FBED9
:10D320000F901F9018951F920F920FB60F92112415
:10D330000BB60F922F933F934F935F936F937F930F
:10D340008F939F93AF93BF93EF93FF93E0913E34FE
:10D35000F0913F34309709F01995FF91EF91BF910B
:10D36000AF919F918F917F916F915F914F913F917D
:10D370002F910F900BBE0F900FBE0F901F9018951E
:10D380001F920F920FB60F9211240BB60F922F938C
:10D390003F934F935F936F937F938F939F93AF933D
:10D3A000BF93EF93FF93E0913C34F0913D3430977D
:10D3B00009F01995FF91EF91BF91AF919F918F91D6
:10D3C0007F916F915F914F913F912F910F900BBE85
:10D3D0000F900FBE0F901F9018951F920F920FB6CF
:10D3E0000F9211240BB60F922F933F934F935F939D
:10D3F0006F937F938F939F93AF93BF93EF93FF931D
:10D40000E0913A34F0913B34309709F01995FF914F
:10D41000EF91BF91AF919F918F917F916F915F91AC
:10D420004F913F912F910F900BBE0F900FBE0F9019
:10D430001F9018951F920F920FB60F9211240BB6E2
:10D440000F922F933F934F935F936F937F938F939D
:10D450009F93AF93BF93EF93FF93E0913834F09194
:10D460003934309709F01995FF91EF91BF91AF9141
:10D470009F918F917F916F915F914F913F912F91EC
:10D480000F900BBE0F900FBE0F901F9018951F921C
:10D490000F920FB60F9211240BB60F922F933F935A
:10D4A0004F935F936F937F938F939F93AF93BF93AC
:10D4B000EF93FF93E0913634F0913734309709F0D1
:10D4C0001995FF91EF91BF91AF919F918F917F91AE
:10D4D0006F915F914F913F912F910F900BBE0F90E5
:10D4E0000FBE0F901F901895CF93CFB7F894282FA9
:10D4F000392F211588E0380749F461E083E00F9463
:10D500006D2464E083E00F946D244FC0203488E0E4
:10D51000380749F462E083E00F946D2464E083E00F
:10D520000F946D2442C0211589E0380749F461E069
:10D5300084E00F946D2464E084E00F946D2435C082
:10D54000203489E0380749F462E084E00F946D24C8
:10D5500064E084E00F946D2428C021158AE0380728
:10D5600049F461E085E00F946D2464E085E00F9458
:10D570006D241BC020348AE0380749F462E085E05E
:10D580000F946D2464E085E00F946D240EC0211586
:10D590003B4049F461E086E00F946D2464E086E04E
:10D5A0000F946D2402C0CFBF01C0CFBFCF910895AB
:10D5B000CF93CFB7F894282F392F211588E038075B
:10D5C00049F461E083E00F94792464E083E00F94F0
:10D5D00079244FC0203488E0380749F462E083E0C2
:10D5E0000F94792464E083E00F94792442C02115DC
:10D5F00089E0380749F461E084E00F94792464E01D
:10D6000084E00F94792435C0203489E0380749F448
:10D6100062E084E00F94792464E084E00F9479243C
:10D6200028C021158AE0380749F461E085E00F94AD
:10D63000792464E085E00F9479241BC020348AE0CB
:10D64000380749F462E085E00F94792464E085E0CE
:10D650000F9479240EC021153B4049F461E086E027
:10D660000F94792464E086E00F94792402C0CFBF40
:10D6700001C0CFBFCF910895811528E0920729F40A
:10D6800060937C3470937D340895803428E0920751
:10D6900029F460937034709371340895811529E0F2
:10D6A000920729F460936834709369340895803444
:10D6B00029E0920729F460935C3470935D340895F7
:10D6C00081152AE0920729F46093543470935534FD
:10D6D000089580342AE0920729F4609348347093C7
:10D6E0004934089581159B4021F460934034709330
:10D6F00041340895FC01918195FFFDCF608380E066
:10D7000090E008954F925F926F927F928F929F92D6
:10D71000AF92BF92EF92FF920F931F93CF937C0132
:10D720004A015B0128013901FC01848182FF16C096
:10D73000D901C801689412F8B695A7959795879571
:10D740001694D1F7B901A801032E36E176956795B5
:10D75000579547953A95D1F7302D15C0D901C80195
:10D76000689413F8B695A795979587951694D1F771
:10D77000B901A801032E37E176956795579547952E
:10D780003A95D1F7302D88159905AA05BB0508F4FF
:10D79000A6C084169506A606B70608F4A2C0F7012F
:10D7A000848182FD04C0880C991CAA1CBB1CC30187
:10D7B000B201A50194010F94E5442F3F31054105C5
:10D7C000510508F490C08FEF90E0A0E0B0E0C9EF01
:10D7D00005C0281739074A075B0758F0880F991FBB
:10D7E000AA1FBB1FCD3F0CF48160CF5FC73089F704
:10D7F0004FC0CC230CF04CC0D501C401880F991F39
:10D80000AA1FBB1F880F991FAA1FBB1F880F991F34
:10D81000AA1FBB1F481A590A6A0A7B0ACE3FF4F4B2
:10D820008DEF9FEF8C1B9109C7FD939504C0440CAD
:10D83000551C661C771C8A95D2F7D501C401B69594
:10D84000A79597958795BC01CD01640D751D861D23
:10D85000971DA50194010F94E54437C083E08C0F18
:10D86000A501940104C0220F331F441F551F8A9540
:10D87000D2F7DA01C901B695A79597958795BC01AE
:10D88000CD01640D751D861D971D0F94E5441DC0C7
:10D8900083E08C0FA501940104C0220F331F441FA5
:10D8A000551F8A95D2F7DA01C901B695A7959795C4
:10D8B0008795BC01CD01640D751D861D971D0F94C4
:10D8C000E5442150310941095109832F8F70C295D8
:10D8D000C07FC82BF701C783268381E018C080E092
:10D8E00016C080E014C0D501C401880F991FAA1F7B
:10D8F000BB1F880F991FAA1FBB1F880F991FAA1F44
:10D90000BB1F481A590A6A0A7B0AC9EF89CFCF910F
:10D910001F910F91FF90EF90BF90AF909F908F90CD
:10D920007F906F905F904F9008950F931F93CF93C8
:10D93000DF93EC018B01009709F41EC1803C910537
:10D9400029F460E180E00F946D2416C1C11584E0D4
:10D95000D80729F464E080E00F946D240DC1C0382D
:10D96000E1E0DE0729F462E080E00F946D2404C159
:10D97000C115F1E0DF0729F461E080E00F946D2428
:10D98000FBC0C03883E0D80729F461E081E00F9440
:10D990006D24F2C0C039E3E0DE0729F461E082E0E3
:10D9A0000F946D24E9C0C115F2E0DF0729F462E0AD
:10D9B00081E00F946D24E0C0C03482E0D80729F4E0
:10D9C00062E082E00F946D24D7C0C032E3E0DE074E
:10D9D00029F464E082E00F946D24CEC0C115F8E014
:10D9E000DF0729F461E083E00F946D24C5C0C11501
:10D9F00089E0D80729F461E084E00F946D24BCC06D
:10DA0000C115EAE0DE0729F461E085E00F946D249A
:10DA1000B3C0C115FBE0DF0729F461E086E00F9495
:10DA20006D24AAC0C03488E0D80729F462E083E0FE
:10DA30000F946D24A1C0C034E9E0DE0729F462E050
:10DA400084E00F946D2498C0C034FAE0DF0729F415
:10DA500062E085E00F946D248FC0C03988E0D8075C
:10DA600029F464E083E00F946D2486C0C039E9E0B6
:10DA7000DE0729F464E084E00F946D247DC0C03992
:10DA8000FAE0DF0729F464E085E00F946D2474C0A8
:10DA9000C0398BE0D80729F464E086E00F946D2448
:10DAA0006BC0C03CE8E0DE0729F468E083E00F9437
:10DAB0006D2462C0C03CF9E0DF0729F468E084E02F
:10DAC0000F946D2459C0C03C8AE0D80729F468E05F
:10DAD00085E00F946D2450C0C03AE8E0DE0729F4D9
:10DAE00060E183E00F946D2447C0C03AF9E0DF079E
:10DAF00029F460E184E00F946D243EC0C03A8AE0CE
:10DB0000D80729F460E185E00F946D2435C0C03A50
:10DB1000EBE0DE0729F460E186E00F946D242CC071
:10DB2000C03BF8E0DF0729F460E283E00F946D2446
:10DB300023C0C03B89E0D80729F460E284E00F9459
:10DB40006D241AC0C03BEAE0DE0729F460E285E0FC
:10DB50000F946D2411C0C038F4E0DF0729F460E4AD
:10DB600083E00F946D2408C0C03A84E0D80721F404
:10DB700060E485E00F946D248D818F738D83F801AF
:10DB800095818481892B9681911198E0892B8D83D1
:10DB9000F801408151816281738100E010E62AEE34
:10DBA00030E0CE01AFDD9C8198609C839C819061C8
:10DBB0009C83DF91CF911F910F910895CF92DF92B7
:10DBC000EF92FF920F931F93CF93DF93EC01D90154
:10DBD000C801B695A79597958795481759076A077D
:10DBE0007B0778F46A017B01CC0CDD1CEE1CFF1C6A
:10DBF000C901B801A70196010F94E54421503109EC
:10DC000002C020E030E0832F8F708F832E83DF915E
:10DC1000CF911F910F91FF90EF90DF90CF900895DB
:10DC2000EF92FF920F931F93CF93DF93EC017B0151
:10DC3000009709F4B9C1803C910529F460E180E0C6
:10DC40000F946D24B1C18115944029F464E080E003
:10DC50000F946D24A9C1C03881E0D80729F462E08F
:10DC600080E00F946D24A0C1C115E1E0DE0729F426
:10DC700061E080E00F946D2497C1C038F3E0DF07C6
:10DC800029F461E081E00F946D248EC1C03933E046
:10DC9000D30729F461E082E00F946D2485C1C1159A
:10DCA00082E0D80729F462E081E00F946D247CC102
:10DCB000C034E2E0DE0729F462E082E00F946D24D4
:10DCC00073C1C032F3E0DF0729F464E082E00F940F
:10DCD0006D246AC1C11538E0D30729F461E083E0FF
:10DCE0000F946D2461C1C11589E0D80729F461E062
:10DCF00084E00F946D2458C1C115EAE0DE0729F4D1
:10DD000061E085E00F946D244FC1C115FBE0DF0792
:10DD100029F461E086E00F946D2446C1C03438E0F8
:10DD2000D30729F462E083E00F946D243DC1C03431
:10DD300089E0D80729F462E084E00F946D2434C1AF
:10DD4000C034EAE0DE0729F462E085E00F946D2438
:10DD50002BC1C039F8E0DF0729F464E083E00F94B9
:10DD60006D2422C1C03939E0D30729F464E084E08E
:10DD70000F946D2419C1C0398AE0D80729F464E0F2
:10DD800085E00F946D2410C1C039EBE0DE0729F463
:10DD900064E086E00F946D2407C1C03CF8E0DF0723
:10DDA00029F468E083E00F946D24FEC0C03C39E0A4
:10DDB000D30729F468E084E00F946D24F5C0C03CDB
:10DDC0008AE0D80729F468E085E00F946D24ECC060
:10DDD000C03AE8E0DE0769F460E183E00F946D2467
:10DDE000E0EAF8E084818F7E8483F7012481225069
:10DDF00053C0C03AF9E0DF0729F460E184E00F94F2
:10DE00006D24D2C0C03A3AE0D30729F460E185E03E
:10DE10000F946D24C9C0C03A8BE0D80729F460E1A3
:10DE200086E00F946D24C0C0C03BE8E0DE0729F413
:10DE300060E283E00F946D24B7C0C03BF9E0DF07D8
:10DE400029F460E284E00F946D24AEC0C03B3AE058
:10DE5000D30729F460E285E00F946D24A5C0C03893
:10DE600084E0D80729F460E483E00F946D249CC01B
:10DE7000C03AE4E0DE0729F460E485E00F946D2405
:10DE800093C08C818F7E8C83FB0124812250CE0134
:10DE9000C03AF8E0DF0731F480914E0684FD8CC073
:10DEA00011E18BC0803B38E0930779F0803AE9E0DC
:10DEB0009E0731F430916E0634FD82C019E110C026
:10DEC000803BF9E09F0789F001C015E1803A3AE014
:10DED000930731F480918E0684FD74C011E212C064
:10DEE000803BEAE09E0759F001C01DE1803A9B406B
:10DEF00049F48091AE0684FD04C019E203C015E226
:10DF000001C01DE2E12FE695E695E69530E2E39F3C
:10DF1000F0011124FA5F177081E090E0012E02C039
:10DF2000880F991F0A94E2F78183223010F040E0B5
:10DF300001C040E4DF015096A10FB11D3FB7F89436
:10DF40002C9127702C939C91942B9C933FBF85839D
:10DF50008D81806C8D83F70184818D7F813021F4E8
:10DF60008D8182608D8303C08D818D7F8D83F701CC
:10DF70008581882321F08D8184608D8303C08D810C
:10DF80008B7F8D83F701408151816281738100E035
:10DF900010E62AEE30E0CE0111DE8C8188608C83A1
:10DFA0008C8180618C8310C08C818F7E8C83F70183
:10DFB00024812250CE0176CF15E180EA98E080CF0F
:10DFC0001DE18ECF15E29ECFDF91CF911F910F9172
:10DFD000FF90EF9008950F93E8ECF4E080818F7D3F
:10DFE000808380818F7D8083ECE7F5E302E00593F9
:10DFF00010927E3510927F3500E2069300E406937E
:10E00000E4E7F5E300E2069300E40693EDE8FEE3BF
:10E010001486158616861786128613861092673523
:10E020000F9108950F9385E080936735EDE7F5E351
:10E0300004E00593E5E7F5E304E005930F91089507
:10E040000F9383E08093673510927E3510927F3571
:10E05000ECE7F5E302E006930F910895E091993E15
:10E06000F0919A3E309709F0199508950F93CF9348
:10E07000DF9380916735833019F4F0DFACDF5EC049
:10E080008091633590916435C091973ED091983ED0
:10E09000C81BD90B71F52091653530916635820F1B
:10E0A000931F80936535909366352091933E309110
:10E0B000943E8217930721F080917E34882341F0AB
:10E0C00084E080936735E4E7F5E302E0069336C029
:10E0D000E0919B3EF0919C3E309799F019958823F2
:10E0E00081F01092633510926435C091973ED091C3
:10E0F000983EC034D10528F010927E34C0E4D0E0C0
:10E1000003C081E080937E34E8E6F5E3C68BD78BCD
:10E1100080916335909164352091953E3091963E83
:10E12000280F391F208F318FC80FD91FC093633537
:10E13000D0936435ECE7F5E302E00693DF91CF91ED
:10E140000F910895FC018181E82FE7708E2F90E0F8
:10E15000FC013197E730F105D8F48827ED55FE4FE3
:10E160008F4F0D94234580E190E0089580E290E088
:10E17000089580E490E0089580E890E0089580E0BC
:10E1800091E0089580E092E008958FEF93E0089584
:10E1900088E090E00895282F2F7030E0220F331F81
:10E1A000082E000C990B8827990F881F9927820F3A
:10E1B000931F02979C01220F331F220F331F220F40
:10E1C000331F820F931F81509B4C08950F93CF9361
:10E1D0008091CC0480FF63C081E08093CC04E4E7AD
:10E1E000F5E300E80693ECE7F5E300E80693809397
:10E1F000CA04E4E7F5E300E10693809167358823DC
:10E2000029F08350823008F429DFE5DE80917635ED
:10E2100090917735089709F044C088E0E3E2F5E390
:10E22000ADE8BEE301900D928A95E1F7E8ECF4E0E9
:10E230008081806280838081806280830E94405FD1
:10E24000C82F811103C0EEDEC1E02CC080918D3E4D
:10E2500088236CF410926535109266351092633500
:10E260001092643582E08093673500DF1BC0809197
:10E27000933E9091943E892B11F4E2DE13C01092EC
:10E28000653510926635109263351092643581E0E1
:10E2900080936735E4E7F5E302E0069303C0C0E04E
:10E2A00001C0C1E08C2FCF910F9108958F929F9262
:10E2B000AF92BF92DF92EF92FF920F931F93CF9393
:10E2C000DF93D82E68DF8C01CD2DCF70D0E0CE014A
:10E2D000880F991FCD2D0D2C000CDD0BCC27DD0FE9
:10E2E000CC1FDD27C80FD91FCE01880F991F880FBB
:10E2F000991F880F991F9C012C583A4C7901C9012C
:10E3000021DF4C01DD200CF07BC0FE01EE0FFF1F72
:10E31000EE0FFF1FEE0FFF1FE859FA4C22893389D9
:10E32000D80115968D919C911697820F931F159683
:10E330008D939C93169713962D913C911497821769
:10E34000930709F447C0281B390B2115B4E03B079C
:10E3500040F02FEF33E0C901B4010F94BE44281BF5
:10E36000390BF801808181FF0AC0C901B4010F9403
:10E37000BE4441E0892B09F040E0842F01C080E0D9
:10E38000D8019C9180FB91F99C93FE01EE0FFF1F39
:10E39000EE0FFF1FEE0FFF1FE859FA4C128A138A87
:10E3A0002687378711962D913C91129715968D915E
:10E3B0009C911697820F931FCC0FDD1FCC0FDD1F92
:10E3C000CC0FDD1FC858DA4C88839983F70102E02F
:10E3D0000693E4C0D8018C9181FFCDC08D7F8C93D2
:10E3E000CC0FDD1FCC0FDD1FCC0FDD1FC859DA4C61
:10E3F0001A8A1B8A1E861F86F70102E00693CEC08A
:10E40000FE01EE0FFF1FEE0FFF1FEE0FFF1FE8597B
:10E41000FA4CA684B784D8018C9182FF1BC0119658
:10E42000ED91FC91129715962D913C9116971396AC
:10E430008D919C911497B4010F94BE44B0E4DB9E7F
:10E44000B0011124615C7B4CAC01CF01820F931FA2
:10E450000F942247F801258136812A0D3B1D258323
:10E460003683838194818217930768F4858396832A
:10E47000CC0FDD1FCC0FDD1FCC0FDD1FC859DA4CD0
:10E480008A899B8978C0FE01EE0FFF1FEE0FFF1FE8
:10E49000EE0FFF1FE859FA4C42895389A416B506BE
:10E4A00009F069C02817390709F465C0AC01421B9F
:10E4B000530B9A01211554E0350748F02FEF33E054
:10E4C000C901B4010F94BE44281B390B06C0C90111
:10E4D000B4010F94BE44281B390BFE01EE0FFF1F41
:10E4E000EE0FFF1FEE0FFF1FE859FA4C1686178636
:10E4F0002815390500F5D8018C9184608C93B0E41F
:10E50000DB9EC0011124815C9B4CFE01EE0FFF1FBE
:10E51000EE0FFF1FEE0FFF1FE858FA4C8083918328
:10E52000CC0FDD1FCC0FDD1FCC0FDD1FC859DA4C1F
:10E530008A8A9B8A1CC0F80141815281858196811B
:10E54000840F951FFE01EE0FFF1FEE0FFF1FEE0F52
:10E55000FF1FE858FA4C80839183CC0FDD1FCC0F4E
:10E56000DD1FCC0FDD1FC859DA4C2A8B3B8BF7011E
:10E5700002E0069313C0D8018C9180FF0FC08E7FFC
:10E580008C931796ED91FC911897309739F015966A
:10E590006D917C9116974D2D80E01995DF91CF916B
:10E5A0001F910F91FF90EF90DF90BF90AF909F90E1
:10E5B0008F900895CF93CFB7F894E1ECF4E0808189
:10E5C0008E7F80831092C00410820F94BC2410921E
:10E5D000A835CFBFCF9108959FB7F89481E080937D
:10E5E000A835EAECF4E080E4808380E28083E1EC0B
:10E5F000F4E0808181608083A9ECB4E08C9182603A
:10E600008C93E8ECF4E08081806480838C9181605D
:10E610008C938081806880839FBF0895CF93DF9320
:10E62000C0E6D0E0188280E30F948424E0ECF4E0AC
:10E6300080818064808381E08883CFB7F894E8E6A6
:10E64000F5E31586158A158E15A215A615AAEFEF06
:10E65000F4E380818E7F8083E8E0F5E380818E7F24
:10E660008083E1E1F5E380818E7F8083EAE1F5E359
:10E6700080818E7F80836AE170E082E00F947E4229
:10E680008F3F19F08093FA0403C08FE18093FA045E
:10E690006BE170E082E00F947E428F3F19F080932F
:10E6A000FB0403C08FE18093FB04E0ECF4E0808185
:10E6B00082608083808180688083808180618083A4
:10E6C00084E795E3868397838081806280838FEFE0
:10E6D0008093C504E8ECF4E080818160808310922F
:10E6E000A8357ADFCFBFDF91CF9108958093C3041F
:10E6F00008958091C3040895EDE8FEE38087918733
:10E70000628773870895282F2F7030E0220F331F00
:10E71000082E000C990B8827990F881F9927820FC4
:10E72000931FFC01EE0FFF1FEE0FFF1FEE0FFF1FE9
:10E73000E859FA4C2585207C09F069C06370613086
:10E7400011F018F404C060EC03C060E801C060E49C
:10E7500040385105E9F050F440325105A9F04034F9
:10E760005105A1F040315105D9F40CC0411522E00A
:10E77000520791F04F3F23E0520781F0411551407D
:10E7800079F408C021E00DC022E00BC023E009C0ED
:10E7900024E007C025E005C026E003C027E001C053
:10E7A00020E0FC01EE0FFF1FEE0FFF1FEE0FFF1F1B
:10E7B000E859FA4C158636E03487262B2587FC016C
:10E7C000EE0FFF1FEE0FFF1FEE0FFF1FE859FA4C71
:10E7D0002585207C203C69F4FC01EE0FFF1FEE0F25
:10E7E000FF1FEE0FFF1FE859FA4C258527702730D1
:10E7F00081F0880F991F880F991F880F991FFC01BE
:10E80000E859FA4C85858062858781E0089580E02B
:10E81000089581E00895E82FEF70F0E0EE0FFF1FFC
:10E82000082E000C990B8827990F881F9927E80F4D
:10E83000F91FEE0FFF1FEE0FFF1FEE0FFF1FE8592E
:10E84000FA4C858582FB882780F90895282F2F7040
:10E8500030E0A901440F551F282F082E000C330B60
:10E860002227330F221F3327240F351FF901EE0F04
:10E87000FF1FEE0FFF1FEE0FFF1FE859FA4C9585A3
:10E8800092FF17C0220F331F220F331F220F331F97
:10E89000F901E859FA4C95859B7F95877CDCFC0152
:10E8A000808180FF06C08E7F80830780F085E02D09
:10E8B000199581E008958F929F92AF92BF92CF9267
:10E8C000DF92EF92FF920F931F93CF93DF93982ED7
:10E8D000862E6A0179015FDC5C01292DC92DCF707C
:10E8E000D0E0CE01880F991FC92D092C000CDD0B3B
:10E8F000CC27DD0FCC1FDD27C80FD91FFE01EE0F7F
:10E90000FF1FEE0FFF1FEE0FFF1FE859FA4C858522
:10E91000807C09F47EC0FE01EE0FFF1FEE0FFF1F8B
:10E92000EE0FFF1FE859FA4C8585807C803C61F032
:10E93000FE01EE0FFF1FEE0FFF1FEE0FFF1FE85946
:10E94000FA4C858582FD67C08FB7F894F5019081F8
:10E9500090FF03C08FBF80E05FC0F50190819160A0
:10E9600090838FBFC182D282E382F48215821682A5
:10E9700007831087811006C091E0E114F10419F0BB
:10E9800090E001C091E0F501808190FB81F98B7FDF
:10E99000808322235CF4CC0FDD1FCC0FDD1FCC0F56
:10E9A000DD1FC859DA4C1A8A1B8A2FC0FE01EE0FF0
:10E9B000FF1FEE0FFF1FEE0FFF1FE859FA4C858572
:10E9C000807C803CB1F4CE01880F991F880F991F7D
:10E9D000880F991F8C589A4CB5DBBC01C7010F9466
:10E9E000BE44892B31F0F50180818E7F808380E0E9
:10E9F00013C0CC0FDD1FCC0FDD1FCC0FDD1FC8599E
:10EA0000DA4C1E861F861A8A1B8A892D4FDC81E00C
:10EA100003C080E001C080E0DF91CF911F910F9192
:10EA2000FF90EF90DF90CF90BF90AF909F908F902E
:10EA30000895FF920F931F93CF93DF93182FC82F42
:10EA4000CF70D0E0CE01880F991FC12F012E000C8E
:10EA5000DD0BCC27DD0FCC1FDD27C80FD91F812F81
:10EA60009ADBDC01FE01EE0FFF1FEE0FFF1FEE0F22
:10EA7000FF1FEC58FA4C02E005938C9180FF22C0F6
:10EA80008E7F8C931796ED91FC9118973097D1F06B
:10EA900011235CF4CC0FDD1FCC0FDD1FCC0FDD1F6D
:10EAA000C859DA4C6A897B890AC0CC0FDD1FCC0FAC
:10EAB000DD1FCC0FDD1FC859DA4C6E857F85412FD5
:10EAC00081E01995DF91CF911F910F91FF900895EB
:10EAD000CF93C82FAEDFEC2FEF70F0E0EE0FFF1FEB
:10EAE0008C2FCC0F990B8827990F881F9927E80F37
:10EAF000F91FEE0FFF1FEE0FFF1FEE0FFF1FE8596C
:10EB0000FA4C1586CF9108950F93E82FEF70F0E03F
:10EB1000EE0FFF1F282F082E000C330B2227330F78
:10EB2000221F3327E20FF31FEE0FFF1FEE0FFF1F11
:10EB3000EE0FFF1FDF01A859BA4C1D969C911D973F
:10EB400094601D969C93EC58FA4C01E0069371DF9B
:10EB500081E00F9108950F931F93CF93DF938B0163
:10EB6000C82FCF70D0E0CC0FDD1F282F082E000C4F
:10EB7000330B2227330F221F3327C20FD31F0BDB88
:10EB8000CC0FDD1FCC0FDD1FCC0FDD1FC859DA4CB9
:10EB90002D8522FF0AC0FC01208120FD0AC02160D2
:10EBA00020830783108781E005C0F801199581E073
:10EBB00001C080E0DF91CF911F910F9108951F92C6
:10EBC0000F920FB60F9211240BB60F920F932F9343
:10EBD0003F934F935F936F937F938F939F93AF93E5
:10EBE000BF93EF93FF938091CB04882344F480E894
:10EBF0008093CA040E94105F0E94465687C080918D
:10EC0000CB0482FF20C084E08093CA0480917C35CD
:10EC100086FF7CC08091CC0481FD78C0D7DA811159
:10EC200075C080916735813011F40ADA6FC0843085
:10EC300009F06CC0EDE7F5E304E00593E5E7F5E3E3
:10EC400004E0059363C08091CB0481FF5AC082E049
:10EC50008093CA048091743586FF58C08091CC049B
:10EC600081FD54C0B3DA811151C080916735823083
:10EC700041F484E080936735E4E7F5E302E006932E
:10EC800045C0833009F042C0EDE7F5E304E00593A9
:10EC9000E5E7F5E304E0059339C080E18093CA0419
:10ECA00081E0C7DE81E8C5DE0E94E55E1092C30404
:10ECB000E8E6F5E3158696E0948783E48587158A70
:10ECC000948B858B83E295E3808B918B84D91EC0D6
:10ECD0008091CB0486FF08C080E48093CA04109220
:10ECE000A8350E94495612C08091CB0485FF0EC002
:10ECF00080E28093CA0481E08093A8350E944A563E
:10ED000005C08091CB0484FFE3CFC7CFFF91EF9183
:10ED1000BF91AF919F918F917F916F915F914F9133
:10ED20003F912F910F910F900BBE0F900FBE0F9040
:10ED30001F9018951F920F920FB60F9211240BB6C9
:10ED40000F920F931F932F933F934F935F936F9364
:10ED50007F938F939F93AF93BF93CF93DF93EF9363
:10ED6000FF938091CC0481FD03C030DA8111C2C0D1
:10ED700082E08093CC048091C5048195880FE4E7FC
:10ED8000F5E3E81BF109208131812457354336959D
:10ED900027953695279536952795822F869520FDC0
:10EDA00002C090E001C090E8890FE82FEF70F0E01A
:10EDB000EE0FFF1F282F082E000C330B2227330FD6
:10EDC000221F3327E20FF31FDF01AA0FBB1FAA0F79
:10EDD000BB1FAA0FBB1FA859BA4C1C969C9195FF4C
:10EDE00089C0EE0FFF1FEE0FFF1FEE0FFF1FEC5845
:10EDF000FA4C00E20693811178C080916735843027
:10EE000019F42CD9E8D876C0009176351091773571
:10EE10008091973E9091983EC0916335D091643532
:10EE200098012C0F3D1F8217930718F48C010C1BBF
:10EE30001D0B8091953E9091963EA80163E275E38B
:10EE40008C0F9D1F0F942247C00FD11FC0936335B5
:10EE5000D09364350034110569F480916535909143
:10EE600066358C0F9D1F2091933E3091943E821702
:10EE7000930780F0EDE8FEE3C287D3870684F78529
:10EE8000E02D309729F01995811102C0CBD832C0FE
:10EE9000D7D830C08091973E9091983EC817D90737
:10EEA000F9F4E0919B3EF0919C3E309711F4BAD872
:10EEB00021C01995811102C0B5D81CC020916535BB
:10EEC000309166358091633590916435820F931F40
:10EED0008093653590936635109263351092643552
:10EEE000E4E7F5E302E0069305C0803811F4BED8EC
:10EEF00001C0DCD9FF91EF91DF91CF91BF91AF912C
:10EF00009F918F917F916F915F914F913F912F9141
:10EF10001F910F910F900BBE0F900FBE0F901F907F
:10EF200018959091800024E0829FB00111246C73A9
:10EF300092709160692B80E890E00F941F42E0E8A6
:10EF4000F0E0828180FDFDCF0895609180006C73B8
:10EF5000636080E890E00F941F42E0E8F0E0828177
:10EF600080FDFDCF0895CF92DF92EF92FF92CF9375
:10EF7000DF93EC016B01E12CF12C60E070E68AEE8E
:10EF800090E0A70196010F94E544CA01B9012FEF63
:10EF90003FEF40E050E00F94E5442115310529F49E
:10EFA00081E08C8321E030E02DC02230310528F44F
:10EFB00082E08C8322E030E025C02430310528F443
:10EFC00083E08C8324E030E01DC02830310528F434
:10EFD00084E08C8328E030E015C02034310528F42B
:10EFE00085E08C8320E430E00DC02F3F310509F02F
:10EFF00028F486E08C8320E031E004C087E08C8335
:10F0000020E034E040E050E060E070E68AEE90E01E
:10F010000F94E544CA01B901A70196010F94E54494
:10F020002D833E832436310518F41C821D821E82F6
:10F03000DF91CF91FF90EF90DF90CF9008950F93E5
:10F040001F93CF93DF93EC018901862F90E08730E7
:10F05000910508F08BC0FC018827E655FE4F8F4FC5
:10F060000D94234580E098E088839983E0E4F6E0FE
:10F07000308181E090E02FEF240F02C0880F991FAC
:10F080002A95E2F7832B808371C080E498E088831F
:10F090009983E0E4F6E0308181E090E023E0240F02
:10F0A00002C0880F991F2A95E2F7832B80835EC0E8
:10F0B00080E099E088839983E0E6F6E0308181E0A2
:10F0C00090E02FEF240F02C0880F991F2A95E2F7D6
:10F0D000832B80834BC080E499E088839983E0E6AA
:10F0E000F6E0308181E090E023E0240F02C0880F39
:10F0F000991F2A95E2F7832B808338C080E09AE03D
:10F1000088839983E0E8F6E0308181E090E02FEF9A
:10F11000240F02C0880F991F2A95E2F7832B808362
:10F1200025C080E49AE088839983E0E8F6E03081A6
:10F1300081E090E023E0240F02C0880F991F2A95F8
:10F14000E2F7832B808312C080E09BE08883998361
:10F15000E0EAF6E0308181E090E02FEF240F02C07A
:10F16000880F991F2A95E2F7832B80834A834230C8
:10F1700061F018F4413031F010C0433049F04430B0
:10F1800051F00BC080E18B8308C080E28B8305C007
:10F1900080E48B8302C080E88B83888199810E9400
:10F1A000746AE881F9818181887F836081831D820F
:10F1B0001E821C82E881F9818081807F8083B80172
:10F1C000CE01D1DEDF91CF911F910F910895CF93A2
:10F1D000DF93EC012D813E81A62FB0E00F942B45EB
:10F1E00024E630E040E050E00F94E5448A81E88175
:10F1F000F981E6FD17C0823061F018F4813031F0FA
:10F200001BC0833049F0843051F016C020AF31AFBD
:10F2100013C022AF33AF10C024AF35AF0DC026AF3F
:10F2200037AF0AC0813019F0823021F005C020AF1D
:10F2300031AF02C022AF33AF8D819E81E881F98169
:10F2400086A397A38B81E881F981E6FD04C09181B3
:10F25000892B818304C091818073892B8183E8810C
:10F26000F9818081807F9C81892B8083DF91CF9180
:10F270000895CF93DF93EC014115510509F443C084
:10F28000AAEFB0E420E030E0922FF901E25CFC4EFE
:10F29000E491ED932F5F3F4F27303105A9F7FA0135
:10F2A000DE01CAEFD0E480818B8381818C83F901F8
:10F2B000E650FF4B8CE28083E2E0E90FF0E0E6509D
:10F2C000FF4B6083C4E0C90F9D5FE92FF0E0E6507B
:10F2D000FF4B8DE78083D0E0FE01E650FF4B1082AC
:10F2E00021E0AE016AEF70E4CD010F9466120E9436
:10F2F0009129811108C021E0AE016AEF70E483E733
:10F3000097E30F946612DF91CF9108954F925F9229
:10F310006F927F928F929F92AF92BF92DF92EF9205
:10F32000FF920F931F93CF93DF931F92CDB7DEB75A
:10F330007C014115510509F466C188E08983AAEF73
:10F34000B0E420E030E0922FF901E25CFC4EE49161
:10F35000ED932F5F3F4F27303105A9F7FA01162FA4
:10F36000AAEFB0E4808113968C9313978181149651
:10F370008C9302E0090FF901E650FF4B8CE2808389
:10F38000623088F5862F0E9410FA8823B1F0812F11
:10F390000E94D5F99F938F931F921F9380E499E267
:10F3A0009F938F93E02FF0E0E650FF4BFF93EF9396
:10F3B0000F945047CDBFDEBF08C1812F0E9468B9AE
:10F3C0009F938F931F921F9380E499E29F938F9353
:10F3D000E02FF0E0E650FF4BFF93EF930F94504780
:10F3E000CDBFDEBFF2C0663109F078C086E10E9471
:10F3F00019F92B013C010E9462F24B015C01672B61
:10F40000682B692BF1F4C301B20120E13EE040E03A
:10F4100050E00F9407455F934F933F932F931F92B4
:10F4200086E18F9387E499E29F938F93E02FF0E03A
:10F43000E650FF4BFF93EF930F945047CDBFDEBFD5
:10F44000C4C0802F0E9403B9992334F5C301B201CF
:10F4500020E13EE040E050E00F940745CA01B901C9
:10F460000F947F17BF92AF929F928F929F938F932B
:10F470007F936F931F9286E18F938FE499E29F931E
:10F480008F93E02FF0E0E650FF4BFF93EF930F9444
:10F490005047CDBFDEBF99C0BF92AF929F928F926F
:10F4A000C301B20120E13EE040E050E00F94074587
:10F4B0005F934F933F932F931F9286E18F938CE539
:10F4C00099E29F938F93E02FF0E0E650FF4BFF937C
:10F4D000EF930F945047CDBFDEBF77C0663071F514
:10F4E000E02FF0E0E650FF4B86E380836894DD2454
:10F4F000D2F8D90E9D5FE92FF0E0E650FF4B8CE289
:10F50000808386E00E9419F98B019C018D2D90E08B
:10F510004BE0BE016F5F7F4F86509F4B0F94D81713
:10F52000E981ED0DAE2FB0E0A650BF4B8DE78C9377
:10F53000EF5FF0E0E650FF4B108247C0653071F599
:10F54000E02FF0E0E650FF4B85E380836894DD24F4
:10F55000D2F8D90E9D5FE92FF0E0E650FF4B8CE228
:10F56000808385E00E9419F98B019C018D2D90E02C
:10F570004BE0BE016F5F7F4F86509F4B0F94241965
:10F58000E981ED0DAE2FB0E0A650BF4B8DE78C9317
:10F59000EF5FF0E0E650FF4B108217C0862F0E940D
:10F5A00019F99F938F937F936F931F921F9387E413
:10F5B00099E29F938F93802F90E086509F4B9F936B
:10F5C0008F930F945047CDBFDEBFEAEFF0E4019078
:10F5D0000020E9F73197EA5FF044E983AF0155274E
:10F5E00021E06AEF70E4C7010F9466120E9491292E
:10F5F000811109C0498150E021E06AEF70E483E79E
:10F6000097E30F9466120F90DF91CF911F910F91A6
:10F61000FF90EF90DF90BF90AF909F908F907F9082
:10F620006F905F904F900895AC016115710571F175
:10F63000E7E4F3E1AAEFB0E422E031E494919D9392
:10F640003196A217B307D1F7FB01CA01AAEFB0E4C4
:10F65000208113962C931397218114962C93149741
:10F6600018961C92189721E048E050E0BD010F94D5
:10F6700066120E949129811109C021E048E050E002
:10F680006AEF70E483E797E30D9466120895EF92B2
:10F69000FF920F931F93CF93DF938C016115710538
:10F6A00009F47FC04115510509F47BC0E5E3F3E19E
:10F6B000AAEFB0E4C2E0D1E494919D933196AC17E7
:10F6C000BD07D1F7FA017B01CAEFD0E480818B83BB
:10F6D00081818C831F922F9388E699E29F938F9369
:10F6E00082E091E49F938F930F94504709900020FC
:10F6F000E9F72197CA5FD044F70181810F900F90FD
:10F700000F900F900F900F90811115C080811F9264
:10F710008F9385E791E29F938F93DD27C650DF4B50
:10F72000DF93CF930F9450470F900F900F900F904F
:10F730000F900F9016C01F928F93F70180811F9238
:10F740008F9382E791E29F938F93DD27C650DF4B23
:10F75000DF93CF930F945047EDB7FEB73896EDBFC8
:10F76000FEBFEAEFF0E401900020E9F73197EA5F8D
:10F77000F044EF01DD2721E0AE016AEF70E4C8013B
:10F780000F9466120E94912981110BC003571743F1
:10F7900041F021E0AE016AEF70E483E797E30F9454
:10F7A0006612DF91CF911F910F91FF90EF90089516
:10F7B000CF93DF93EC014115510509F43FC0662357
:10F7C00061F0E7E4F3E1AAEFB0E490E024912D9337
:10F7D0009F5F31969730D1F70BC0EEE3F3E1AAEFCC
:10F7E000B0E490E024912D939F5F31969730D1F74C
:10F7F000DA01CE01EAEFF0E42C91238311962C91EB
:10F8000024832CE227833CE43087218720E322876E
:10F810002DE72387148621E04CE050E0BF010F94D0
:10F8200066120E949129811109C021E04CE050E04C
:10F830006AEF70E483E797E30F946612DF91CF914C
:10F840000895EF92FF920F931F93CF93DF9300D011
:10F850001F92CDB7DEB70097C9F166307105C0F1D0
:10F86000FC0120812035B1F521812C32A9F52481BC
:10F870002C32A1F57A018C010B5F1F4FAB01455073
:10F8800051099E012F5F3F4FB8018CE20F94AF17D3
:10F89000882349F149815A814B5F5F4F49835A83DD
:10F8A00046305105E8F045509E012D5F3F4F60E026
:10F8B000C8010F9437168823B1F08B819C818C315D
:10F8C000910580F4F701808381E00DC080E00BC0DA
:10F8D00080E009C080E007C080E005C080E003C090
:10F8E00080E001C080E02496CDBFDEBFDF91CF91E4
:10F8F0001F910F91FF90EF900895CF92DF92EF92BA
:10F90000FF920F931F93CF93DF93CDB7DEB72C9762
:10F91000CDBFDEBF009709F423C16630710508F43E
:10F9200021C1FC012081203509F01EC121812C322A
:10F9300009F01CC124812C3209F01AC17B018C0111
:10F940006C01F5E0CF0ED11CAB01455051099E0171
:10F950002F5F3F4FB6018CE20F94AF17982F88238B
:10F9600009F415C149815A814B5F5F4F49835A831E
:10F970004630510508F4FEC045509E012D5F3F4FB3
:10F9800060E0C6010F943716982F882309F4FFC052
:10F990002B813C812C31310508F0EEC049815A8120
:10F9A000DA011196AE15BF0508F0E8C02C3131051B
:10F9B00008F0E6C0F9018827EF54FE4F8F4F0D94F1
:10F9C0002345C8018A0F9B1FFC0160816D3241F401
:10F9D000FA013296EE15FF0508F0D4C040E002C0EF
:10F9E000FD0141E02631310559F46E2D6E1B9E015B
:10F9F000275F3F4FC8018E0F9F1F0E9472E912C000
:10FA00002630310541F46E2D6A1BAE01475F5F4F12
:10FA10000E943FEC07C06E2D6A1BAE01475F5F4F2F
:10FA20000E945BED882309F4AFC049855A856B8538
:10FA30007C858B810E945BBA982F882309F4A7C02C
:10FA400049855A856B857C858B810E942CF991E0D4
:10FA50009EC04E2D4A1B9E012B5F3F4F60E0C801A8
:10FA60008A0F9B1F0F94C216982F882309F48FC00A
:10FA70004D815E816F81788549875A876B877C8746
:10FA80008B810E945BBA982F882309F480C08985F6
:10FA90009A85AB85BC850B97A105B10541F480EC37
:10FAA0009AE30E940C2E982F882309F470C0498590
:10FAB0005A856B857C858B810E942CF991E067C00B
:10FAC0004E2D4A1B9E012B5F3F4F60E0C8018A0FFD
:10FAD0009B1F0F94C216982F882309F458C04D819C
:10FAE0005E816F81788549875A876B877C878B8198
:10FAF0000E945BBA982F882349F049855A856B8507
:10FB00007C858B810E942CF991E041C02B813C8146
:10FB1000A9014C50510946305105C8F549855A850F
:10FB20006B857C85452B462B472B89F540E050E0C3
:10FB3000BA01822F0E942CF991E029C0C7018A1BCB
:10FB40009B0B899718F56E2D6A1B422FC8018A0FEF
:10FB50009B1F0E9497F991E0811119C090E017C096
:10FB600090E015C090E013C090E011C090E00FC08D
:10FB700090E00DC090E00BC090E009C090E007C09D
:10FB800090E005C090E003C090E001C090E0892FB4
:10FB90002C96CDBFDEBFDF91CF911F910F91FF90CB
:10FBA000EF90DF90CF9008950F931F93CF93DF9343
:10FBB0001F921F92CDB7DEB7009741F166307105F5
:10FBC00038F1FC012081203529F521812C3221F5E5
:10FBD00024812C3219F58C01AB0145505109BC012F
:10FBE0006B5F7F4F9E012F5F3F4F8CE20F94AF17EB
:10FBF0008823B9F089819A810596069788F081E07B
:10FC0000F8019581963469F080E00BC080E009C06E
:10FC100080E007C080E005C080E003C080E001C054
:10FC200080E00F900F90DF91CF911F910F91089579
:10FC3000EF92FF920F931F93CF93DF9300D000D0EA
:10FC4000CDB7DEB7009709F453C06630710508F4EC
:10FC500051C0FC012081203509F04EC021812C3299
:10FC600009F04CC024812C3209F04AC07B018C0180
:10FC7000AB0145505109BC016B5F7F4F9E012F5F67
:10FC80003F4F8CE20F94AF17882309F442C089815B
:10FC90009A819C012B5F3F4F29833A83263031059F
:10FCA00088F1F8012581263479F506968E159F0591
:10FCB00068F54E2D481B9E012D5F3F4F60E0800F81
:10FCC000911F0F94C216882321F16B817C818D8155
:10FCD0009E818B019C010150110921093109073EC8
:10FCE000134021053105A0F40E94ECB981E011C058
:10FCF00080E00FC080E00DC080E00BC080E009C054
:10FD000080E007C080E005C080E003C080E001C063
:10FD100080E02696CDBFDEBFDF91CF911F910F917E
:10FD2000FF90EF9008950F931F93CF93DF93EC0113
:10FD30006115710509F444C0AAEFB0E420E030E099
:10FD4000922FF901E25CFC4EE491ED932F5F3F4F5F
:10FD500027303105A9F7FB01AAEFB0E480811396A3
:10FD60008C931397818114968C931497F901E65024
:10FD7000FF4B8CE280839E5FE92FF0E0E650FF4B63
:10FD800086E49DE7808391831282FD01019000202B
:10FD9000E9F73197EA5FF0448F01112721E0A801CC
:10FDA000BD01CE010F9466120E949129811108C0F5
:10FDB00021E0A8016AEF70E483E797E30F946612ED
:10FDC000DF91CF911F910F910895FC01892B61F074
:10FDD0006530710558F08081803551F481E0918162
:10FDE0009C3239F080E0089580E0089580E0089525
:10FDF00080E00895009799F06330710590F0FC0160
:10FE00002081203581F421812C3279F424812C3217
:10FE100071F485818354823060F080E0089580E041
:10FE2000089580E0089580E0089580E0089580E0DE
:10FE3000089581E00895009791F06330710588F08E
:10FE4000FC012081203579F421812C3271F4248148
:10FE50002C3269F485818F3461F080E0089580E070
:10FE6000089580E0089580E0089580E0089580E09E
:10FE7000089581E00895009791F06330710588F04E
:10FE8000FC012081203579F421812C3271F4248108
:10FE90002C3269F48581873561F080E0089580E037
:10FEA000089580E0089580E0089580E0089580E05E
:10FEB000089581E00895CF92DF92EF92FF920F9321
:10FEC0001F93CF93DF934115510509F4AFC00097FD
:10FED00009F4AEC06630710508F4ACC0FC012081A5
:10FEE000203509F0A9C021812C3209F0A7C0248156
:10FEF0002C3209F0A5C08581873509F0A3C0EA013D
:10FF000080EC9AE30E949413883009F49DC080EC41
:10FF10009AE30E949413863009F498C00F94730AF0
:10FF20000E941B5161E086EC9AE30E948F530E946D
:10FF300054FA0E946A1C813079F582E00E9411B95E
:10FF40006B017C01DD24EE24FF24B701A60182E0D1
:10FF50000E942CF9B701A60182E00E94F9B80E9424
:10FF60009129811119C084E1ECE6F9E2A5E5B2E43A
:10FF700001900D928A95E1F7E5E5F2E40190002009
:10FF8000E9F73197AF014555524420E065E572E449
:10FF900083E797E30F946612CE010E94B91B80E0BD
:10FFA0000E94DFB89B01AC016894EE24E2F806EBF6
:10FFB00012E2BE01685E7F4FCE0106960E94E954B0
:10FFC0008D8340E050E0BA01CE010E94BC2D8D81AE
:10FFD000882351F182E00E9403B9062F8BE00E9432
:10FFE00003B921E0611120E044E65EE3BE016D5CEF
:10FFF0007F4FCE01C5960E94ED4DCE010E948F1B12
:020000021000EC
:100000009E01275A3D4FAE01485A5D4FBE016D5AC1
:100010007D4FCE018E5A9D4F0E94432C0E94B332D9
:1000200068E0CE010E9481138D8111C080E00FC075
:1000300080E00DC080E00BC080E009C080E007C018
:1000400080E005C080E003C080E001C080E0DF9177
:10005000CF911F910F91FF90EF90DF90CF90089577
:10006000CF92DF92EF92FF920F93CF93DF934115E0
:10007000510509F4B0C0009709F4AFC066307105AE
:1000800008F4ADC0FC012081203509F0AAC021810F
:100090002C3209F0A8C024812C3209F0A6C0EA0154
:1000A0008581833409F493C0843409F0A0C00E9490
:1000B000A1B90E94F2F980EC9AE30E94941388306F
:1000C00009F497C080EC9AE30E949413863009F4F7
:1000D00092C00F94730A0E941B5161E086EC9AE370
:1000E0000E948F530E9454FA0E946A1C813079F555
:1000F00082E00E9411B96B017C01DD24EE24FF2413
:10010000B701A60182E00E942CF9B701A60182E0A6
:100110000E94F9B80E949129811119C084E1ECE68E
:10012000F9E2A5E5B2E401900D928A95E1F7E5E5E3
:10013000F2E401900020E9F73197AF0145555244B0
:1001400020E065E572E483E797E30F94661280E0B0
:100150000E94DFB89B01AC01BE01685E7F4FCE01FB
:1001600006960E9423518D8340E050E0BA01CE01F3
:100170000E94BC2D8D81882341F182E00E9403B949
:10018000062F8BE00E9403B921E0611120E044E6D4
:100190005EE3BE016D5C7F4FCE01C5960E94ED4DC2
:1001A000CE010E948F1B9E01275A3D4FAE01485A37
:1001B0005D4FBE016D5A7D4FCE018E5A9D4F0E94FC
:1001C000432C68E0CE010E9481138D8115C00E94EE
:1001D000F2F981E011C080E00FC080E00DC080E046
:1001E0000BC080E009C080E007C080E005C080E06F
:1001F00003C080E001C080E0DF91CF910F91FF90BC
:10020000EF90DF90CF900895BF92CF92DF92EF9260
:10021000FF920F931F93CF93DF931F92CDB7DEB75B
:100220006115710509F464C0DB017C01EAEFF0E4BB
:100230008BE7808380E781838CE282839C91938328
:1002400011969C91948385839FE49683878380E0B5
:100250000E9425C08B019C0148E0BE016F5F7F4F6B
:1002600082E091E40F948619E981E85FD12C0F2E8A
:10027000FCE2BF2EF02DCC24C394CE0EF0E0E6506D
:10028000FF4BB082D3948D2D0E9425C08B019C0121
:100290008C2D90E048E0BE016F5F7F4F86509F4BF2
:1002A0000F948619E981EC0D83E0D812E4CF81E048
:1002B0008E0FF0E0E650FF4B9DE79083482F50E013
:1002C000FA01E650FF4B1082898321E06AEF70E467
:1002D000C7010F9466120E949129811109C04981BA
:1002E00050E021E06AEF70E483E797E30F94661231
:1002F0000F90DF91CF911F910F91FF90EF90DF90C2
:10030000CF90BF900895CF93DF9341155105A9F188
:100310000097A9F165307105A0F1FC01208120351D
:1003200091F521812C3289F52281263481F5EA016B
:1003300084818235E9F0833531F0843451F50E94AF
:10034000CBB981E027C00F94730ABE016D5C7F4F6B
:10035000CE01C5960E94F24B80EC9AE30E942222C5
:1003600081110F94950ACE010E942B298D8112C014
:10037000CA01C5960E94BCF10DC080E00BC080E0B0
:1003800009C080E007C080E005C080E003C080E0D5
:1003900001C080E0DF91CF910895FC01892B79F0B5
:1003A0006630710570F08081833569F481818C320B
:1003B00061F481E094819C3249F080E0089580E00E
:1003C000089580E0089580E0089580E008950F93F7
:1003D000CF93DF93009709F476C06630710508F477
:1003E00074C0FC016081633509F071C061816C32B9
:1003F00009F06FC064816C3209F06DC04115510580
:1004000009F46BC02115310509F469C08581813378
:1004100009F067C0B901EA01F9011082CA010E941E
:100420000920882309F45FC0CE010E94EA1F8111D0
:100430002BC0CE010E942B2961E0CE010E945A26DA
:1004400064E0CE010E94811361E0CE010E94DB1FB7
:1004500019820E946C9DE6E3F1E4808190E0DC016A
:10046000AA5CBE4B25853685880F991FFC01EA5C86
:10047000FE4B418152811F960C9161E080EC9AE322
:100480000E94892481E032C00E94912981112DC0EF
:1004900083E1E0E8F9E2AAEFB0E401900D928A95D9
:1004A000E1F7EAEFF0E401900020E9F73197AF01BE
:1004B0004A5F504421E06AEF70E483E797E30F94CA
:1004C000661281E013C080E011C080E00FC080E0C0
:1004D0000DC080E00BC080E009C080E007C080E074
:1004E00005C080E003C081E001C081E0DF91CF91D1
:1004F0000F9108950F93CF93DF93009709F45EC196
:100500006630710508F45CC1DC012C91233509F0DB
:1005100059C111962C9111972C3209F055C114969E
:100520002C9114972C3209F051C14115510509F451
:100530004FC11596EC918E2F90E0FC01F097E534B9
:10054000F10508F047C1EA018827E353FE4F8F4FBA
:100550000D942345CA010E949413843031F0CE01DA
:100560000E949413893009F037C1CE010E94671FA1
:10057000CE010E94EBFCCE010E942B290F94730A3E
:1005800060E080EC9AE30E945A2663E0CE010E946C
:10059000811319820E94599DE6E3F1E4808190E085
:1005A000DC01AA5CBE4B25853685880F991FFC01AE
:1005B000EA5CFE4B418152811F960C9161E080EC18
:1005C0009AE30E94892491E016C1CA010E94EA1FA1
:1005D000882309F403C181E0898360E0CE010E9491
:1005E0007D1460E0CE010E946B140E94912981115C
:1005F000F7C080E1E3E9F9E2AAEFB0E401900D92DF
:100600008A95E1F7EAEFF0E401900020E9F73197ED
:10061000AF014A5F504421E06AEF70E483E797E35B
:100620000F94661291E0E7C0CA010E94EA1F882376
:1006300009F4D8C060E0CE010E947D1460E0CE01D4
:100640000E946B14FE01EE5AFD4FDE01A85ABD4F09
:100650008C918083319611968C91808319820E94AF
:1006600091298111C1C080E1E3EAF9E2AAEFB0E487
:1006700001900D928A95E1F7EAEFF0E401900020F5
:10068000E9F73197AF014A5F504421E06AEF70E427
:1006900083E797E30F94661291E0ADC0CA010E9410
:1006A000EA1F982F882309F4A6C0CE010E94F726DE
:1006B00091E08111A0C090E09EC0CA010E94EA1F93
:1006C000882329F0CE010E948126982F94C00E9491
:1006D00077C091E090C0CA010E94EA1F982F88233A
:1006E00009F489C00F94730A60E080EC9AE30E94D9
:1006F0005A2669E0CE010E9481131982CE010E9420
:10070000FBFCCE010E94231CCE010F9495010F9497
:10071000770D61E0CE010E94DB1F91E06CC0CA0141
:100720000E949413893009F061C064E67EE3CE0133
:100730000F943201CE010E94F2FC8D3009F058C0B6
:10074000CE010E94FBFCCE010F9495010F94770D12
:1007500091E051C0CA010E949413893009F04AC047
:10076000CE010E94EBFCCE010E942B2961E0CE015C
:100770000E945A2664E0CE010E94811361E0CE01FE
:100780000E94DB1F19820E946C9DE6E3F1E48081E8
:1007900090E0DC01AA5CBE4B25853685880F991F49
:1007A000FC01EA5CFE4B418152811F960C9161E095
:1007B00080EC9AE30E94892491E01DC090E01BC068
:1007C00090E019C090E017C090E015C090E013C011
:1007D00090E011C090E00FC091E00DC091E00BC01F
:1007E00091E009C091E007C091E005C090E003C02E
:1007F00091E001C090E0892FDF91CF910F91089592
:10080000FC01892B61F06630710558F080818D34D0
:1008100051F481E091819C3239F080E0089580E0CC
:10082000089580E0089580E00895FC01892B61F02F
:100830006630710558F08081823551F481E09181F4
:100840009C3239F080E0089580E0089580E00895BA
:1008500080E00895FC01892B61F06530710558F046
:1008600080818A3551F481E091819C3239F080E0B9
:10087000089580E0089580E0089580E00895CF9283
:10088000DF92EF92FF920F931F93CF93DF93CDB739
:10089000DEB72897CDBFDEBF009709F457C065309B
:1008A000710508F455C0FC0120812A3509F052C0B9
:1008B00021812C3209F050C07B018C016C01F2E0E7
:1008C000CF0ED11CAB01425051099E012F5F3F4F0B
:1008D000B6018CE20F94AF17882309F446C0498112
:1008E0005A814E5F5F4F49835A8343305105B0F1BF
:1008F00042509E012D5F3F4F60E0C6010F943716B6
:10090000882399F18B819C81039750F589819A8185
:1009100001968E159F0530F54E2D481B9E012B5FCD
:100920003F4F60E0800F911F0F94C2168823E9F0BB
:100930006D817E818F819885623071058105910579
:1009400098F48B810E94AFD481E00FC080E00DC08D
:1009500080E00BC080E009C080E007C080E005C0F7
:1009600080E003C080E001C080E02896CDBFDEBFFC
:10097000DF91CF911F910F91FF90EF90DF90CF907B
:1009800008952F923F924F925F926F927F928F9233
:100990009F92AF92BF92CF92DF92EF92FF920F930E
:1009A0001F93CF93DF93CDB7DEB76397CDBFDEBF85
:1009B0008C01F62E81E08D830115110509F423C306
:1009C0008093CE2089E10E9403B9672B682B692BA5
:1009D00009F025C30E94F1F4B82E811103C0F11073
:1009E00020C385C380EC9AE30E945C20B82E882344
:1009F00009F47DC380EC9AE30E9494138F87F11071
:100A000004C08150823008F400C32F85243031F4B3
:100A100080EC9AE30E946F2933E03F870E94F5FA49
:100A20000E94DEFA80EC9AE30E94222281110F9448
:100A3000950A80EC9AE30E942B2982E00E9403B978
:100A4000E62E8FEF8E0D8A3008F0E1C2AE014A5FCC
:100A50005F4FBE016B5F7F4F8E2D0E9497218E816D
:100A60000E941AD48E8184700E948ED48D810E943F
:100A70000FF70F2EFAEFCF2EF0E4DF2EF02D8BE7DD
:100A8000D6018C938DE611968C9311978CE2129679
:100A90008C93129787E713968C9320E044E050E004
:100AA000B601C8010F9466121F92EF9283EB99E290
:100AB0009F938F93DF92CF920F945047F60101904E
:100AC0000020E9F73197AF014A5F504420E0B601BA
:100AD000C8010F946612E8EAF1E587858F93868551
:100AE0008F9385858F9384858F930F2EF7EBAF2E91
:100AF000F9E2BF2EF02DBF92AF92DF92CF920F940A
:100B00005047F60101900020E9F73197AF014A5FA5
:100B1000504420E0B601C8010F9466128AE00E949A
:100B200003B99F938F937F936F93BF92AF92DF929E
:100B3000CF920F945047F60101900020E9F73197CA
:100B4000AF014A5F504420E0B601C8010F9466121D
:100B50008BE00E9403B99F938F937F936F93BF9213
:100B6000AF92DF92CF920F945047F6010190002090
:100B7000E9F73197AF014A5F504420E0B601C80160
:100B80000F9466120F2EF2ECCF2EF1E5DF2EF02D32
:100B9000CDBFDEBF412C512C320145010F2EFAEFA3
:100BA000AF2EF0E4BF2EF02D2BC0D6018C91119604
:100BB0009C91119712962C91129713963C91B4E048
:100BC000CB0ED11C3F932F939F938F939F928F9225
:100BD000BF92AF920F945047F50101900020E9F7C2
:100BE0003197AF014A5F504420E0B501C8010F942E
:100BF0006612EFEF4E1A5E0A6E0A7E0ACDBFDEBFA6
:100C00000F94740D90E0A0E0B0E0481659066A0613
:100C10007B0658F28DE78093FA4021E041E050E0F6
:100C20006AEF70E4C8010F94661265E080EC9AE305
:100C30000E9481130F94730A80EC9AE30E9474243B
:100C40000E94C85660E072E080E090E00E94BA57CF
:100C500010929D3E10929E3E8BE491E40E94D6A29B
:100C60000E945B598111FCCFB82EF11004C00E9484
:100C70004F1F8823E1F389E00E9403B96F317105AA
:100C80008105910508F59B01AC01012E1CE0220FA6
:100C9000331F441F551F1A95D1F7102D2B873C8702
:100CA0004D875E87CA01B9010E9497FA0F943D0BE8
:100CB00081E00F948D0D80E090E1A0E0B0E08F83A3
:100CC0009887A987BA873FC09B01AC01012E19E024
:100CD000220F331F441F551F1A95D1F7102D2B8754
:100CE0003C874D875E87CA01B9010E9497FA0F942D
:100CF0003D0B0F94BD0D80E092E0A0E0B0E08F834B
:100D00009887A987BA871FC0412C512C32019F2C8C
:100D1000CB84DC84ED84FE840F94FA0D8823E1F00B
:100D20008D810F9467096BE471E40E9439A3A82EAA
:100D30000F94E90D9FEF491A590A690A790AA1101F
:100D40000BC0F92C0FC02B853C854D855E85232B70
:100D5000242B252BC9F606C04C145D046E047F04B9
:100D6000D8F2F92C0F94E40D8BE491E40E949DA33A
:100D7000E82E0E9447580F94A007EE2031F06F85AF
:100D800080EC9AE30E948113B2C184E793E40E944D
:100D9000A6C5882351F0F11008C06091734470E03B
:100DA00084E793E40E94FDA309C0EAEFF0E4108217
:100DB000118262E070E0CF010E94FDA360E072E06A
:100DC00080E090E00E94D0560E945B598111FCCFD8
:100DD0008B859C85AD85BE85892B8A2B8B2B09F451
:100DE000F3C0C12CD12C76010F2EFAEF2F2EF0E498
:100DF0003F2EF02D4F80588469847A8491E0491AFF
:100E00005108610871080E94ECA380939D3E909365
:100E10009E3EAE014F5F5F4FBC018D810E948F14DB
:100E2000882309F463C1C701B6012F81388549853C
:100E30005A850F94E5444B015C01672B682B692BA5
:100E4000A1F5C701B6012F81388549855A850F94D0
:100E5000E544288B398B4A8B5B8B89E00E9403B970
:100E6000AB89AF93BA89BF93E989EF93F889FF9370
:100E70009F938F937F936F932CEB39E23F932F9344
:100E80003F922F920F945047F10101900020E9F713
:100E90003197AF014A5F504420E0B101C8010F947F
:100EA00066121092CE20CDBFDEBF2F8138854985D6
:100EB0005A85211582E038074105510509F4BAC069
:100EC000211530414105510509F4DDC0D701C601A6
:100ED00087709927AA27BB27892B8A2B8B2B09F090
:100EE00043C08C818F938B818F938A818F9389816B
:100EF0008F93A4E0BAE2BF93AF933F922F920F94E7
:100F00005047F10101900020E9F73197AF014A5FA6
:100F1000504420E0B101C8010F946612C701B60128
:100F20002F81388549855A850F94E5442F5F3F4FBF
:100F30004F4F5F4F6F81788589859A850F94A344C1
:100F4000CDBFDEBFA7019601285F3F4F4F4F5F4FD8
:100F5000621773078407950719F41092CE20C0C05A
:100F600031E03093CE20BCC01092CE208414950482
:100F7000A604B70479F4EDE7D101EC9321E041E058
:100F800050E0B101C8010F9466120FC0ECE2D1012C
:100F9000EC9304C08091CE20882339F020E041E01A
:100FA00050E0B101C8010F946612FFEFCF1ADF0ABB
:100FB000EF0AFF0A2B853C854D855E85C216D30658
:100FC000E406F50609F01FCF0E949B570F94A00777
:100FD0000F942F1B84E69EE30F94F53C6F8580EC05
:100FE0009AE30E9481130E946CFB80EC9AE30E94BA
:100FF000222281110F94950A80EC9AE30E942B29FA
:10100000BB24B39474C0B12C72C0B12C70C0B12C8D
:101010006EC080EC9AE30E9494138F87F6CCFF2475
:10102000F39480EC9AE30E945C20B82E882309F4A4
:101030005EC0EFCF8C818F938B818F938A818F934A
:1010400089818F9344E05AE25F934F933F922F92AE
:101050000F945047F10101900020E9F73197AF015B
:101060004A5F504420E0B101C8010F94661291E03C
:101070009093CE20CDBFDEBF481459046A047B0490
:1010800009F084CF78CF8C818F938B818F938A8165
:101090008F9389818F93E4E0FAE2FF93EF933F927D
:1010A0002F920F945047F10101900020E9F73197FA
:1010B000AF014A5F504420E0B101C8010F946612AD
:1010C00031E03093CE20CDBFDEBF481459046A040E
:1010D0007B0409F05BCF4FCFECE2D101EC935ACF08
:1010E00084149504A604B704B9F745CFB82E8B2D08
:1010F0006396CDBFDEBFDF91CF911F910F91FF901F
:10110000EF90DF90CF90BF90AF909F908F907F90A7
:101110006F905F904F903F902F900895CF92DF9205
:10112000EF92FF921F93CF93DF936115710509F43E
:1011300074C04630510508F472C0DB01EC91ED3407
:1011400009F06FC01196EC91EC3209F06CC02115DA
:10115000310509F46AC0009709F469C069017A0190
:10116000EB012D81203341F440E060E00ADC11E026
:10117000811160C010E05EC0233541F5C6010E94B8
:101180006920182F882309F455C0C70106970297D4
:1011900018F40E94BEA40CC08E818C3219F00E94FB
:1011A000BEA406C069EF6E0DCE0107960E9489A409
:1011B000A601485E5F4FB6016B5C7F4F80E00E94E6
:1011C000854711E0811136C010E034C00E9491299A
:1011D000182F81112EC08D811F928F9388EC99E278
:1011E0009F938F93CAEFD0E4DF93CF930F94504730
:1011F00009900020E9F72197AE014A5F504421E0B1
:101200006AEF70E483E797E30F9466120F900F90F4
:101210000F900F900F900F900DC010E00BC010E0DA
:1012200009C010E007C010E005C010E003C010E0E6
:1012300001C010E0812FDF91CF911F91FF90EF90BF
:10124000DF90CF900895FC01892BA9F068307105DB
:10125000A0F08081813599F481818C3291F4848170
:101260008C3289F486818C3281F481E095819033CF
:1012700069F080E0089580E0089580E0089580E0BE
:10128000089580E0089580E0089580E00895EF9249
:10129000FF920F931F93CF93DF9300D0CDB7DEB7AC
:1012A0009CE29B8321153105A9F161157105A1F11E
:1012B000FA013197F39790F5823390F5803391F5E9
:1012C000C9017A018B010E949413843069F59E0153
:1012D0002F5F3F4F41E050E0BE016D5F7F4F84E6DE
:1012E0009EE30F94473B9E012F5F3F4FA701B8013C
:1012F00084E69EE30F94473B84E69EE30F94F53C1F
:101300000F942C0D8FE99EE30E94869C0F94020C93
:1013100081E00BC080E009C080E007C080E005C02C
:1013200080E003C081E001C080E02396CDBFDEBF36
:10133000DF91CF911F910F91FF90EF900895FC01E5
:10134000892B61F06330710558F080818C3451F441
:1013500081E091819C3239F080E0089580E0089529
:1013600080E0089580E00895452BB1F00097B1F03A
:10137000672BB1F0FC0185818136A1F484EE9FE3F7
:101380000E94B99C811110C060E070E084EE9FE380
:101390000E94C49C81E0089580E0089580E0089553
:1013A00080E0089580E0089580E00895CF93DF9372
:1013B000452B41F1009741F16531710538F1FC0190
:1013C0002581203729F52781203319F41092F23F27
:1013D00009C0213321F421E02093F23F03C022E031
:1013E0002093F23FEC0184EE9FE30E94B99C8111AF
:1013F00011C0BE01675F7F4F84EE9FE30E94C49CD3
:1014000081E009C080E007C080E005C080E003C043
:1014100080E001C080E0DF91CF910895CF93DF930A
:10142000452B61F1009761F16531710558F1FC01BF
:1014300025812E3649F52781203319F41092F23F89
:1014400009C0213321F421E02093F23F03C022E0C0
:101450002093F23FEC0184EE9FE30E94B99C81113E
:1014600015C08091F23F882399F0BE01675F7F4FDE
:1014700084EE9FE30E94E59C81E00BC080E009C000
:1014800080E007C080E005C080E003C080E001C0CC
:1014900081E0DF91CF910895009799F06630710552
:1014A00090F0FC018581833681F484EE9FE30E94F5
:1014B000B99C882361F00E945B9B1092E43F81E01D
:1014C000089580E0089580E0089580E0089581E027
:1014D0000895FC01892B49F06630710540F081E0E8
:1014E0009581933729F080E0089580E0089580E0A9
:1014F0000895FC01892B49F06630710540F081E0C8
:101500009581953629F080E0089580E0089580E087
:101510000895BF92CF92DF92EF92FF920F931F93A5
:10152000CF93DF9300D0CDB7DEB79CE29B838823B7
:1015300059F00091D23F002311F010E009C0009152
:101540009F3E1091A03E04C00091D33F1091D43F24
:101550000D3291E0190710F00CE211E001151105B0
:1015600009F44CC0B82E9E012F5F3F4F41E050E080
:10157000BE016D5F7F4F84E69EE30F94473B109260
:10158000A13E1092A23E20E030E0C12CD12C0F2EC3
:10159000FFE9EF2EFEE3FF2EF02DF901E156F14CAD
:1015A00095819B839E012F5F3F4F41E050E0BE013C
:1015B0006D5F7F4F84E69EE30F94473B29813A811C
:1015C000232B19F4EFEFCE1ADE0AF70122813381C3
:1015D0002F5F3F4F2283338320173107F0F284E6D9
:1015E0009EE30F94F53CB11004C01092D33F1092CB
:1015F000D43F81E0CD2819F080E001C080E023963F
:10160000CDBFDEBFDF91CF911F910F91FF90EF9083
:10161000DF90CF90BF900895FC01892B49F0663090
:10162000710540F081E09581943629F080E00895BD
:1016300080E0089580E00895EAEFF0E42BE720834E
:101640002CE621832CE22283662321F02FE62093CF
:10165000FD4003C025E62093FD40EAEFF0E42DE7CE
:101660002483158221E045E050E0BF010F9466120B
:101670000E949129811109C021E045E050E06AEF04
:1016800070E483E797E30D9466120895EF92FF925A
:101690000F931F93CF93DF936115710509F410C267
:1016A000009709F40DC2FB012081222309F408C22E
:1016B000EB018C010E949129811125C088811F9224
:1016C0008F938DEC99E29F938F930F2EF5E5EF2E7C
:1016D000F2E4FF2EF02DFF92EF920F945047F701A6
:1016E00001900020E9F73197AF014555524421E0C0
:1016F000B70183E797E30F9466120F900F900F9056
:101700000F900F900F90888190E08A30910508F03B
:10171000D1C1FC018827EE5EFD4F8F4F0D9423450C
:101720008DE19DE30E94179B0F943D0B08EF10E4A1
:101730001EC066E770E48DE19DE30F941212F8017C
:1017400080818130A1F40E94912981110BC04091C8
:1017500076405091774021E068E770E483E797E3B3
:101760000F94661286E790E40F94031207C00F945B
:10177000540B6838734181059105D8F289819FEF38
:10178000980F983020F088818F5F888399C1888373
:1017900097C1EAEFF0E483E580838DE481838CE2F6
:1017A00082838E85823021F481E38093FD4003C0E3
:1017B00080E38093FD401092FE4021E044E050E041
:1017C0006AEF70E48DE19DE30F94661288818F5F6C
:1017D00088830F943D0BC8EFD0E41DC066E770E42A
:1017E0008DE19DE30F94121288818130A1F40E9453
:1017F000912981110BC0409176405091774021E0B2
:1018000068E770E483E797E30F94661286E790E455
:101810000F94031255C10F94540B62337105810567
:101820009105E0F24DC1EAEFF0E483E5808380E5C5
:1018300081838CE282838E8581110CC081E3838356
:1018400082E3848383E3858384E3868388818F5F57
:1018500088831AC0813059F4EAEFF0E480E383838F
:1018600084838583868388818F5F88830DC0EAEFB8
:10187000F0E481E3838382E3848383E3858384E3E9
:10188000868388818F5F88831092014121E047E041
:1018900050E06AEF70E48DE19DE30F9466120F94BF
:1018A0003D0BC8EFD0E41DC066E770E48DE19DE319
:1018B0000F94121288818130A1F40E949129811124
:1018C0000BC0409176405091774021E068E770E48A
:1018D00083E797E30F94661286E790E40F94031270
:1018E000EFC00F94540B6233710581059105E0F24E
:1018F000E7C0EAEFF0E483E5808382E581838CE250
:101900008283DE011296EDEFF0E429E031E48D915F
:101910008193E217F307D9F71092094121E04FE0D4
:1019200050E06AEF70E48DE19DE30F9466128881C8
:101930008F5F88830F943D0BC8EFD0E41DC066E72E
:1019400070E48DE19DE30F94121288818130A1F43F
:101950000E94912981110BC04091764050917740AF
:1019600021E068E770E483E797E30F94661286E767
:1019700090E40F940312A4C00F94540B62337105CA
:1019800081059105E0F29CC0EAEFF0E482E58083F6
:101990008CE2818381E38283138221E043E050E083
:1019A000BF018DE19DE30F94661288818F5F88836C
:1019B00087C08DE19DE30E94179B0F943D0B08EFBC
:1019C00010E41EC066E770E48DE19DE30F941212EF
:1019D000F80180818130A1F40E94912981110BC00E
:1019E000409176405091774021E068E770E483E7CA
:1019F00097E30F94661286E790E40F94031207C0F2
:101A00000F94540B6233710581059105D8F28881DA
:101A10008F5F888355C0EAEFF0E483E480838CE233
:101A20008183DE011296ECEFF0E428E031E48D9141
:101A30008193E217F307D9F71092084121E04EE0B5
:101A400050E06AEF70E48DE19DE30F9466128881A7
:101A50008F5F88830F941A0733C00E943B9D8823B1
:101A600061F061E0C801E8DD0F941A078DE19DE3A4
:101A70000E94399B1882198223C00F940607813176
:101A80009742F0F060E0C801D7DD0F941A078DE1AE
:101A90009DE30E94399B1882198212C00F94060799
:101AA000883E934068F00E946C9B0F941A0718823E
:101AB000198206C08DE19DE30E94399B188219822C
:101AC000DF91CF911F910F91FF90EF900895EAEF72
:101AD000F0E42BE720832CE621832CE22283605D57
:101AE00063832DE72483158221E045E050E0BF01A8
:101AF0000F9466120E949129811109C021E045E0EE
:101B000050E06AEF70E483E797E30D94661208955E
:101B1000DF92EF92FF920F931F93CF93DF93009783
:101B200009F481C1EC01888190E08931910508F0C8
:101B300075C1FC018827E45EFD4F8F4F0D9423454E
:101B40008AE798E30E94179B88818F5F88836BC127
:101B5000EAEFF0E487E480838BE48183128221E062
:101B600042E050E0BF018AE798E30F946612888153
:101B70008F5F888383EF9FE30F94031222968CE09C
:101B8000FE0111928A95E9F74EC10F943D0BF12C9D
:101B900005E710E429C063EF7FE38AE798E30F9439
:101BA0001212F80180818130F9F48091F33F909115
:101BB000F43F059731F48091F53F813311F4FF2410
:101BC000F3940E94912981110BC04091F33F5091F1
:101BD000F43F21E065EF7FE383E797E30F9466121C
:101BE00083EF9FE30F9403120F94540B623371053C
:101BF0008105910580F2FF2021F088818F5F888325
:101C000012C188E088830FC1EAEFF0E487E48083A3
